:100000000C9419240C9446240C9446240C944624F5
:100010000C9446240C9446240C9446240C944624B8
:100020000C9446240C9446240C9446240C944624A8
:100030000C9446240C949CF60C9446240C94462470
:100040000C9446240C94AE2C0C9446240C94462418
:100050000C9446240C9446240C942EDD0C94F3F45A
:100060000C9446240C94A09A0C9446240C94462498
:100070000C9446240C9446240C9446240C94462458
:100080000C9446240C9446240C9446240C94462448
:100090000C9446240C9446240C9446240C9457EB60
:1000A0000C9446240C9446240C9446240C94462428
:1000B0000C9446240C9446240C9446240C94462418
:1000C0000C9446240C9446240C9446240C94462408
:1000D0000C9446240C9446240C9446240C944624F8
:1000E0000C944624084AD73B3BCE016E84BCBFFD2E
:1000F000C12F3D6C74319ABD56833DDA3D00C77FF8
:1001000011BED9E4BB4C3E916BAAAABE0000008090
:100110003F05A84CCDB2D44EB93836A9020C50B91F
:10012000918688083CA6AAAA2ABE000000803F4506
:10013000313A200045303A20005A3A2000593A20FE
:1001400000583A20004D53312C4D53322050696EE7
:10015000730A0024F404D9201BC40C5C0E9804C458
:10016000095F0265077101F405F900FB04B300485B
:10017000048700C10369005803550003034500BE0E
:10018000023A008402310053022A002902250004A9
:10019000022000E4011C00C8011900AF01170098FB
:1001A000011400840113007101100061011000515D
:1001B000010E0043010D0036010B002B010B002046
:1001C000010B00150109000C01090003010800FBE7
:1001D000000800F3000800EB000700E4000600DE62
:1001E000000600D8000600D2000600CC000500C7BB
:1001F000000500C2000500BD000400B9000400B500
:10020000000400B1000400AD000400A9000400A532
:10021000000300A20003009F0004009B000300985D
:100220000003009500020093000300900003008D7E
:100230000002008B00030088000200860002008498
:10024000000300810002007F0002007D0002007BAD
:1002500000020079000200770001007600020074BD
:1002600000020072000100710002006F0002006DC8
:100270000001006C0002006A0001006900020067D2
:1002800000010066000100650001006400020062D8
:1002900000010061000100600001005F0002005DDC
:1002A0000001005C0001005B0001005A00010059E0
:1002B00000010058000100570001005600010055E0
:1002C00000010054000100530000005300010052DF
:1002D00000010051000100500001004F0001004EDC
:1002E0000000004E0001004D0001004C0001004BD9
:1002F0000000004B0001004A0001004900010048D5
:1003000000000048000100470001004600000046D0
:1003100000010045000000450001004400010043C9
:1003200000000043000100420000004200010041C3
:1003300000000041000100400001003F0000003FBC
:100340000001003E0000003E0001003D0000003DB5
:100350000001003C0000003C0000003C0001003BAC
:100360000000003B0001003A0000003A00010039A3
:10037000000000390001003800000038000000389B
:100380000001003700000037000100360000003691
:100390000000003600010035000000350000003587
:1003A000000100340000003400000034000100337C
:1003B0000000003300000033000100320000003272
:1003C0000000003200010031000000310000003167
:1003D0000001003000000030000000300001002F5C
:1003E0000000002F0000002F0000002F0001002E51
:1003F0000000002E0000002E0001002D0000002D46
:100400000000002D0000002D0001002C0000002C39
:100410000000002C0000002C0001002B0000002B2D
:100420000000002B0000002B0001002A0000002A21
:100430000000002A0000002A000100290000002915
:100440000000002900000029000000290001002808
:1004500000000028000000280000002800000028FC
:1004600000010027000000270000002700000027EF
:1004700000000027000100260000002600000026E2
:1004800000000026000000260001002500000025D5
:1004900000000025000000250000002500000025C8
:1004A00000010024000000240000002400000024BB
:1004B00000000024000100230000002300000023AE
:1004C00000000023000000230000002300000023A0
:1004D0000001002200000022000000220000002293
:1004E0000000002200000022000100210000002185
:1004F0000000002100000021000000210000002178
:100500000000002100010020000000200000002069
:10051000000000200000002000000020000000205B
:10052000000000200001001F0000001F0000001F4D
:100530000000001F0000001F0000001F0000001F3F
:100540000001001E0000001E0000001E0000001E32
:1005500000000024F4D43050C38E20C2A240178281
:100560008B7011127A910D816CD90AA861E108C7CC
:10057000586607615143061E4B5D05C145A7041A25
:10058000411104093D9803713931034036DB02659E
:10059000339102D4305402802E1D02632CEE01757B
:1005A0002AC501B028A001102781018F2564012BE5
:1005B000244B01E0223401AC211F018D200D01806C
:1005C0001FFC00841EED00971DDF00B81CD200E662
:1005D0001BC600201BBC00641AB200B219A8000A96
:1005E00019A0006A189900D117910040178B00B527
:1005F00016840031167E00B31579003A157300C7D2
:10060000146F0058146A00EE136600881363002507
:10061000135E00C7125B006C12570015125400C124
:1006200011510070114F0021114B00D61049008D5F
:100630001047004610440002104200C00F400080E6
:100640000F3E00420F3C00060F3B00CB0E380093DC
:100650000E37005C0E3500270E3400F30D3200C15A
:100660000D3100900D3000600D2E00320D2D000573
:100670000D2C00D90C2B00AE0C2900850C29005C38
:100680000C2700350C27000E0C2600E80B2400C4B4
:100690000B2400A00B23007D0B23005A0B210039F3
:1006A0000B2100180B2000F80A1F00D90A1E00BBFE
:1006B0000A1E009D0A1D00800A1D00630A1C0047D7
:1006C0000A1B002C0A1B00110A1A00F7091A00DD88
:1006D000091900C4091900AB091900920917007B18
:1006E000091800630917004C091600360916002086
:1006F0000916000A091500F5081500E0081400CCD9
:10070000081400B8081400A4081400900813007D11
:100710000812006B08130058081200460812003433
:10072000081100230811001208110001081100F03F
:10073000071000E0071000D0071000C0071000B03D
:10074000070F00A107100091070E0083070F007428
:10075000070F0065070E0057070E0049070E003B04
:10076000070D002E070E0020070D0013070D0006D1
:10077000070D00F9060C00ED060D00E0060C00D494
:10078000060C00C8060C00BC060C00B0060C00A449
:10079000060B0099060C008D060B0082060B0077F5
:1007A000060B006C060B0061060A0057060B004C96
:1007B000060A0042060A0038060A002E060A00242D
:1007C000060A001A060A001006090007060A00FDBC
:1007D000050900F4050900EB050900E2050900D947
:1007E000050900D0050900C7050900BE050900B5C7
:1007F000050800AD050800A50509009C0508009442
:100800000508008C050800840508007C05080074B4
:100810000508006C050700650508005D0507005622
:100820000508004E05070047050700400508003889
:10083000050700310507002A050700230507001CEE
:10084000050600160507000F05070008050600024B
:10085000050700FB040600F5040700EE040600E8A7
:10086000040600E2040700DB040600D5040600CFFE
:10087000040600C9040600C3040600BD040600B750
:10088000040600B1040500AC040600A6040600A09E
:100890000405009B04060095040500900406008AE8
:1008A00004050085040500800406007A040500752F
:1008B000040500700405006B040500660405006172
:1008C0000405005C04050057040500520405004DB2
:1008D00004050048040500430405003E0404003AF2
:1008E00004050035040500300404002C040500272D
:1008F000040400230405001E0404001A0404001666
:10090000040500110404000D04040009040500049A
:1009100004040000040400FC030400F8030400F4D1
:10092000030400F0030400EC030400E8030400E403
:10093000030400E0030400DC030400D8030400D433
:10094000030400D0030400CC030400C8030300C563
:100950000303006563686F3A00656E6473746F70BB
:1009600073206869743A205A00205A3A00656E6410
:1009700073746F7073206869743A20590020593A73
:1009800000656E6473746F7073206869743A2058E0
:100990000020583A00656E6473746F707320686944
:1009A000743A20006563686F3A0020746F6F206CA2
:1009B0006F6E6720657874727573696F6E207072E0
:1009C0006576656E7465640020636F6C642065787D
:1009D00074727573696F6E2070726576656E74657A
:1009E00064007C3C3E5E2B3D3F2F5B5D3B2C2A220E
:1009F0005C0000060900FE06018902FE20FFFE07DA
:100A0000FE06FE0000000600070106060602008042
:100A10008080800080030303060103A0A0A00507D7
:100A2000070600FF5050F850F8505005090906001D
:100A3000FE2070A8A07028A870200608080600FFF5
:100A400040A84810204854080507070600FF60909A
:100A5000906098906801030306020380808002077B
:100A6000070602FF40808080808040020707060260
:100A7000FF8040404040408005050506000088504A
:100A8000F850880505050600002020F82020020403
:100A9000040602FEC0404080050101060002F80283
:100AA0000202060200C0C004060606010010102063
:100AB00040808004060606010060909090906003DC
:100AC000060606010040C0404040E004060606015C
:100AD000006090102040F0040606060100F020603F
:100AE0001010E005060606000010305090F81004C3
:100AF0000606060100F080E01010E004060606017C
:100B0000006080E0909060040606060100F010107E
:100B1000204040040606060100609060909060044A
:100B2000060606010060909070106002050506023E
:100B300000C0C000C0C00207070602FEC0C000C05F
:100B40004040800505050600001860806018050318
:100B500003060001F800F8050505060000C030088E
:100B600030C0040707060100609010604000400597
:100B700006060600007090A8B08070050606060004
:100B800000205088F88888050606060000F088F0E6
:100B90008888F0040606060100609080809060045A
:100BA0000606060100E090909090E004060606011B
:100BB00000F080E08080F0040606060100F080E08E
:100BC000808080040606060100609080B09060047A
:100BD00006060601009090F090909003060606012C
:100BE00000E040404040E0050606060000381010D6
:100BF00010906004060606010090A0C0A09090042A
:100C000006060601008080808080F005060606004A
:100C10000088D8A8A8888804060606010090D0B0ED
:100C200090909005060606000070888888887004F9
:100C30000606060100E09090E080800407070601A8
:100C4000FF609090D0B06010040606060100E090AE
:100C500090E09090040606060100609040209060AD
:100C6000050606060000F8202020202004060606BF
:100C7000010090909090906004060606010090900C
:100C800090F060600506060600008888A8A8D8884D
:100C90000506060600008850202050880506060636
:100CA0000000888850202020040606060100F0106D
:100CB000204080F0030606060100E080808080E08E
:100CC0000406060601008080402010100306060678
:100CD0000100E020202020E005030306000320504F
:100CE000880501010600FEF80202020602048040A7
:100CF00004040406010070909070040606060100CA
:100D00008080E09090E00404040601007080807010
:100D1000040606060100101070909070040404068A
:100D2000010060B0C070040606060100205040E0DB
:100D300040400406060601FE6090907010600406B4
:100D4000060601008080E0909090030606060100F0
:100D50004000C04040E00308080601FE200060207B
:100D60002020A0400406060601008080A0C0A090BC
:100D7000030606060100C040404040E005040406AA
:100D80000000D0A8A888040404060100E090909018
:100D9000040404060100609090600406060601FE4B
:100DA000E09090E080800406060601FE709090704E
:100DB0001010040404060100A0D08080040404067E
:100DC000010070C030E00406060601004040E0402B
:100DD000502004040406010090909070040404065E
:100DE00001009090606005040406000088A8A850E7
:100DF000040404060100906060900406060601FEEB
:100E0000909090709060040404060100F02040F07F
:100E100003070706010020404080404020010707EB
:100E20000602FF8080808080808003070706010023
:100E30008040402040408004020206010350A0FF91
:100E4000FFFFFFFFFFFFFFFFFFFFFFFFFFFFFFFFB2
:100E5000FFFFFFFFFFFFFFFFFFFFFFFFFFFFFFFFA2
:100E600000000006000701060606020080008080E0
:100E700080800406060601FF2070A0A070200507F0
:100E8000070600FF304840F04040F8050505060021
:100E900000A8508850A80506060600008850F820D3
:100EA000F8200107070602FF808080008080800410
:100EB00007070601FF708060906010E003010106E3
:100EC0000105A0060707060000788494A49484789E
:100ED00003050506010160A06000E00505050600A8
:100EE000002850A05028040303060100F01010044D
:100EF0000101060102F00607070600007884B4A489
:100F0000A48478040101060105F00403030601022C
:100F10006090600507070600FF2020F8202000F8F9
:100F200003050506010140A02040E0030505060178
:100F300001C0204020C002020206020440800405D5
:100F4000050601FF9090B0D08005060606000078E7
:100F5000E8E8682828010101060202800202020670
:100F600002FE408003050506010140C04040E00349
:100F7000050506010140A04000E00505050600004A
:100F8000A0502850A00508080600FF40C04050703F
:100F90003078100508080600FF40C040506808106F
:100FA000380508080600FFC0204030F030781004F3
:100FB00007070601002000206080906005070706F3
:100FC00000004020205070888805070706000010A8
:100FD0002020507088880507070600002050205008
:100FE0007088880507070600002850205070888800
:100FF0000507070600005000205070888805070785
:101000000600002050205070888805060606000063
:1010100078A0F0A0A0B80408080601FE60908080C7
:10102000906020400407070601004020F080E08027
:10103000F00407070601002040F080E080F004077C
:10104000070601002050F080E080F0040707060149
:10105000005000F080E080F00307070601008040A8
:10106000E0404040E00307070601002040E0404028
:1010700040E003070706010040A0E0404040E003D5
:101080000707060100A000E0404040E00506060614
:1010900000007048E848487004070706010050A0A7
:1010A00090D0B09090040707060100402060909017
:1010B0009060040707060100204060909090600453
:1010C0000707060100205060909090600407070613
:1010D000010050A060909090600407070601005046
:1010E0000060909090600505050600008850205033
:1010F000880408080601FF1070B0B0D0D0E080046A
:1011000007070601004020909090906004070706B2
:101110000100204090909090600407070601002095
:101120005090909090600407070601005000909046
:1011300090906005070706000010208850202020AE
:1011400004060606010080E09090E0800406060692
:1011500001006090A0A090A00407070601004020B5
:101160000070909070040707060100204000709006
:1011700090700407070601002050007090907004E2
:10118000070706010050A000709090700406060644
:101190000100500070909070040707060100205075
:1011A000207090907005040406000070A8B07804C8
:1011B00006060601FE7080807020400407070601C5
:1011C0000040200060B0C070040707060100204006
:1011D0000060B0C07004070706010020500060B036
:1011E000C070040606060100500060B0C07003071E
:1011F00007060100804000C04040E00307070601E9
:1012000000204000C04040E003070706010040A066
:1012100000C04040E0030606060100A000C04040B8
:10122000E00407070601003060107090906004072A
:101230000706010050A000E0909090040707060107
:1012400000402000609090600407070601002040E5
:101250000060909060040707060100205000609035
:10126000906004070706010050A0006090906004A1
:101270000606060100500060909060050505060016
:10128000002000F8002004040406010070B0D0E043
:1012900004070706010040200090909070040707A3
:1012A000060100204000909090700407070601009E
:1012B00020500090909070040606060100500090A7
:1012C0009090700409090601FE20400090909070F3
:1012D00090600408080601FE8080E09090E0808025
:1012E0000408080601FE500090909070906000067F
:1012F0000900FE070199032B20FFFE08FE07FE00F0
:101300000000060000010707060200808080808040
:101310000080030303060104A0A0A0050707060040
:10132000005050F850F85050050707060000207094
:10133000A07028702005070706000048A85020501C
:10134000A89005070706000040A0A040A8906801EB
:101350000303060204808080030707060100204083
:101360008080804020030707060100804020202065
:1013700040800505050600018850F85088050505E0
:101380000600012020F820200303030601FF60402F
:1013900080050101060003F80303030601FF40E096
:1013A0004005070706000008081020408080050758
:1013B000070600002050888888502005070706008F
:1013C000002060A0202020F8050707060000708894
:1013D00008304080F8050707060000F808103008BC
:1013E000887005070706000010305090F8101005AF
:1013F0000707060000F880B0C808887005070706D0
:101400000000304080B0C88870050707060000F86B
:1014100008101020404005070706000070888870FB
:1014200088887005070706000070889868081060B3
:101430000307070601FF40E0400040E040030707C4
:101440000601FF40E04000604080040707060100FD
:1014500010204080402010050303060002F800F829
:101460000407070601008040201020408005070780
:1014700006000070881020200020050707060000E5
:10148000708898A8B0807005070706000020508873
:1014900088F88888050707060000F0484870484823
:1014A000F0050707060000708880808088700507B7
:1014B00007060000F04848484848F00507070600BE
:1014C00000F88080F08080F8050707060000F880AB
:1014D00080F0808080050707060000708880809873
:1014E0008870050707060000888888F888888803C0
:1014F0000707060100E04040404040E005070706BE
:1015000000003810101010906005070706000088D2
:1015100090A0C0A09088050707060000808080800A
:101520008080F80507070600008888D8A888888882
:101530000507070600008888C8A898888805070757
:1015400006000070888888888870050707060000F4
:10155000F08888F08080800508080600FF70888881
:101560008888A87008050707060000F08888F0A0A2
:10157000908805070706000070888070088870054D
:101580000707060000F82020202020200507070676
:10159000000088888888888870050707060000880A
:1015A000888850505020050707060000888888A8C2
:1015B000A8D888050707060000888850205088882A
:1015C000050707060000888850202020200507070F
:1015D000060000F80810204080F803070706010005
:1015E000E08080808080E005070706000080804062
:1015F00020100808030707060100E0202020202013
:10160000E00503030600042050880501010600FFE1
:10161000F802020206020680400505050600007079
:10162000087888780507070600008080B0C888C859
:10163000B00505050600007088808870050707065C
:10164000000008086898889868050505060000707D
:1016500088F88070050707060000304840F04040D9
:10166000400507070600FE78888878088870050717
:10167000070600008080B0C8888888030707060135
:10168000004000C0404040E00409090601FE10008F
:1016900030101010909060050707060000808088C9
:1016A00090E09088030707060100C040404040409A
:1016B000E0050505060000D0A8A8A88805050506D0
:1016C0000000B0C888888805050506000070888875
:1016D00088700507070600FEB0C888C8B08080057E
:1016E00007070600FE68988898680808050505063B
:1016F0000000B0C88080800505050600007080707D
:1017000008F00507070600004040F040404830055B
:10171000050506000088888898680505050600000C
:1017200088885050200505050600008888A8A85024
:1017300005050506000088502050880507070600AB
:10174000FE88889868088870050505060000F8106E
:101750002040F8040707060100304020C020403038
:1017600001070706020080808080808080040707D0
:10177000060100C02040304020C0050303060004DD
:1017800048A89000000001000000000001000000D7
:101790000000010000000000010000000000010046
:1017A0000000000001000000000001000000000037
:1017B0000100000000000100000000000100000026
:1017C0000000010000000000010000000000010016
:1017D0000000000001000000000001000000000007
:1017E00001000000000001000000000001000000F6
:1017F00000000100000000000100000000000100E6
:1018000000000000010000000000010000000000D6
:1018100001000000000001000000000001000000C5
:1018200000000100000000000100000000000100B5
:1018300000000000010000000000010000000000A6
:10184000010000000000010000000000060000018F
:101850000707060200800080808080800507070659
:1018600000FF2078A0A0A078200507070600003020
:101870004840E04048B005050506000088705070FB
:10188000880508080600FF88885020F820202001DD
:101890000707060200808080008080800508080617
:1018A00000FF7080E09048380870030101060107CE
:1018B000A00507070600007088A8C8A8887004065D
:1018C000060601017090B05000F006050506000004
:1018D0002448904824040202060102F01004010189
:1018E000060103F00507070600007088E8C8C888ED
:1018F00070050101060007F803030306010440A078
:10190000400506060600002020F82020F804050502
:1019100006010360902040F0040505060103E01075
:101920006010E0020202060206408005060606007C
:10193000FF888888C8B08005070706000078E8E8B7
:10194000682828280101010602038002020206021B
:10195000FE408003050506010340C04040E0040648
:10196000060601016090906000F006050506000083
:1019700090482448900609090600FF40C04040E412
:101980000C143C040609090600FF40C04040E8145E
:1019900004081C0509090600FFC0204020C81828BB
:1019A0007808050707060000200020204088700501
:1019B00008080600004020708888F8888805080814
:1019C0000600001020708888F8888805080806003E
:1019D000002050708888F8888805080806000048AC
:1019E000B0708888F88888050808060000500070E4
:1019F0008888F888880508080600002050708888C4
:101A0000F888880607070600003C50909CF0909CE0
:101A10000509090600FE70888080808870204005D6
:101A2000080806000040F88080F08080F80508086B
:101A300006000010F88080F08080F8050808060095
:101A40000020F88080F08080F8050808060000502B
:101A5000F88080F08080F80308080601008040E0EC
:101A600040404040E00308080601002040E04040BC
:101A70004040E003080806010040A0E0404040402C
:101A8000E0030808060100A000E040404040E005F7
:101A90000707060000F04848E84848F0050808062F
:101AA0000000285088C8A898888805080806000003
:101AB000402070888888887005080806000010207B
:101AC0007088888888700508080600002050708893
:101AD0008888887005080806000028507088888863
:101AE0008870050808060000500070888888887093
:101AF00005050506000088502050880507070600E8
:101B000000709898A8C8C870050808060000402012
:101B10008888888888700508080600001020888852
:101B2000888888700508080600002050008888888A
:101B3000887005080806000050008888888888702A
:101B4000050808060000102088885020202005077E
:101B50000706000080F088F08080800507070600F7
:101B600000708890A09088B005080806000040200A
:101B700000700878887805080806000010200070BA
:101B8000087888780508080600002050007008785A
:101B900088780508080600002850007008788878C2
:101BA00005070706000050007008788878050808C7
:101BB0000600002050207008788878060505060089
:101BC0000078147C907C0507070600FE70888088EA
:101BD0007020400508080600004020007088F8804A
:101BE000700508080600001020007088F880700555
:101BF00008080600002050007088F880700507076C
:101C000006000050007088F8807003080806010084
:101C1000804000C0404040E00308080601004080CA
:101C200000C0404040E003080806010040A000C09A
:101C3000404040E0060A0A0600FEA4A800FC84809A
:101C4000808084FC060A0A0600FE549400FC84048A
:101C5000040484FC050808060000285000B0C88869
:101C60008888050808060000402000708888887071
:101C7000040A0A0602FE3040809090909090909066
:101C8000040A0A0600FEC020109090909090909058
:101C9000060707060001448C8C8480403C06070739
:101CA00006000188C4C4840408F005050506000187
:101CB0002000F8002005080806000040F0C88888C9
:101CC000987810050808060000E0F8888888888859
:101CD000F80505050600012030F830200508080643
:101CE00000002070F820202020E00509090600FFF0
:101CF0002070A8A8B8888850200509090600FFE0D0
:101D000080C0B0A8A83028280509090600FFF8A857
:101D10008888888888A8F8050A0A0600FE2050509E
:101D2000505088A8A8887000000000000000000043
:101D30000000007FFFE00000000000000000000045
:101D400000007000E0000000000000000000000043
:101D500000630C60000000000000000000000000B4
:101D6000470E200000000000000000000000004FAF
:101D70000F200000000000000000000000005F0FC6
:101D8000A00000000000000000000000005E07A0AE
:101D90007F80003FC0003FC000410400406020FB46
:101DA000C00079E00079E00020820040F020F3C01C
:101DB0000076E00076E00020820040F020EBC000DA
:101DC0007EE0007EE0004104004060207B80003D1A
:101DD000C00039C0008208005E07A07B80003BC0C5
:101DE000003EC0010410005F0FA0FBC00077E000C0
:101DF00076E0010410004F0F20FBC00070E0007976
:101E0000E000820800470E20FFC0007FE0007FE076
:101E100000410400630C603F00001F80001F800031
:101E20000000007000E01E00000F00000F0001FF26
:101E3000FF807FFFE00C0000060000060001FFFFAE
:101E40008000000000000000000000000000000012
:101E50007FFFE000000000000000000000000070B4
:101E600000E000000000000000000000000061F839
:101E70006000000000000000000000000041F820A9
:101E800000000000000000000000000040F0200002
:101E90000000000000000000000000406020000082
:101EA000000000000000000000005801A07F80003A
:101EB0003FC0003FC0004104005C63A0FBC000794C
:101EC000E00079E0002082005EF7A0F3C00076E039
:101ED0000076E0002082005EF7A0EBC0007EE0000C
:101EE0007EE0004104005C63A07B80003DC00039BF
:101EF000C0008208005801A07B80003BC0003EC0AB
:101F000001041000406020FBC00077E00076E00193
:101F100004100040F020FBC00070E00079E0008277
:101F2000080041F820FFC0007FE0007FE00041048E
:101F30000061F8603F00001F80001F80000000006B
:101F40007000E01E00000F00000F0001FFFF807F07
:101F5000FFE00C0000060000060001FFFF8000000B
:101F6000005900B02000B02000B02000B020002DAB
:101F70002D3A2D2D004E6F2043617264005072691E
:101F80006E742066726F6D2053440053746F70201E
:101F90005072696E7400526573756D652050726978
:101FA0006E74005061757365205072696E740043E1
:101FB0006F6E74726F6C0050726570617265005460
:101FC000756E6500496E666F2073637265656E009D
:101FD000F92E2E004D61696E004D3234004D3233C2
:101FE000202573004D383420582059205A204500B0
:101FF000526573746F7265204661696C73616665C2
:10200000004C6F6164206D656D6F72790053746F61
:102010007265206D656D6F7279004D6F74696F6EBA
:102020000054656D7065726174757265004D61690B
:102030006E004531737470732F6D6D00453173748C
:1020400070732F6D6D004573746570732F6D6D0027
:102050004573746570732F6D6D005A73746570737A
:102060002F6D6D005A73746570732F6D6D00597309
:10207000746570732F6D6D005973746570732F6D77
:102080006D005873746570732F6D6D0058737465AF
:1020900070732F6D6D00412D7265747261637400F1
:1020A000412D7265747261637400416D61782065C1
:1020B00000416D6178206500416D6178207A0041B2
:1020C0006D6178207A00416D6178207900416D6101
:1020D00078207900416D6178207800416D61782029
:1020E00078005654726176206D696E0056547261A4
:1020F00076206D696E00566D696E00566D696E00D2
:10210000566D6178206500566D6178206500566DCA
:102110006178207A00566D6178207A00566D61787A
:10212000207900566D6178207900566D61782078AD
:1021300000566D617820780056652D6A65726B00D7
:1021400056652D6A65726B00567A2D6A65726B0052
:10215000567A2D6A65726B005678792D6A65726BB6
:10216000005678792D6A65726B00416363656C0077
:10217000416363656C005A204F6666736574005A4C
:10218000204F666673657400436F6E74726F6C00E7
:10219000507265686561742041425320436F6E66DA
:1021A000005072656865617420504C4120436F6E29
:1021B00066005049442D43005049442D4300504986
:1021C000442D44005049442D44005049442D4900B9
:1021D0005049442D49005049442D50005049442D48
:1021E0005000200220466163740020022046616393
:1021F00074002002204D6178002002204D6178009B
:102200002002204D696E002002204D696E004F664D
:1022100066004F6E20004F6666004F6E20004175CD
:10222000746F74656D700046616E207370656564CF
:102230000046616E2073706565640042656400420B
:102240006564004E6F7A7A6C6532004E6F7A7A6CF4
:102250006532004E6F7A7A6C65004E6F7A7A6C65E3
:1022600000436F6E74726F6C0053746F7265206DF3
:10227000656D6F72790042656400426564004E6F5F
:102280007A7A6C65004E6F7A7A6C650046616E20D2
:1022900073706565640046616E20737065656400E7
:1022A00054656D70657261747572650053746F72F8
:1022B00065206D656D6F72790042656400426564EA
:1022C000004E6F7A7A6C65004E6F7A7A6C650046C4
:1022D000616E2073706565640046616E2073706581
:1022E00065640054656D7065726174757265004D4A
:1022F0006F7665204178697300436F6F6C646F7708
:102300006E005072656865617420414253005072DE
:10231000656865617420504C410047323800417552
:10232000746F20486F6D65004D38340044697361E7
:10233000626C65205374657070657273004D6169DD
:102340006E004D6F766520302E316D6D004D6F76CD
:102350006520316D6D004D6F76652031306D6D00FB
:10236000507265706172650045787472756465724B
:10237000004D6F7665205A004D6F76652059004DEF
:102380006F76652058004D6F76652041786973003F
:102390004578747275646572005A00590058004D92
:1023A000363030004368616E67652066696C616D28
:1023B000656E7400466C6F7700466C6F77004661FF
:1023C0006E2073706565640046616E20737065658C
:1023D000640042656400426564004E6F7A7A6C6501
:1023E00032004E6F7A7A6C6532004E6F7A7A6C6585
:1023F000004E6F7A7A6C65005370656564005370A7
:10240000656564004D61696E0043617264207265A8
:102410006D6F766564004361726420696E736572E6
:10242000746564000000000000000000000000006F
:10243000000000000000000000000000000000009C
:10244000000000000000000C000000000000000C74
:102450000000000000000012000000000000002347
:102460000000000000000021000000000000004CFF
:10247000800000000000005E80000000000000926C
:1024800040000000000000A1400000000000012109
:10249000200000000000027F900000000000020009
:1024A00010000000000007FFF8000000000004001A
:1024B0000800000000000800040000000000080000
:1024C0000600000000001000020000000000301EA6
:1024D000010000000000207F81000000000041FF9B
:1024E000E0800000000043FCF08000000000873B1B
:1024F0007840000000018EDBFC60000000010FEB63
:10250000CC20000000021FEDB610000000021FDE0C
:10251000B6100000000439CD7F080000000436E04A
:10252000FF08000000087EC0BB84000000187F0088
:102530005D86000000107FC0ED82000000203CC0DE
:102540007301000000203B337F01000000701BE797
:102550007E03800000C81DEEDE04C00000880FDE90
:10256000DC04400001240FDF3C092000012607DBCA
:10257000F8192000027203E7F0139000025101FFE6
:10258000E02290000489007F802448000904801E16
:10259000004824000BFE400000DFF4001000400063
:1025A000008002001FFFFFFFFFFFFE000000000091
:1025B000000000000000000000000000000000001B
:1025C000000000001022103C3C0E1F0010221004DE
:1025D00022110400102210082211040010221008F9
:1025E0003C110400102210102211040010221020AF
:1025F000221104001E1C1E3C3C0E040000000000C2
:1026000000000000000000000000000000000000CA
:1026100000000000000000000000000000000000BA
:1026200000000000000000000000000000000000AA
:10263000000000000000000000000000000000009A
:10264000000000000000000000000000000000008A
:10265000000000000000000000000000000000007A
:1026600000006563686F3A0048617264636F646577
:10267000642044656661756C742053657474696E7A
:102680006773204C6F616465640053746F72656496
:102690002073657474696E677320726574726965FE
:1026A000766564002044002049002020204D33300E
:1026B000312050005049442073657474696E67730B
:1026C0003A00205A0020590020204D323036205840
:1026D00000486F6D65206F666673657420286D6DA8
:1026E000293A00204500205A0020580020420020AE
:1026F000540020204D323035205300416476616E05
:10270000636564207661726961626C65733A205317
:102710003D4D696E20666565647261746520286D43
:102720006D2F73292C20543D4D696E207472617693
:10273000656C20666565647261746520286D6D2F17
:1027400073292C20423D6D696E696D756D2073652E
:10275000676D656E742074696D6520286D73292C12
:1027600020583D6D6178696D756D205859206A65F6
:10277000726B20286D6D2F73292C20205A3D6D61BE
:1027800078696D756D205A206A65726B20286D6DB1
:102790002F73292C2020453D6D6178696D756D2062
:1027A00045206A65726B20286D6D2F7329002054B7
:1027B0000020204D323034205300416363656C6546
:1027C000726174696F6E3A20533D616363656C6535
:1027D000726174696F6E2C20543D7265747261630E
:1027E0007420616363656C65726174696F6E00204B
:1027F0004500205A0020590020204D323031205809
:10280000004D6178696D756D20416363656C65721B
:102810006174696F6E20286D6D2F7332293A002024
:102820004500205A0020590020204D3230332058D6
:10283000004D6178696D756D2066656564726174BF
:10284000657320286D6D2F73293A002045310020D3
:102850004500205A0020590020204D3932205800D0
:1028600053746570732070657220756E69743A00D8
:1028700053657474696E67732053746F7265640076
:102880006563686F3A004572726F723A0053544F35
:10289000505045442E20005072696E74657220734A
:1028A000746F707065642064756520746F20657244
:1028B000726F72732E204669782074686520657285
:1028C000726F7220616E6420757365204D393939DD
:1028D00020746F20726573746172742E20285465A1
:1028E0006D706572617475726520697320726573AD
:1028F00065742E2053657420697420616674657256
:102900002072657374617274696E6729004B494C5B
:102910004C45442E20005072696E746572206861C7
:102920006C7465642E206B696C6C28292063616C63
:102930006C656421006F6B00526573656E643A20AC
:10294000002200556E6B6E6F776E20636F6D6D6148
:102950006E643A2022004368616E67652066696C88
:10296000616D656E74006C636420636F6E74726178
:1029700073742076616C75653A20007A5F6D696EBC
:102980003A2000795F6D696E3A2000785F6D696E5C
:102990003A20005A3A00593A0020436F756E74206D
:1029A000583A2000453A005A3A00593A00583A003D
:1029B0004649524D574152455F4E414D453A4D6152
:1029C000726C696E2056313B20537072696E74656B
:1029D000722F6772626C206D617368757020666F0C
:1029E000722067656E36204649524D574152455F09
:1029F00055524C3A687474703A2F2F7777772E6D52
:102A0000656E64656C2D70617274732E636F6D20DA
:102A100050524F544F434F4C5F56455253494F4EBF
:102A20003A312E30204D414348494E455F5459506C
:102A3000453A54415A2045585452554445525F43F3
:102A40004F554E543A3120555549443A3030303084
:102A5000303030302D303030302D303030302D307F
:102A60003030302D30303030303030303030303069
:102A70000A0054415A204F66662E0054415A205293
:102A8000656164792E0042656420646F6E652E0076
:102A900020423A0020453A00543A004265642048FA
:102AA000656174696E672E0048656174696E6720A0
:102AB000646F6E652E0020573A0020453A00543A64
:102AC0000048656174696E672E2E2E002042403AE0
:102AD0000020403A00202F003A00205400202F0010
:102AE00020423A00202F006F6B20543A00256920C5
:102AF0006D696E2C2025692073656300456E642026
:102B000066696C65206C69737400426567696E2044
:102B100066696C65206C697374004E6F206D6F760A
:102B2000652E00526573756D696E67207072696EEF
:102B300074005761697420666F7220757365722E18
:102B40002E2E00536C6565702E2E2E0000009543CE
:102B50000080894300007A43FFFFFF00000000006F
:102B60000000000000000000000000000000000065
:102B7000000000000095430080894300007A430074
:102B800000A0400000A04000008040256920686F40
:102B9000757273202569206D696E757465730044C4
:102BA0006F6E65207072696E74696E672066696CFD
:102BB000650053544F505045442E20005072696EAA
:102BC0007465722073746F7070656420647565201D
:102BD000746F206572726F72732E2046697820744C
:102BE0006865206572726F7220616E64207573650E
:102BF000204D39393920746F207265737461727495
:102C00002E202854656D7065726174757265206937
:102C1000732072657365742E205365742069742067
:102C200061667465722072657374617274696E672F
:102C300029006F6B004E6F204C696E65204E756DDC
:102C4000626572207769746820636865636B737569
:102C50006D2C204C617374204C696E653A20004ED7
:102C60006F20436865636B73756D207769746820A6
:102C70006C696E65206E756D6265722C204C617397
:102C800074204C696E653A2000636865636B7375E8
:102C90006D206D69736D617463682C204C61737471
:102CA000204C696E653A20004C696E65204E756D4A
:102CB000626572206973206E6F74204C617374209A
:102CC0004C696E65204E756D6265722B312C204CFF
:102CD000617374204C696E653A20004D31313000CB
:102CE000446F6E6520736176696E672066696C65F6
:102CF0002E006F6B004D3239002020506C616E6EDB
:102D0000657242756666657242797465733A200031
:102D10002046726565204D656D6F72793A200046D8
:102D20006562203230203230313500436F6D70697A
:102D30006C65643A200028416C657068204F626AB7
:102D4000656374732C20496E632C2054415A2020F3
:102D5000636F6E6669672900207C20417574686F17
:102D6000723A200046656220323020323031352000
:102D700031303A35353A303700204C617374205584
:102D80007064617465643A2000312E302E30004D3D
:102D900061726C696E200020536F66747761726592
:102DA00020526573657400205761746368646F67AF
:102DB000205265736574002042726F776E206F75C4
:102DC00074205265736574002045787465726E6175
:102DD0006C20526573657400506F77657255700092
:102DE0007374617274002200656E717565696E6737
:102DF0002022002200656E717565696E67202200D1
:102E00004D383420582059205A2045006563686F9A
:102E10003A0043616E6E6F7420656E746572207344
:102E200075626469723A20004D3234004D323320AD
:102E30002573006175746F25692E67004572726F86
:102E4000723A006572726F722077726974696E6788
:102E500020746F2066696C65004E6F7420534420A7
:102E60007072696E74696E67002F0053442070722F
:102E7000696E74696E67206279746520002E004463
:102E8000656C6574696F6E206661696C65642C2081
:102E900046696C653A200046696C652064656C651E
:102EA0007465643A002E006F70656E206661696C0F
:102EB00065642C2046696C653A2000577269746914
:102EC0006E6720746F2066696C653A20002E006F73
:102ED00070656E206661696C65642C2046696C655E
:102EE0003A20002E006F70656E206661696C656423
:102EF0002C2046696C653A200046696C6520736534
:102F00006C6563746564002053697A653A200046F5
:102F1000696C65206F70656E65643A20002E006FE5
:102F200070656E206661696C65642C2046696C650D
:102F30003A20004E6F772066726573682066696C70
:102F4000653A20004E6F7720646F696E672066696E
:102F50006C653A20002220706F730022207061722D
:102F6000656E743A2200535542524F5554494E45AE
:102F70002043414C4C207461726765743A2200749E
:102F80007279696E6720746F2063616C6C20737551
:102F9000622D67636F64652066696C65732077696D
:102FA000746820746F6F206D616E79206C65766532
:102FB0006C732E204D4158206C6576656C206973CA
:102FC0003A0053442063617264206F6B006F706538
:102FD0006E526F6F74206661696C656400766F6C09
:102FE000756D652E696E6974206661696C65640033
:102FF000534420696E6974206661696C0045727281
:103000006F723A004572723A204D415854454D5006
:10301000204245440054656D706572617475726537
:1030200020686561746564206265642073776974E3
:1030300063686564206F66662E204D415854454D87
:1030400050207472696767657265642021210045AC
:1030500072723A204D494E54454D50003A20457801
:10306000747275646572207377697463686564202F
:103070006F66662E204D494E54454D50207472693E
:103080006767657265642021004572723A204D4180
:103090005854454D50003A204578747275646572F5
:1030A000207377697463686564206F66662E204DAF
:1030B000415854454D502074726967676572656464
:1030C000202100202D20496E76616C69642065788E
:1030D000747275646572206E756D62657220210070
:1030E0001000AD0330016A0150022B0170030A0188
:1030F0009004F500B005E500D006D800F007CE003A
:103100001009C500300ABE00500BB700700CB100AA
:10311000900DAB00B00EA600D00FA200F0109D00E5
:1031200010129900301395005014920070158E0003
:1031300090168B00B0178700D0188400F01981001A
:10314000101B7E00301C7B00501D7900701E760025
:10315000901F7300B0207000D0216E00F0226B0031
:103160001024690030256600502663007027610036
:1031700090285E00B0295C00D02A5900F02B560040
:10318000102D5400302E5100502F4E0070304B0047
:1031900090314800B0324500D0334200F0343E0058
:1031A00010363B00303737005038330070392E006E
:1031B000903A2900B03B2300D03C1B00F03D1100A9
:1031C000103F0100F03F0000504944204175746FEA
:1031D00074756E652066696E697368656421205038
:1031E000757420746865204B702C204B6920616ECB
:1031F00064204B6420636F6E7374616E7473206916
:103200006E746F20436F6E66696775726174696F63
:103210006E2E6800504944204175746F74756E6558
:10322000206661696C6564212074696D656F7574D1
:103230000020403A006F6B20543A006F6B20423AF6
:1032400000504944204175746F74756E6520666145
:10325000696C6564212054656D7065726174757266
:103260006520746F6F206869676800204B643A209E
:1032700000204B693A2000204B703A200020436C1C
:10328000617369632050494420002054753A20003E
:10329000204B753A2000206D61783A2000206D693E
:1032A0006E3A200020643A200020626961733A205F
:1032B00000000A1400FC0D024A049920FFFC10FCD7
:1032C0000DFC0000000A0010020D0D0A0400C0C031
:1032D000C0C0C0C0C0C0C0C000C0C00604040A0254
:1032E00009CCCCCC48090B160A01011B001B001BA2
:1032F000007F80360036003600FF006C006C006CEA
:1033000000080D0D0A0100187EDBD8D8D87E1B1BE3
:103310001BDB7E18090C180A01007300DB00DE00BD
:1033200076000C000C001800180037003D806D80FE
:103330006700090D1A0A010038006C006C006C006F
:10334000780030007000D800CD80C700C600EF00C4
:1033500079800205050A0408C0C0C0C080050D0DB3
:103360000A030018306060C0C0C0C0C06060301880
:10337000050D0D0A0200C0603030181818181830FA
:103380003060C00807070A010366663CFF3C6666BA
:103390000807070A0103181818FF18181804030370
:1033A0000A03FF7070E00801010A0106FF0303032E
:1033B0000A0400E0E0E0070C0C0A020006060C0C10
:1033C000181830306060C0C0080D0D0A0100183CAC
:1033D0006666C3C3C3C3C366663C18080D0D0A0105
:1033E00000183878D81818181818181818FF080D69
:1033F0000D0A01003C66C3C30303061C3060C0C055
:10340000FF080D0D0A01003C66C3C303061C06033A
:10341000C3C3663C080D0D0A010002060E1E366687
:10342000C6C6FF06060606080D0D0A0100FFC0C04D
:10343000C0C0DCE6030303C3663C080D0D0A0100AF
:103440003C66C2C0C0DCE6C3C3C3C3663C080D0D06
:103450000A0100FF030306060C0C181830306060E8
:10346000080D0D0A01003C66C3C3C3663C66C3C3B6
:10347000C3663C080D0D0A01003C66C3C3C3C367A5
:103480003B030343663C0308080A0400E0E0000035
:103490000000E0E00409090A03FF7070000000006A
:1034A0007070E0070D0D0A010002060C183060C0B4
:1034B0006030180C06020806060A0103FF0000002F
:1034C00000FF070D0D0A020080C06030180C060CCA
:1034D000183060C080080D0D0A01003C66C3C3C3EC
:1034E000060C181818001818080D0D0A01003C6683
:1034F000C3CFDFDBDBDBDECCC0633E080D0D0A0192
:1035000000183C6666C3C3C3FFC3C3C3C3C3080D6F
:103510000D0A0100F8CCC6C6C6CCFCC6C3C3C3C6E0
:10352000FC080D0D0A01003C66C3C0C0C0C0C0C08D
:10353000C0C3663C080D0D0A0100FCC6C3C3C3C36B
:10354000C3C3C3C3C3C6FC080D0D0A0100FFC0C03E
:10355000C0C0C0FCC0C0C0C0C0FF080D0D0A010043
:10356000FFC0C0C0C0C0FCC0C0C0C0C0C0080D0DFE
:103570000A01003C66C3C0C0C0CFC3C3C3C3673D1C
:10358000080D0D0A0100C3C3C3C3C3C3FFC3C3C334
:10359000C3C3C3080D0D0A0100FF18181818181826
:1035A0001818181818FF090D1A0A01001F800600C4
:1035B0000600060006000600060006000600C6001B
:1035C000C6006C003800080D0D0A0100C3C3C6C652
:1035D000CCCCF8CCCCC6C6C3C3080D0D0A0100C0C4
:1035E000C0C0C0C0C0C0C0C0C0C0C0FF080D0D0A70
:1035F0000100C3C3E7E7FFDBDBDBDBC3C3C3C308F7
:103600000D0D0A0100C3E3E3F3F3DBDBCFCFC7C744
:10361000C3C3080D0D0A01003C66C3C3C3C3C3C3C3
:10362000C3C3C3663C080D0D0A0100FCC6C3C3C377
:10363000C3C6FCC0C0C0C0C0080E0E0A01FF3C6675
:10364000C3C3C3C3C3C3C3DBCF663E03080D0D0AA8
:103650000100FCC6C3C3C3C3C6FCCCC6C6C3C308F3
:103660000D0D0A01003C66C3C0C0603C060303C3E5
:10367000663C080D0D0A0100FF18181818181818D4
:103680001818181818080D0D0A0100C3C3C3C3C3C6
:10369000C3C3C3C3C3C3663C080D0D0A0100C3C343
:1036A000C3C36666663C3C3C181818080D0D0A0139
:1036B00000C3C3C3C3C3DBDBDBDBE7E7C3C3080D66
:1036C0000D0A0100C3C366663C3C183C3C6666C3F9
:1036D000C3080D0D0A0100C3C366663C3C181818E8
:1036E00018181818080D0D0A0100FF0303060C0C2A
:1036F00018303060C0C0FF060D0D0A0200FCC0C0CB
:10370000C0C0C0C0C0C0C0C0C0FC070C0C0A0200D2
:10371000C0C06060303018180C0C0606060D0D0A8B
:103720000200FC0C0C0C0C0C0C0C0C0C0C0CFC0813
:1037300004040A0109183C66C30901020A01FFFFDB
:10374000800403030A030AC060300808080A010065
:103750003E63037FC3C3C37D080D0D0A0100C0C0D3
:10376000C0C0C0DCE6C3C3C3C3E6DC0808080A0166
:10377000003E63C0C0C0C0633E080D0D0A010003D7
:10378000030303033B67C3C3C3C3673B0808080ABB
:1037900001003C66C3FFC0C0633E080D0D0A010076
:1037A0001E33333030FC30303030303030080C0CC9
:1037B0000A01FC7DC7C6C6C67CC07EC3C3C37E08E3
:1037C0000D0D0A0100C0C0C0C0C0DCE6C3C3C3C346
:1037D000C3C3080B0B0A0100181800781818181832
:1037E0001818FF070F0F0A02FC0606001E06060641
:1037F00006060606C6C6C67C080D0D0A0100C0C036
:10380000C0C0C0C6CCD8F0F8CCC6C3080D0D0A01A4
:1038100000781818181818181818181818FF080819
:10382000080A0100B6FFDBDBDBDBDBDB0808080A8C
:103830000100DCE6C3C3C3C3C3C30808080A010010
:103840003C66C3C3C3C3663C080C0C0A01FCDCE63F
:10385000C3C3C3C3E6DCC0C0C0C0080C0C0A01FC73
:103860003B67C3C3C3C3673B030303030808080ADA
:103870000100DE736060606060600808080A010093
:103880007EC3C07E0303C37E080B0B0A01003030E9
:1038900030FC3030303030331E0808080A0100C3D5
:1038A000C3C3C3C3C3673B0808080A0100C3C36698
:1038B000663C3C18180808080A0100C3C3C3DBDBD8
:1038C000DBFF660808080A0100C3663C18183C665E
:1038D000C3080C0C0A01FCC3C3C3C3C3C3673B03C7
:1038E000C3663C0708080A0200FE060C183060C0D8
:1038F000FE080D0D0A01000F1818181818F01818F6
:103900001818180F020D0D0A0400C0C0C0C0C0C0B6
:10391000C0C0C0C0C0C0C0080D0D0A0100F018181A
:103920001818180F1818181818F00803030A010AB5
:1039300073DBCEFFFFFFFFFFFFFFFFFFFFFFFFFF78
:10394000FFFFFFFFFFFFFFFFFFFFFFFFFFFFFFFF87
:10395000FFFFFFFF0000000A0010020D0D0A040027
:10396000C0C000C0C0C0C0C0C0C0C0C0C0070C0C38
:103970000A010018183C66C2C0C0C2663C1818098B
:103980000C180A01001E003300330030003000FC28
:1039900000300030003000F800AD80E70009091267
:1039A0000A00018080DD807F006300630063007F88
:1039B00000DD808080080B0B0A010081C3663C7E1D
:1039C000187E18181818020D0D0A0400C0C0C0C0D7
:1039D000C0000000C0C0C0C0C0080D0D0A01003CFE
:1039E00066C66078CC66331E0663663C0602020A31
:1039F000020BCCCC080B0B0A01003C66C3BDA5A191
:103A0000A5BDC3663C0809090A01043E43037FC300
:103A1000C37D00FF090B160A000004800D801B0007
:103A200036006C00D8006C0036001B000D8004804E
:103A30000804040A0104FFFF03030601010A020649
:103A4000FC080B0B0A01003C66C3BDA5BDA9ADC3B4
:103A5000663C0801010A010DFF0606060A0207304E
:103A600078CCCC78300807070A01021818FF18181C
:103A700000FF0507070A020670D8183060C0F80575
:103A800007070A020670D8183018D8700403030A12
:103A9000030A3060C0070A0A0A01FDC6C6C6C6C6C8
:103AA000EEFAC0C0C0080D0D0A01007FFFFBFBFB52
:103AB0007B1B1B1B1B1B1B1B0303030A0405E0E0F2
:103AC000E00504040A02FC3018D8700407070A0253
:103AD0000660E060606060F00709090A0104386C64
:103AE000C6C6C66C3800FE090B160A01009000D845
:103AF000006C0036001B000D801B0036006C00D8E7
:103B0000009000080C0C0A010140C04142E4081278
:103B1000264A9E0202080C0C0A010140C04142E400
:103B20000816294182040F080C0C0A0101E01061FB
:103B300012E40812264A9F0202080D0D0A0100181D
:103B400018001818183060C3C3C3663C080F0F0A6A
:103B5000010060301800183C66C3C3C3FFC3C3C371
:103B6000C3080F0F0A0100060C1800183C66C3C3F7
:103B7000C3FFC3C3C3C3080F0F0A0100183C66008C
:103B8000183C66C3C3C3FFC3C3C3C3080F0F0A01F6
:103B900000327E4C00183C66C3C3C3FFC3C3C3C31B
:103BA000080F0F0A0100666600183C6666C3C3C3AF
:103BB000FFC3C3C3C30810100A01003C66663C0083
:103BC000183C66C3C3C3FFC3C3C3C3080D0D0A01BA
:103BD000001F3C6C6CCCCCFFCCCCCCCCCCCF081137
:103BE000110A01FC3C66C3C0C0C0C0C0C0C0C366EF
:103BF0003C180C6C38080F0F0A010060301800FFE9
:103C0000C0C0C0C0FCC0C0C0C0FF080F0F0A010088
:103C10000C183000FFC0C0C0C0FCC0C0C0C0FF084E
:103C20000F0F0A0100183C6600FFC0C0C0C0FCC0F6
:103C3000C0C0C0FF080F0F0A010066660000FFC089
:103C4000C0C0C0FCC0C0C0C0FF060F0F0A020060A9
:103C5000301800FC303030303030303030FC060F5F
:103C60000F0A020018306000FC3030303030303045
:103C70003030FC060F0F0A02003078CC00FC3030E8
:103C800030303030303030FC060F0F0A0200CCCC20
:103C900000FC30303030303030303030FC090D1A1C
:103CA0000A00007E0063006180618061806180F9AC
:103CB00080618061806180618063007E00080F0FF9
:103CC0000A0100327E4C00C3E3F3F3DBDBCFCFC746
:103CD000C3C3080F0F0A010030180C003C66C3C3B1
:103CE000C3C3C3C3C3663C080F0F0A01000C1830DE
:103CF000003C66C3C3C3C3C3C3C3663C080F0F0AFB
:103D00000100183C66003C66C3C3C3C3C3C3C3669B
:103D10003C080F0F0A0100327E4C003C66C3C3C34F
:103D2000C3C3C3C3663C080F0F0A01006666003CAC
:103D300066C3C3C3C3C3C3C3C3663C0708080A0141
:103D40000082C66C38386CC682080F0F0A01FF016A
:103D50003E66C7C7CBCBCBD3D3D3E3667C80080FFB
:103D60000F0A010030180C00C3C3C3C3C3C3C3C3CD
:103D7000C3663C080F0F0A01000C183000C3C3C310
:103D8000C3C3C3C3C3C3663C080F0F0A0100183C7A
:103D90006600C3C3C3C3C3C3C3C3C3663C080F0F1A
:103DA0000A0100666600C3C3C3C3C3C3C3C3C3C39E
:103DB000663C080F0F0A01000C183000C3C366668A
:103DC0003C3C1818181818070D0D0A0200C0C0C096
:103DD000FCC6C6C6C6C6FCC0C0C0080D0D0A0100A0
:103DE0001C36636366EC6C66636363666C080C0C7C
:103DF0000A010030180C007EC3037FC3C3C37D08D3
:103E00000C0C0A01000C1830007EC3037FC3C3C32F
:103E10007D080C0C0A0100183C66007EC3037FC3BA
:103E2000C3C37D080C0C0A0100327E4C007EC30324
:103E30007FC3C3C37D080B0B0A01006666007EC307
:103E4000037FC3C3C37D080D0D0A01003C66663CB9
:103E5000007EC3037FC3C3C37D0808080A01007640
:103E60009B1B1E78D8D96E080C0C0A01FC3E63C05F
:103E7000C0C0C0633E180C6C38080C0C0A0100600E
:103E80003018003C66C3FFC0C0633E080C0C0A013A
:103E900000060C18003C66C3FFC0C0633E080C0C53
:103EA0000A0100183C66003C66C3FFC0C0633E08C0
:103EB0000B0B0A01006666003C66C3FFC0C0633E90
:103EC000080C0C0A0100603018007818181818182F
:103ED00018FF080C0C0A01000C183000781818188C
:103EE000181818FF080C0C0A0100183C6600781816
:103EF0001818181818FF080B0B0A010066660078DE
:103F0000181818181818FF080D0D0A010088D87025
:103F100070D88C3E67C3C3C3663C080C0C0A010012
:103F2000327E4C00DCE6C3C3C3C3C3C3080C0C0A17
:103F30000100603018003C66C3C3C3C3663C080C74
:103F40000C0A0100060C18003C66C3C3C3C3663CE0
:103F5000080C0C0A0100183C66003C66C3C3C3C3CE
:103F6000663C080C0C0A0100327E4C003C66C3C360
:103F7000C3C3663C080B0B0A01006666003C66C3BF
:103F8000C3C3C3663C080A0A0A010118180000FFEF
:103F9000FF00001818080A0A0A01FF013E66CBCB91
:103FA000D3D3667C80080C0C0A010030180C00C3C7
:103FB000C3C3C3C3C3673B080C0C0A0100060C183B
:103FC00000C3C3C3C3C3C3673B080C0C0A0100187A
:103FD0003C6600C3C3C3C3C3C3673B080B0B0A01E2
:103FE00000666600C3C3C3C3C3C3673B0810100A9F
:103FF00001FC0C183000C3C3C3C3C3C3673B03C376
:10400000663C0711110A02FCC0C0C0C0C0C0F8CC99
:10401000C6C6C6CCF8C0C0C0C0080F0F0A01FC66F7
:104020006600C3C3C3C3C3C3673B03C3663C010588
:104030000800FF060121023520FFFF07FF06FF09E8
:104040000050221656808080800080153353A0A037
:10405000A00257575050F850F85050025757207050
:10406000A07028702013355580A040A0200247572B
:1040700040A0A040A0A05025135380808012265657
:104080004080808080401226568040404040800220
:1040900045559060F060900255552020F820201181
:1040A0003353604080044151F011335340E04002EB
:1040B000465610102040808012365640A0A0A0A086
:1040C0004012365640C0404040E0024656609010D4
:1040D0006080F0024656F020601090600246562044
:1040E00060A0F02020024656F080E010906002466A
:1040F000566080E0909060024656F01020204040CC
:1041000002465660906090906002465660909070B3
:104110001060122555C0C000C0C011365660600046
:10412000604080123656204080804020034353F088
:1041300000F012365680402020408012365640A0B3
:1041400020400040015858304898A8A890403002BC
:104150004656609090F09090024656E090E0909025
:10416000E0024656609080809060024656E0909053
:104170009090E0024656F080E08080F0024656F0D3
:1041800080E0808080024656609080B09060024659
:10419000569090F0909090123656E040404040E0AB
:1041A00002465670202020A04002465690A0C0A093
:1041B000A0900246568080808080F002465690F0A3
:1041C000F090909002465690D0F0B0B090024656D3
:1041D000609090909060024656E09090E080800160
:1041E0004757609090D0B06010024656E09090E043
:1041F0009090024656609040209060123656E04003
:104200004040404002465690909090906002465642
:10421000909090906060024656909090F0F09002DE
:1042200046569090606090900256568888502020A4
:1042300020024656F010204080F0123656E0808072
:104240008080E0024656808040201010123656E0F2
:1042500020202020E016325240A0014151F01622C9
:10426000528040024454709090700246568080E024
:104270009090E012345460808060024656101070B6
:1042800090907002445460B0C06002465620504086
:10429000E0404001455560907010600246568080B5
:1042A000E09090901236564000C04040E0113757E1
:1042B0002000202020A040024656808090E0909070
:1042C000123656C040404040E0025454D0A8A8A83E
:1042D000024454E0909090024454609090600145F4
:1042E00055E090E0808001455570907010100244B8
:1042F00054A0D0808012345460C020C00246564082
:1043000040E040502002445490909070123454A0E9
:10431000A0A04002545488A8A85002445490606061
:10432000900145559090709060024454F02040F008
:10433000024757304020C0204030221656808080EF
:10434000808080024757C02040304020C006425243
:1043500050A0FFFFFFFFFFFFFFFFFFFFFFFFFFFF7B
:10436000FFFFFFFFFFFFFFFFFFFFFFFFFFFFFFFF5D
:10437000FFFFFF09005022165680008080808001D8
:1043800046562070A0A070200246562050E04050B3
:10439000A002555588705070880256568850F820F3
:1043A000F820221757808080008080800247577055
:1043B00080E0907010E0173151A002565670A8C8E6
:1043C000C8A87014355560A06000E003435350A0A6
:1043D00050123353E02020143151E002565670E859
:1043E000D8E8D870173151E015335340A04012354A
:1043F0005540E04000E014355540A02040E0143521
:1044000055C020C020C016225240800145559090D2
:1044100090E08002565678E8E868282824115180F8
:10442000112252408014355540C04040E0143555AB
:1044300040A04000E0034353A050A00247578080B3
:1044400080A060F0200247578080A0D0102070022A
:10445000475780408060A0F02012365640004080D0
:10446000A04002475740206090F0909002475720AC
:10447000406090F0909002475760906090F090906C
:1044800002475750A06090F090900247579000600C
:1044900090F0909002475760906090F090900246A4
:1044A0005670A0A0F0A0B001475760908080906047
:1044B000400247574020F080E080F00247572040FC
:1044C000F080E080F00247576090F080E080F002DA
:1044D00047579000F080E080F01237578040E0406E
:1044E0004040E01237572040E0404040E01237574C
:1044F00040A0E0404040E0123757A000E04040407C
:10450000E00256567048E848487002475750A0905D
:10451000D0B0909002475740206090909060024742
:104520005720406090909060024757609060909054
:10453000906002475750A06090909060024757905B
:10454000006090909060123353A040A002465670D5
:10455000B0B0D0D0E00247574020909090906002D9
:1045600047572040909090906002475760909090FD
:10457000909060024757900090909090600257573B
:104580001020885020202002465680E09090E08045
:104590000246566090A0A090A002475740200070AD
:1045A00090907002475720400070909070024757DB
:1045B0002050007090907002475750A0007090906B
:1045C000700246565000709090700247576090609D
:1045D00070909070025454F068B078113555608036
:1045E00080604002475740200060B0C060024757DB
:1045F00020400060B0C06002475760900060B0C0CB
:1046000060024656500060B0C060123757804000CC
:10461000C04040E0123757204000C04040E0123711
:104620005740A000C04040E0123656A000C04040B5
:10463000E0024757A040A01070906002475750A07A
:1046400000E09090900247574020006090906002F8
:10465000475720400060909060024757609000608C
:1046600090906002475750A00060909060024656BC
:104670009000609090601235554000E00040024488
:104680005470B0D0E00247574020009090907002E4
:1046900047572040009090907002475760900090DC
:1046A000909070024656900090909070014858206B
:1046B000400090907090600147578080E090E080CB
:1046C0008001475790009090709060000021002476
:1046D0000027002A002D00300033000101000004F3
:1046E0000107010A0100002200250028002B002EEE
:1046F000003100340002010000050108010B010037
:104700000020002300260029002C002F003200008A
:10471000010000030106010901050505050705085B
:10472000080808020202020A0A0808040404040134
:104730000101010101010103030303030303030456
:104740000707070C0C0C0C0C0C0C0C0202020206E6
:10475000060606060606060B0B0B0B0B0B0B0B01D6
:104760000210202008081020401020408002010282
:10477000010804020101020408102040808040204A
:104780001008040201800402018040201008040285
:104790000108040201010204081020408001020403
:1047A00008102040800000090A02080B0C0D0706C3
:1047B00003040100000000000000000000000000F1
:1047C00000000000000000000000000000000000E9
:1047D0000011100F000000000000000000000000A9
:1047E000000000000000000000000002494E4649A1
:1047F0004E4954594E414ECDCCCC3D0AD7233C179F
:10480000B7D13877CC2B329595E6241FB14F0A00EB
:104810000020410000C84200401C4620BCBE4CCADB
:104820001B0E5AAEC59D74004294349B56A7C6EA2F
:1048300051A711241FBECFEFD1E2DEBFCDBF00E0F4
:104840000CBF14E0A0E0B2E0E8ECFEEF01E00BBF2B
:1048500002C007900D92AE3BB107D9F71BBE15E120
:10486000AEEBB4E001C01D92AA3CB107E1F718E439
:10487000C0E3D8E404C02297FE010E940AFFC832B8
:10488000D107C9F70E94EAF90C9458FF0C94000074
:10489000A0E0B0E0EEE4F4E20C9427FFEC015B0151
:1048A0006115710519F0FB0191838083F9908F2DBB
:1048B00090E00E940EFF892BC9F7FDE2FF1621F45C
:1048C000F990EE24E39405C02BE2F21609F4F99076
:1048D000EE248E0101501040C8016CEE77E443E0F5
:1048E00050E072D2892BF9F48E010E5F1F4FC80180
:1048F0006FEE77E445E050E067D2892B19F48E0122
:10490000095F1F4FA114B10419F0F5011183008351
:10491000E0FC04C070E090E080E813C070E090E03C
:1049200080E86FEF07C1C80164EF77E443E050E02F
:104930004BD2892B69F4A114B10429F470E090E002
:1049400080EC6FE7F7C02296F501D183C083F6CFE4
:104950008824992440E050E060E070E0EF2DE053BF
:10496000EA30A0F5F2E0EF2A8E2D90E09C0128704D
:104970003070E2FE06C0232B79F50894811C911C4F
:104980002BC0232B19F0089481089108DB01CA0180
:1049900012E0880F991FAA1FBB1F1A95D1F7480F65
:1049A000591F6A1F7B1F440F551F661F771F4E0F2D
:1049B000511D611D711D483929E9520729E9620716
:1049C00029E1720748F084E0E82A06C0EE3F31F49E
:1049D000E3FC39C098E0E92AF990C0CFE53311F043
:1049E000E53189F529912D3219F4E0E1EE2A05C06F
:1049F0002B3219F081E090E003C0299182E090E031
:104A0000E22FE053EA3018F0C81BD90B1CC020E09D
:104A100030E0FCE020383F075CF4C901880F991FA3
:104A2000880F991F280F391F220F331F2E0F311D9A
:104A3000E991E053EA3068F3E4FE03C03095219534
:104A40003F4F820E931ECE2CDD24E1FE07C0A11441
:104A5000B10421F02197F501D183C083CB01BA01C4
:104A60000E9473FB7B018C01F3E0CF22DD2423E065
:104A7000C216D10421F417FB109517F910955701B0
:104A80006801C801B70120E030E040E050E00E943A
:104A9000D3FA882309F44AC097FE0DC02BE0E22E1A
:104AA00028E4F22E9094819491089394C0E2D0E08F
:104AB00000E010E012C093E2E92E98E4F92EF6CF60
:104AC000F7012591359145915491C601B5010E9498
:104AD000B3FD5B016C018C1A9D0A8C169D0684F750
:104AE000D595C7950F5F1F4F0630110529F08CEF44
:104AF0009FEFE80EF91EF1CFC501D6017C018D01B3
:104B00008C2D880F8D2D881F8F3F51F0C601B50168
:104B100020E030E040E050E00E94D3FA882331F4F6
:104B200082E290E09093C9158093C8157E2D9F2D49
:104B3000802F612F272F392F482F562FB901CA01F7
:104B4000CDB7DEB7ECE00C9443FF2F923F925F921B
:104B50006F927F928F929F92AF92BF92CF92DF928D
:104B6000EF92FF920F931F93CF93DF938C011B0162
:104B7000EA016115710519F0FB019183808320978B
:104B800049F0CE010297839728F020E030E040E022
:104B900050E0F6C0F801A1908F018A2D90E00E94AC
:104BA0000EFF892BB9F7FDE2AF1631F4F801A190A1
:104BB0008F015524539407C0FBE2AF1619F4F80196
:104BC000A1908F015524209719F0C031D105C1F46F
:104BD000F0E3AF1679F4F8018081883711F0883559
:104BE00049F4F801A1800E5F1F4FF2E05F2AC0E197
:104BF000D0E006C0209721F480E3A816E9F427C08E
:104C0000C830D10531F1C930D10524F4C230D10505
:104C100031F50CC0CA30D10589F0C031D105F9F4A5
:104C2000C12CD12CE12CB8E0FB2E28C0C12CD12CFA
:104C3000E12CA0E4FA2E22C0CAE0D0E0FCECCF2E9A
:104C4000FCECDF2EFCECEF2EFCE0FF2E17C0C8E0E2
:104C5000D0E0C12CD12CE12CE0E1FE2E0FC09E0152
:104C6000442737FD4095542F60E070E080E090E8E5
:104C70000E94CBFEC901DA016C017D0120E030E029
:104C800040E050E060E03E01882477FC8094982C5E
:104C900070EDB72EBA0CE9E0EB1570F48A2D815453
:104CA0008A3118F499ECB92E06C08A2D81568A31C2
:104CB00050F589EAB82EBA0C8B2D90E08C179D0721
:104CC00014F56F3FE1F0C216D306E406F506B0F026
:104CD000CA01B901A40193010E9485FE9B01AC01A8
:104CE0002B0D311D411D511D2130F0E03F07F0E03B
:104CF0004F07F0E85F0710F461E001C06FEFF801C3
:104D0000A1908F01C5CF2114310481F0662331F0C9
:104D100001501040F1011183008308C051FE1AC0F8
:104D200002501040F1011183008314C067FF12C0CC
:104D300050FC05C02FEF3FEF4FEF5FE704C020E0CE
:104D400030E040E050E882E290E09093C915809313
:104D5000C81516C050FE08C0509540953095219555
:104D60003F4F4F4F5F4F0CC057FF0AC082E290E0A9
:104D70009093C9158093C8152FEF3FEF4FEF5FE772
:104D8000B901CA01DF91CF911F910F91FF90EF9070
:104D9000DF90CF90BF90AF909F908F907F906F905B
:104DA0005F903F902F900895FB01DC0105900D92DC
:104DB0000020E1F70895FC0105900020E9F78095B7
:104DC00090958E0F9F1F0895FB01DC0141505040CC
:104DD00088F08D9181341CF08B350CF4805E6591E8
:104DE00061341CF06B350CF4605E861B611171F34D
:104DF000990B0895881BFCCFFB01DC01415050400A
:104E000048F005900D920020C9F701C01D92415055
:104E10005040E0F70895FB0155915523A9F0BF01DB
:104E2000DC014D9145174111E1F759F4CD01059091
:104E3000002049F04D9140154111C9F3FB0141118A
:104E4000EFCF81E090E001970895FB01DC0104C001
:104E50008D910190801921F441505040C8F7881B72
:104E6000990B0895FB01DC0102C001900D924150A5
:104E70005040D8F70895FB01DC010D900020E9F7C0
:104E8000119701900D920020E1F70895FC018191A6
:104E9000861721F08823D9F7992708953197CF01F4
:104EA0000895FB01DC0101900D920020E1F70895C7
:104EB000FB01DC014150504030F08D910190801990
:104EC00019F40020B9F7881B990B0895FB01DC0148
:104ED0004150504048F001900D920020C9F701C0A8
:104EE0001D9241505040E0F70895AEE0B0E0EBE78E
:104EF000F7E20C942FFF0E891F898EE08C831A83B2
:104F000009838FEF9FE79E838D839E01265E3F4F2F
:104F1000CE010196688D798DA9010AD02F8138853F
:104F2000020F131FF80110822E96E4E00C944BFF41
:104F3000ABE0B0E0EEE9F7E20C9421FF3C012B017D
:104F40005A01FC0117821682838181FD03C06FEF35
:104F50007FEFB9C19AE0892E1E010894211C311CF3
:104F6000F3012381F20123FD859123FF81912F011C
:104F7000882309F4A5C1853239F423FD859123FFE7
:104F800081912F01853221F490E0B301B7D1E8CFB0
:104F9000982FFF24EE249924FFE1FF15D0F09B32D7
:104FA00069F09C3228F4903259F0933291F40EC09B
:104FB0009D3249F0903369F441E024C052E0F52A73
:104FC00084E0F82A28C098E0F92A25C0E0E1FE2A0A
:104FD00022C0F7FC29C0892F80538A3070F4F6FE76
:104FE00005C0989C902C1124980E15C0E89CE02CCC
:104FF0001124E80EF0E2FF2A0EC09E3229F4F6FCDE
:105000005FC140E4F42A07C09C3619F450E8F52A41
:1050100002C0983649F4F20123FD959123FF919146
:105020002F01992309F0B8CF892F8554833018F0C8
:105030008052833038F444E050E0A40EB51E5FE3A4
:1050400059830FC0933631F0933779F0933509F0D7
:1050500052C01FC0F5018081898342E050E0A40E58
:10506000B51E610101E010E011C0F501C080D180E2
:10507000F6FC03C06FEF7FEF02C0692D70E042E0E5
:1050800050E0A40EB51EC6012ED18C015FE7F522BB
:1050900013C0F501C080D180F6FC03C06FEF7FEF35
:1050A00002C0692D70E042E050E0A40EB51EC601BA
:1050B0000FD18C0150E8F52AF3FE06C018C080E23B
:1050C00090E0B3011BD1EA948E2D90E008171907E8
:1050D000B0F30DC0F601F7FC8591F7FE81916F01E9
:1050E00090E0B3010BD1E110EA940150104001159A
:1050F000110581F7E2C0943611F0993661F5F7FE9B
:1051000008C0F501208131814281538184E090E023
:105110000AC0F501808191819C01442737FD4095AB
:10512000542F82E090E0A80EB91E9FE6F92257FFA7
:1051300009C050954095309521953F4F4F4F5F4F97
:10514000E0E8FE2ACA01B901A1012AE030E002D15B
:10515000D82ED2183FC0953729F41F2D1F7E2AE084
:1051600030E01DC01F2D197F9F3661F0903720F46D
:10517000983509F0A5C00FC0903739F0983709F07D
:105180009FC004C028E030E00AC0106114FD146024
:1051900020E130E004C014FD166020E132E017FF8A
:1051A00008C0F501608171818281938144E050E003
:1051B00008C0F50180819181BC0180E090E042E06F
:1051C00050E0A40EB51EA101C5D0D82ED2188FE78D
:1051D000F82EF122F6FE0BC05EEFF522D91438F45A
:1051E000F4FE07C0F2FC05C08FEEF82202C01D2DB0
:1051F00001C0192DF4FE0DC0FE01ED0DF11D8081E1
:10520000803319F499EEF92208C01F5FF2FE05C041
:1052100003C08F2D867809F01F5F0F2DF3FC13C09C
:10522000F0FE0EC01E1510F09D2C0AC09D2C9E0C89
:10523000911A1E2D05C080E290E0B3015FD01F5F80
:105240001E15C8F304C01E1510F4E11A01C0EE24A7
:1052500004FF0EC080E390E0B30150D002FF1BC0FA
:1052600001FD03C088E790E00EC088E590E00BC028
:10527000802F867881F001FF02C08BE201C080E2BE
:10528000F7FC8DE290E0B30139D005C080E390E0F7
:10529000B30134D09A94D914C8F3DA94F101ED0D26
:1052A000F11D808190E0B30129D0DD20B1F705C068
:1052B00080E290E0B30122D0EA94EE20C9F750CE0C
:1052C000F30166817781CB012B96E2E10C943DFFDF
:1052D000FC010590615070400110D8F780959095C1
:1052E0008E0F9F1F0895FC016150704001900110C6
:1052F000D8F7809590958E0F9F1F08950F931F9359
:10530000CF93DF938C01EB018B8181FF1BC082FF68
:105310000DC02E813F818C819D812817390764F44F
:10532000E881F9810193F983E88306C0E885F9856E
:10533000802F1995892B31F48E819F8101969F834F
:105340008E8302C00FEF1FEFC801DF91CF911F9135
:105350000F910895FA01AA27283051F1203181F1E7
:10536000E8946F936E7F6E5F7F4F8F4F9F4FAF4F6D
:10537000B1E03ED0B4E03CD0670F781F891F9A1F80
:10538000A11D680F791F8A1F911DA11D6A0F711D34
:10539000811D911DA11D20D009F468943F912AE040
:1053A000269F11243019305D3193DEF6CF01089528
:1053B000462F4770405D4193B3E00FD0C9F7F6CF59
:1053C000462F4F70405D4A3318F0495D31FD405221
:1053D000419302D0A9F7EACFB4E0A69597958795B7
:1053E00077956795BA95C9F7009761057105089596
:1053F0009B01AC010A2E0694579547953795279542
:10540000BA95C9F7620F731F841F951FA01D0895D9
:105410001092F2041092F4041092F604089580930E
:105420008F030895EFE6F0E0808182608083089525
:105430001F93FC011FB7F89480819181A281B381F1
:105440008093CC049093CD04A093CE04B093CF046A
:10545000FB0180819181A281B3818093D0049093DC
:10546000D104A093D204B093D304FA018081918136
:10547000A281B3818093D4049093D504A093D604E1
:10548000B093D704F90180819181A281B381809387
:10549000D8049093D904A093DA04B093DB041FBF1F
:1054A0001F910895FC012FB7F89480819181A2810A
:1054B000B3818093D8049093D904A093DA04B09375
:1054C000DB042FBF0895E82F8FB7F894F0E0EE0FBC
:1054D000FF1FEE0FFF1FE453FB4F208131814281FC
:1054E00053818FBFB901CA01089580916F008D7FEC
:1054F00080936F0006C08091970C8F5F8F708093B0
:10550000970C9091960C8091970C981751F41092EB
:10551000BF041092BE0480916F00826080936F0080
:1055200008959091960C8091970C981751F3E3CFC2
:10553000E5E4F1E0949108C08091C00085FFFCCFC4
:105540009093C600319694919923B1F7E1E4F1E08C
:10555000949108C08091C00085FFFCCF9093C60055
:10556000319694919923B1F788E20E94E6F3BC0149
:105570008EEB9FE04AE050E00E941C9C89E20E9472
:10558000E6F3BC018EEB9FE04AE050E00E941C9CD9
:105590008091C00085FFFCCF8AE08093C600EDE3D8
:1055A000F1E0949108C08091C00085FFFCCF9093FA
:1055B000C600319694919923B1F785E40E94E6F3F1
:1055C000BC018EEB9FE04AE050E00E941C9C87E209
:1055D0000E94E6F3BC018EEB9FE04AE050E00E949F
:1055E0001C9C8091C00085FFFCCF8AE08093C600A0
:1055F000E9E3F1E0949108C08091C00085FFFCCF01
:105600009093C600319694919923B1F784E40E9457
:10561000E6F3BC018EEB9FE04AE050E00E941C9C48
:1056200083E40E94E6F3BC018EEB9FE04AE050E089
:105630000E941C9C8091C00085FFFCCF8AE0809373
:10564000C600E4E3F1E0949108C08091C00085FFBA
:10565000FCCF9093C600319694919923B1F781E4E1
:105660000E94E6F3BC018EEB9FE04AE050E00E940E
:105670001C9C82E40E94E6F3BC018EEB9FE04AE0B2
:1056800050E00E941C9C8091C00085FFFCCF8AE006
:105690008093C600EFE2F1E0949108C08091C000D1
:1056A00085FFFCCF9093C600319694919923B1F772
:1056B0008FE30E94E6F3BC018EEB9FE04AE050E0EE
:1056C0000E941C9C80E40E94E6F3BC018EEB9FE0EC
:1056D0004AE050E00E941C9C8091C00085FFFCCFF6
:1056E0008AE08093C60008950F931F93182F042F0C
:1056F00067FD19C0823081F0833028F4882341F09F
:10570000813089F407C0833049F0843061F408C0E7
:1057100088E207C085E405C084E403C081E401C0D9
:105720008FE30E94B4F307FD1AC0123081F01330EA
:1057300028F4112341F0113091F407C0133049F0DF
:10574000143069F408C089E207C087E205C083E429
:1057500003C082E401C080E4602F0E94B4F31F9173
:105760000F910895643089F0653028F4613041F07C
:10577000623099F407C0683051F0603171F40AC0AA
:1057800060E001C061E040E004C060E001C061E0B1
:1057900041E0AACF61E041E0A7CF08950F931F93A6
:1057A000182F062F86E260E00E94B4F31EBD0DB4F0
:1057B00007FEFDCF8EB50EBD0DB407FEFDCF8EB535
:1057C00086E261E00E94B4F31F910F910895EDE12C
:1057D000F4E0E80FF11D808190E0E0CFCF93DF93FC
:1057E00089E261E00E9401F387E261E00E9401F337
:1057F00083E461E00E9401F382E461E00E9401F32E
:1058000080E461E00E9401F3C0E0D0E0FE01E85EC8
:10581000FB4F8C2F6081A6DF2196C530D105B1F7F3
:10582000DF91CF910895CF93DF930E94EFF286E24C
:1058300061E00E9401F3C0E0D0E0FE01E35EFB4FB7
:10584000DE01AE5DBB4F6C91808190E070E0A6DF21
:105850002196C530D10589F7DF91CF910895E3DF17
:10586000BDDFEAE0F1E08081826080838081816039
:105870008083808184608083808180648083808154
:10588000806880830F9A179A0E9A169A0D9A159A25
:105890000C9A149A0B9A139A26982E9A25982D9A58
:1058A00024982C9A389A4098179A10927B12399A19
:1058B0004198169A10927C123A9A4298159A109230
:1058C0007D123B9A4398149A3C9A4498A1E8B0E020
:1058D0008C918F7E8C938C9188608C93E0E8F0E0C3
:1058E00080818D7F808380818E7F808380818F7394
:1058F000808380818F7C80838C91887F82608C9371
:1059000080E090E490938900809388001092850055
:1059100010928400EFE6F0E080818260808381E075
:1059200080938F03789408959091960C8091970CB2
:10593000981739F00E94D1E00E9460A80E948A95D1
:10594000F3CF0895F1DF179A10927B12169A1092F6
:105950007C12159A10927D12149A08951F920F923C
:105960000FB60F920BB60F921124AF92BF92CF9247
:10597000DF92EF92FF920F931F932F933F934F93DA
:105980005F936F937F938F939F93AF93BF93CF93C7
:10599000DF93EF93FF938091BE049091BF04892B16
:1059A00009F097C19091960C8091970C981719F473
:1059B000E0E0F0E014C08091970C90E021E530E049
:1059C000829FF001839FF00D929FF00D1124EA5702
:1059D000F84FE05BFF4F81E08083E055F040F093AB
:1059E000BF04E093BE04309709F46DC1E05BFF4F44
:1059F00081E08083E055F0401092FE041092FF0495
:105A0000109200051092010560AD71AD2CE9613472
:105A1000720718F060E47CE904C03EE46132730769
:105A200030F0769567957695679584E007C047E2F4
:105A30006131740730F07695679582E08093F704C2
:105A400007C08093F7046032710510F460E270E0E3
:105A50006052704058E060307507E8F0472F50E022
:105A6000440F551F440F551F4D5A5E4F9A012E5F2C
:105A70003F4FF901859194919C01AA27639FC00132
:105A8000629F810D9A1F06948A1F9A1F1124FA01A2
:105A9000459154911EC0CB01969587958C7F8D5A68
:105AA0009A4FFC0145915491FC0132962591349115
:105AB000862F90E087709070FC012E9FC0012F9F71
:105AC000900D3E9F900D1124B3E096958795BA9561
:105AD000E1F7481B590B44365105A8F4E0E0F2E029
:105AE00007C08091C00085FFFCCF31969093C6001F
:105AF00090819923B1F78EEB9FE04AE050E00E943D
:105B0000439C44E650E05093030540930205809186
:105B1000F704992787FD90959093050580930405D8
:105B2000E091BE04F091BF0464AD75AD7093FD04C7
:105B30006093FC04FCE961347F0718F060E47CE9C1
:105B400004C02EE46132720730F076956795769541
:105B5000679584E007C037E26131730730F07695CE
:105B6000679582E08093F70408C081E08093F70492
:105B70006032710510F460E270E06052704048E0FD
:105B800060307407E8F0472F50E0440F551F440F72
:105B9000551F4D5A5E4F9A012E5F3F4FF901859177
:105BA00094919C01AA27639FC001629F810D9A1F57
:105BB00006948A1F9A1F1124FA01459154911EC020
:105BC000CB01969587958C7F8D5A9A4FFC01459114
:105BD0005491FC01329625913491862F90E0877084
:105BE0009070FC012E9FC0012F9F900D3E9F900D45
:105BF000112433E0969587953A95E1F7481B590BA8
:105C000044365105A8F4E0E0F2E007C08091C000FE
:105C100085FFFCCF31969093C60090819923B1F710
:105C20008EEB9FE04AE050E00E94439C44E650E047
:105C3000CA01A0E0B0E08093F8049093F904A09327
:105C4000FA04B093FB045093890040938800E091DC
:105C5000BE04F091BF0480899189A289B389B69569
:105C6000A79597958795B095A095909581959F4F0D
:105C7000AF4FBF4F8093DC049093DD04A093DE040C
:105C8000B093DF048093E0049093E104A093E204D6
:105C9000B093E3048093E4049093E504A093E604B6
:105CA000B093E7048093E8049093E904A093EA0496
:105CB000B093EB041092EC041092ED041092EE04F9
:105CC0001092EF0406C080ED97E0909389008093D6
:105CD0008800C091BE04D091BF04209709F4AEC4DF
:105CE00088A18093F00480FF0AC08FB7F894909148
:105CF0000B019D7F90930B018FBF8FEF09C08FB772
:105D0000F89490910B01926090930B018FBF81E00A
:105D100080938B038091F00481FF0AC08FB7F894C1
:105D200090910B01916090930B018FBF8FEF09C091
:105D30008FB7F89490910B019E7F90930B018FBFCA
:105D400081E080938C038091F00480FF3CC08091BF
:105D50008F038823C1F183B18295869586958370E0
:105D60008095282F217080FF2CC08091F10488231A
:105D700041F188819981AA81BB81181619061A06FA
:105D80001B06FCF48091CC049091CD04A091CE042C
:105D9000B091CF048093C0049093C104A093C20437
:105DA000B093C30481E08093F20488899989AA8919
:105DB000BB898093EC049093ED04A093EE04B09320
:105DC000EF042093F1048091F00481FF3BC08091A7
:105DD0008F038823B9F183B182958695877080956A
:105DE000282F217080FF2CC08091F304882341F17B
:105DF0008C819D81AE81BF81181619061A061B067B
:105E0000FCF48091D0049091D104A091D204B0917F
:105E1000D3048093C4049093C504A093C604B093A4
:105E2000C70481E08093F40488899989AA89BB8991
:105E30008093EC049093ED04A093EE04B093EF04F0
:105E40002093F3048091F00482FF47C09FB7F89439
:105E500080910B018B7F80930B019FBF8FEF80930D
:105E60008D0380918F03882309F442C083B182950A
:105E70008F708095282F217080FF2CC08091F504B1
:105E8000882341F188859985AA85BB85181619064E
:105E90001A061B06FCF48091D4049091D504A091BD
:105EA000D604B091D7048093C8049093C904A093FA
:105EB000CA04B093CB0481E08093F6048889998961
:105EC000AA89BB898093EC049093ED04A093EE041F
:105ED000B093EF042093F5040BC08FB7F894909122
:105EE0000B01946090930B018FBF81E080938D0331
:105EF0008091F00483FF0AC08FB7F89490910B0152
:105F0000906490930B018FBF8FEF09C08FB7F89407
:105F100090910B019F7B90930B018FBF81E0809349
:105F20008E0360E06AC18091C00087FF19C0409174
:105F3000C600E091BA0FF091BB0F31969F012F7709
:105F4000307031978091BC0F9091BD0F28173907A1
:105F500039F0E65CF04F40833093BB0F2093BA0FCB
:105F6000288139814A815B818091DC049091DD0434
:105F7000A091DE04B091DF04280F391F4A1F5B1F78
:105F80002093DC043093DD044093DE045093DF045F
:105F900012161306140615066CF5409A888999891D
:105FA000AA89BB89281B390B4A0B5B0B2093DC04A5
:105FB0003093DD044093DE045093DF042091CC0441
:105FC0003091CD044091CE045091CF0480918B0349
:105FD000992787FD9095A92FB92F820F931FA41F92
:105FE000B51F8093CC049093CD04A093CE04B093BE
:105FF000CF0440982C813D814E815F818091E004E7
:106000009091E104A091E204B091E304280F391FBC
:106010004A1F5B1F2093E0043093E1044093E204A5
:106020005093E30412161306140615066CF5419AF4
:1060300088899989AA89BB89281B390B4A0B5B0B74
:106040002093E0043093E1044093E2045093E3048E
:106050002091D0043091D1044091D2045091D304C6
:1060600080918C03992787FD9095A92FB92F820FD6
:10607000931FA41FB51F8093D0049093D104A093C5
:10608000D204B093D3044198288539854A855B852D
:106090008091E4049091E504A091E604B091E704B6
:1060A000280F391F4A1F5B1F2093E4043093E50437
:1060B0004093E6045093E7041216130614061506DF
:1060C0006CF5429A88899989AA89BB89281B390B62
:1060D0004A0B5B0B2093E4043093E5044093E60401
:1060E0005093E7042091D4043091D5044091D60414
:1060F0005091D70480918D03992787FD9095A92F02
:10610000B92F820F931FA41FB51F8093D4049093BF
:10611000D504A093D604B093D70442982C853D852E
:106120004E855F858091E8049091E904A091EA048E
:10613000B091EB04280F391F4A1F5B1F2093E8041E
:106140003093E9044093EA045093EB0412161306CB
:10615000140615066CF5439A88899989AA89BB8922
:10616000281B390B4A0B5B0B2093E8043093E9049E
:106170004093EA045093EB042091D8043091D90461
:106180004091DA045091DB0480918E03992787FDBA
:106190009095A92FB92F820F931FA41FB51F80932D
:1061A000D8049093D904A093DA04B093DB04439805
:1061B0008091EC049091ED04A091EE04B091EF0475
:1061C0000196A11DB11D8093EC049093ED04A09362
:1061D000EE04B093EF042091EC043091ED04409173
:1061E000EE045091EF0488899989AA89BB89281700
:1061F00039074A075B0730F46F5F8091F70468172F
:106200000CF491CE2091EC043091ED044091EE0419
:106210005091EF048C899D89AE89BF8982179307BD
:10622000A407B50708F4E3C0E090F804F090F9047F
:106230000091FA041091FB04AC8CBD8CCE8CDF8CE9
:10624000A8019701C601B501AA27279FB12D389F44
:10625000F001489FF00D479FE00DF11D289FB00D04
:10626000E11DFA1F379FB00DE11DFA1F469FB00DCB
:10627000E11DFA1F369FB10DEA1FFA1FB695EA1FFE
:10628000FA1F11248CAD9DAD8E0F9F1F9093FD04BE
:106290008093FC0428AD39AD4AAD5BADA0E0B0E021
:1062A000281739074A075B0720F43093FD04209331
:1062B000FC046091FC047091FD048CE96134780762
:1062C00018F060E47CE904C09EE46132790730F0A4
:1062D000769567957695679584E007C0E7E261312A
:1062E0007E0730F07695679582E08093F70408C0CA
:1062F00081E08093F7046032710510F460E270E091
:1063000060527040F8E060307F07E8F0472F50E0BF
:10631000440F551F440F551F4D5A5E4F9A012E5F73
:106320003F4FF901859194919C01AA27639FC00179
:10633000629F810D9A1F06948A1F9A1F1124FA01E9
:10634000459154911EC0CB01969587958C7F8D5AAF
:106350009A4FFC0145915491FC013296259134915C
:10636000862F90E087709070FC012E9FC0012F9FB8
:10637000900D3E9F900D1124B3E096958795BA95A8
:10638000E1F7481B590B44365105A8F4E0E0F2E070
:1063900007C08091C00085FFFCCF31969093C60066
:1063A00090819923B1F78EEB9FE04AE050E00E9484
:1063B000439C44E650E050938900409388009A0142
:1063C00040E050E08091F8049091F904A091FA0423
:1063D000B091FB04820F931FA41FB51F8093F80494
:1063E0009093F904A093FA04B093FB0402C12091A6
:1063F000EC043091ED044091EE045091EF04888D4F
:10640000998DAA8DBB8D82179307A407B50708F055
:10641000E4C06091FE047091FF04809100059091AA
:1064200001052C8D3D8D4E8D5F8DAA27639FB12D6B
:10643000749FF001849FF00D839FE00DF11D649F18
:10644000B00DE11DFA1F739FB00DE11DFA1F829F71
:10645000B00DE11DFA1F729FB10DEA1FFA1FB6952C
:10646000EA1FFA1F11248091FC049091FD048E17FD
:106470009F0738F4C05CDF4F68817981C054D040F9
:1064800003C0BC016E1B7F0BC05CDF4F28813981CC
:106490004A815B81CB01A0E0B0E082179307A4079B
:1064A000B50708F4B901FCE961347F0718F060E42E
:1064B0007CE904C02EE46132720730F0769567956E
:1064C0007695679584E007C037E26131730730F055
:1064D0007695679582E08093F70408C081E0809309
:1064E000F7046032710510F460E270E060527040B1
:1064F00048E060307407E8F0472F50E0440F551F24
:10650000440F551F4D5A5E4F9A012E5F3F4FF901C0
:10651000859194919C01AA27639FC001629F810D80
:106520009A1F06948A1F9A1F1124FA0145915491CB
:106530001EC0CB01969587958C7F8D5A9A4FFC0192
:1065400045915491FC01329625913491862F90E02B
:1065500087709070FC012E9FC0012F9F900D3E9F71
:10656000900D112423E0969587952A95E1F7481B15
:10657000590B44365105A8F4E0E0F2E007C08091E1
:10658000C00085FFFCCF31969093C600908199237F
:10659000B1F78EEB9FE04AE050E00E94439C44E656
:1065A00050E050938900409388009A0140E050E009
:1065B0008091FE049091FF04A0910005B091010527
:1065C000820F931FA41FB51F8093FE049093FF04B6
:1065D000A0930005B09301050CC080910205909135
:1065E000030590938900809388008091040580932F
:1065F000F7042091EC043091ED044091EE045091A9
:10660000EF04E091BE04F091BF0480899189A289D2
:10661000B389281739074A075B0780F01092BF0437
:106620001092BE049091960C8091970C981731F0BF
:106630008091970C8F5F8F708093970CFF91EF91F3
:10664000DF91CF91BF91AF919F918F917F916F918A
:106650005F914F913F912F911F910F91FF90EF907C
:10666000DF90CF90BF90AF900F900BBE0F900FBEFA
:106670000F901F9018958091F204882349F480911F
:10668000F404882329F48091F604882309F49CC03B
:10669000E3E5F9E0949108C08091C00085FFFCCF4C
:1066A0009093C600319694919923B1F7E5E9F9E00A
:1066B000949108C08091C00085FFFCCF9093C600E4
:1066C000319694919923B1F78091F2048823F1F0E7
:1066D0006091C0047091C1048091C2049091C30480
:1066E0000E9475FB209125073091260740912707CE
:1066F000509128070E94DAFAAB01BC0181E999E0C8
:106700000E9421AC81E899E00E94AD948091F4044C
:106710008823F1F06091C4047091C5048091C6048F
:106720009091C7040E9475FB2091290730912A0798
:1067300040912B0750912C070E94DAFAAB01BC0163
:106740008DE799E00E9421AC8DE699E00E94AD941E
:106750008091F6048823F1F06091C8047091C90417
:106760008091CA049091CB040E9475FB20912D0763
:1067700030912E0740912F07509130070E94DAFA8E
:10678000AB01BC0189E699E00E9421AC89E599E062
:106790000E94AD94E4E1F2E007C08091C00085FF63
:1067A000FCCF31969093C60090819923B1F78091E8
:1067B000C00085FFFCCF8AE08093C6001092F204EF
:1067C0001092F4041092F604089580910C07882327
:1067D00099F1409106055091070560910805709167
:1067E000090580910A0790910B072AE035E00E9485
:1067F000E7E8882319F140910D0750910E07609149
:106800000F0770911007411551056105710591F051
:1068100080910A0790910B072AE035E00E94E7E893
:10682000882361F010920D0710920E0710920F0747
:106830001092100710920C0781E0089580E00895EF
:10684000DF92EF92FF920F931F937B018C01D42E66
:106850008091060590910705A0910805B091090562
:106860008E159F05A007B107B9F0AFDF8823E1F0CF
:1068700080910A0790910B07B801A7012AE035E043
:106880000E949AE9882381F0E0920605F0920705BC
:106890000093080510930905DD2011F481E005C07F
:1068A00081E080930C0701C080E01F910F91FF9061
:1068B000EF90DF9008958F929F92AF92BF92CF9208
:1068C000DF92EF92FF920F931F93CF93DF936C01B0
:1068D000142F70930B0760930A07FC01178A82E05C
:1068E00090E0A0E0B0E080839183A283B383109214
:1068F0000C0710920D0710920E0710920F071092BE
:1069000010078FEF9FEFAFEFBFEF809306059093D7
:106910000705A0930805B0930905442321F48824B2
:10692000992454013FC0453008F01CC160E070E07C
:1069300080E090E040E084DF882309F413C1C12F98
:10694000D0E02197FE0174E0EE0FFF1F7A95E1F78A
:10695000E65FFA4FE254FE4F8081EE5BF14090E03B
:106960008F779070892B09F0FDC0E653FE4F808130
:106970009181A281B38184369105A105B10508F406
:10698000F1C064E0CC0FDD1F6A95E1F7C053D94F29
:1069900088809980AA80BB8081149104A104B104ED
:1069A00009F4E0C0C501B40140E04ADF882309F4DE
:1069B000D9C080911505909116058050924009F03C
:1069C000D1C020911A05222309F4CCC0809118056A
:1069D00090911905892B09F4C5C08091170588236A
:1069E00009F4C0C0F601228B8091170584831586B7
:1069F00061E070E007C04F5FF601458741504830C5
:106A000008F0B0C0F6014585848190E09B01042E1A
:106A100002C0220F331F0A94E2F78217930759F737
:106A200020912005309121052115310519F040E014
:106A300050E008C020912E0530912F05409130057F
:106A400050913105F6012583368347835087E090C6
:106A50001805F090190500E010E0E80CF91C0A1D7B
:106A60001B1DE38AF48A058B168B80911B05909180
:106A70001C05918F808F60911A0570E080E090E096
:106A80000E9485FE6E0D7F1D801F911FF601628F93
:106A9000738F848F958F20911B0530911C0555E0D5
:106AA000220F331F5A95E1F721503E4F232F3327F2
:106AB000269540E050E0260F371F481F591F2687B4
:106AC0003787408B518B80911D0590911E05009753
:106AD00019F0A0E0B0E008C080912A0590912B0544
:106AE000A0912C05B0912D0585017401E21AF30ADD
:106AF000040B150BA8019701280F391F4A1F5B1FB4
:106B0000F601058404C056954795379527950A9454
:106B1000D2F72187328743875487253FFFE03F071D
:106B2000F0E04F07F0E05F0720F48CE0F601878B80
:106B300019C0255F3F4F4040504018F480E1F601F6
:106B40000EC08091360590913705A0913805B0911F
:106B50003905F601828F938FA48FB58F80E2878BE2
:106B600081E001C080E0DF91CF911F910F91FF90F4
:106B7000EF90DF90CF90BF90AF909F908F9008954F
:106B80006F927F928F929F92AF92BF92CF92DF923D
:106B9000EF92FF920F931F93CF93DF93EC015A0173
:106BA0006B0138014901423051056105710508F456
:106BB0005DC089859A85AB85BC850196A11DB11DF7
:106BC00084179507A607B70708F450C08F8980314E
:106BD00029F4E52EF62E072F11270CC0803209F07C
:106BE00045C07A018B0187E016950795F794E794E5
:106BF0008A95D1F78B899C89AD89BE89E80EF91EEB
:106C00000A1F1B1FC801B70141E01ADE882371F17A
:106C10008F89803149F4F501F070EE0FFF1FE65FB8
:106C2000FA4F718260820DC0F501EF77F070EE0FC0
:106C3000FF1FEE0FFF1FE65FFA4F608271828282B4
:106C400093828A89823080F08D819E81AF81B88560
:106C5000E80EF91E0A1F1B1FE0920D07F0920E07A7
:106C600000930F071093100781E001C080E0DF91CF
:106C7000CF911F910F91FF90EF90DF90CF90BF9039
:106C8000AF909F908F907F906F900895CF92DF92FA
:106C9000EF92FF920F931F93CF93DF93EC017A0152
:106CA0008B01690189859A85AB85BC850196A11DFB
:106CB000B11D84179507A607B70708F452C08F893E
:106CC000803129F45527412F302F2F2D0CC08032D1
:106CD00009F047C09A01AB0167E056954795379593
:106CE00027956A95D1F78B899C89AD89BE89280F34
:106CF000391F4A1F5B1F8091060590910705A091DF
:106D00000805B0910905281739074A075B0731F0D4
:106D1000CA01B90140E094DD882319F18F898031DF
:106D200059F4F701F070EE0FFF1FE65FFA4F808114
:106D30009181A0E0B0E00EC0F701EF77F070EE0FA8
:106D4000FF1FEE0FFF1FE65FFA4F80819181A28146
:106D5000B381BF70F60180839183A283B38381E006
:106D600001C080E0DF91CF911F910F91FF90EF90D4
:106D7000DF90CF900895AF92BF92CF92DF92EF92C3
:106D8000FF920F931F93DF93CF9300D00F92CDB755
:106D9000DEB76C017A018B0182E090E0A0E0B0E008
:106DA000F60180839183A283B3835E010894A11CC2
:106DB000B11CC601B801A701950168DF882339F12C
:106DC000C601B801A70100E010E020E030E0D8DE05
:106DD0008823E9F0E980FA800B811C81F60187891C
:106DE000803151F4F8EFEF16FFEFFF06F0E00F07E8
:106DF000F0E01F07F0F209C088EFE8168FEFF80601
:106E00008FEF08078FE01807A0F281E001C080E053
:106E10000F900F900F900F90CF91DF911F910F91D6
:106E2000FF90EF90DF90CF90BF90AF9008954F927A
:106E30005F926F927F928F929F92AF92BF92CF920A
:106E4000DF92EF92FF920F931F93DF93CF9300D0C7
:106E50000F92CDB7DEB76C0149835A836B837C8375
:106E60003901EE24FF2487012E010894411C511C96
:106E7000812CE2E09E2EA12CB12C49815A816B819C
:106E80007C81C601920102DF882339F1D501C4015A
:106E9000F601058404C0880F991FAA1FBB1F0A941E
:106EA000D2F7E80EF91E0A1F1B1F29813A814B8178
:106EB0005C818789803131F4285F3F4F40405040EA
:106EC000E0F205C0285F3F4F4F4F5F40B0F2F30143
:106ED000E082F1820283138381E00F900F900F9084
:106EE0000F90CF91DF911F910F91FF90EF90DF9066
:106EF000CF90BF90AF909F908F907F906F905F905A
:106F00004F9008952F923F924F925F926F927F928F
:106F10008F929F92AF92BF92CF92DF92EF92FF92A9
:106F20000F931F93DF93CF93CDB7DEB72F970FB695
:106F3000F894DEBF0FBECDBF1C014A875B876C870C
:106F40007D873F872E87DC0119968D919D910D904D
:106F5000BC91A02D0196A11DB11D8E839F83A88792
:106F6000B987F90100811181228133810115110551
:106F70002105310549F0480159010894811C911CF3
:106F8000A11CB11C1D8210C0D1018D909D90AD90AF
:106F9000BC901D828A859B85AC85BD850197A10526
:106FA000B10511F491E09D837501640144245524D9
:106FB00032018E010F5F1F4FF10181859285A385FC
:106FC000B485481659066A067B0608F08CC08E8187
:106FD0009F81A885B9858C159D05AE05BF0550F428
:106FE000A2E08A2E912CA12CB12CF2E0CF2ED12C34
:106FF000E12CF12CC101B701A601980147DE8823DD
:1070000009F471C089819A81AB81BC81A701960185
:107010002F5F3F4F4F4F5F4F0097A105B10519F00C
:1070200049015A010DC0281939094A095B098A85A5
:107030009B85AC85BD85281739074A075B0759F042
:107040000894411C511C611C711C0894C11CD11C6A
:10705000E11CF11CB1CFC101A601B7010FEF1FEF79
:107060002FEF3FE08DDD882391F43DC026013701ED
:1070700008944108510861087108C101B301A201D7
:10708000970186017DDD882371F1730162018C1403
:107090009D04AE04BF0450F3AE85BF854D915D9154
:1070A0006D917C91411551056105710531F0C1016A
:1070B0009501840165DD8823B1F0EE85FF8580822E
:1070C0009182A282B382FD81FF2359F00894811C32
:1070D000911CA11CB11CD1018D929D92AD92BC92CC
:1070E000139781E001C080E02F960FB6F894DEBFC1
:1070F0000FBECDBFCF91DF911F910F91FF90EF9009
:10710000DF90CF90BF90AF909F908F907F906F90C7
:107110005F904F903F902F9008953F924F925F92D3
:107120006F927F928F929F92AF92BF92CF92DF9297
:10713000EF92FF920F931F93CF93DF938091850778
:10714000882309F4F6C08090940390909503A09052
:107150009603B09097036091651470916614882728
:1071600077FD8095982F0E9475FB20E030E040E08D
:1071700050E40E94FAF9A50194010E94D3FA87FD18
:10718000D8C03090970C0F2EF0E04F2EF0E05F2E1D
:10719000F0E06F2EF0E07F2EF02DC1E5D0E058C07A
:1071A000232D30E02C9FF0012D9FF00D3C9FF00D22
:1071B0001124EA57F84F80819181A281B381009711
:1071C000A105B10581F484819581A681B7810097DD
:1071D000A105B10541F480859185A285B38500970D
:1071E000A105B10591F12C9F60012D9FD00C3C9F12
:1071F000D00C112486E897E0C80ED91EF6016485EC
:107200007585868597850E9475FB7B018C01F6014B
:1072100060897189828993890E9473FB9B01AC010B
:10722000C801B7010E94DAFAF60122A133A144A1F4
:1072300055A10E94B3FD7B018C01A30192010E9424
:10724000E1FC181614F4270138013394FFE03F22C3
:107250008091960C381609F0A3CFC301B20120919A
:1072600098033091990340919A0350919B030E9497
:10727000B3FD9B01AC01C501B4010E94FAF97B0189
:107280008C01A50194010E94D3FA87FD02C0470139
:1072900058011091900300919103F0909203E090B7
:1072A0009303C501B401212F302F4F2D5E2D0E9475
:1072B000E1FC181634F4812F902FAF2DBE2D4C0118
:1072C0005D014090AC0C5090AD0C6090AE0C709095
:1072D000AF0CC301B201A50194010E94E1FC181694
:1072E000C4F4C501B40120E037ED43EA5CE30E9439
:1072F000B3FD7B018C01C301B20128E431EE4AE702
:107300005FE30E94B3FDA80197010E94FAF94B01C7
:107310005C018092AC0C9092AD0CA092AE0CB0923D
:10732000AF0CC501B4010E9442FB709366146093D8
:107330006514DF91CF911F910F91FF90EF90DF9037
:10734000CF90BF90AF909F908F907F906F905F9005
:107350004F903F9008958091960C9091970C891BC7
:107360008F70089560939C0370939D0380939E0398
:1073700090939F0308950F931F93CF93DF93C0E0E3
:10738000D0E08E010B59184FFE01E75CF84F608189
:107390007181828193810E9473FBFE01EB5DF84F46
:1073A00020813181428153810E94B3FD0E9447FBBD
:1073B000F80160837183828393832496C031D10561
:1073C00001F7DF91CF911F910F910895FC018091FA
:1073D0008212882369F46081718182819381209176
:1073E00031073091320740913307509134070EC076
:1073F0008130C1F460817181828193812091350750
:107400003091360740913707509138070E94B3FDFD
:107410000E9483FD609381077093820780938307A6
:107420009093840781E897E00C94522ACF92DF92E0
:10743000EF92FF920F931F93CF93DF93FC018B0189
:107440007A01690160817181828193812091250790
:107450003091260740912707509128070E94B3FDDD
:107460000E9483FDC5E7D7E06093750770937607A8
:107470008093770790937807F8016081718182810A
:1074800093812091290730912A0740912B07509131
:107490002C070E94B3FD0E9483FDFE013496609389
:1074A0007907718382839383F7016081718182817F
:1074B000938120912D0730912E0740912F075091F5
:1074C00030070E94B3FD0E9483FDFE013896609351
:1074D0007D0771838283938380918212882371F464
:1074E000F601608171818281938120913107309111
:1074F000320740913307509134070FC08130C1F4F7
:10750000F6016081718182819381209135073091EC
:10751000360740913707509138070E94B3FD0E940B
:1075200083FDFE013C966093810771838283938380
:1075300085E797E069E777E04DE757E021E837E036
:107540000E94182A80E090E0A0E0B0E08093980CC0
:107550009093990CA0939A0CB0939B0C80939C0CE5
:1075600090939D0CA0939E0CB0939F0C8093A00CC5
:107570009093A10CA093A20CB093A30C8093A40CA5
:107580009093A50CA093A60CB093A70C8093A80C85
:107590009093A90CA093AA0CB093AB0CDF91CF9160
:1075A0001F910F91FF90EF90DF90CF9008958F92F1
:1075B0009F92AF92BF92CF92DF92EF92FF920F9382
:1075C0001F93CF93DF93EC016B01009709F45CC02C
:1075D0008FA9882309F058C0EEA0FFA008A519A51F
:1075E000FB01B6A0A7A090A481A4C801B7012B2DD0
:1075F0003A2D492D582D0E94D3FA88230CF044C00F
:10760000C801B701A80197010E94B3FD7B018C015D
:107610006AA97BA98CA99DA9905820E030E040E0A0
:1076200050EC0E94B3FD2EA53FA548A959A90E9480
:10763000B3FD9B01AC01C801B7010E94FAF90E9499
:1076400020FE7B018C016B2D7A2D892D982D9701C1
:10765000A8010E94D3FA882324F4EB2CFA2C092DDC
:10766000182D6B2D7A2D892D982D9701A8010E9438
:10767000D3FA882349F0C701D801F60186A397A35E
:10768000A0A7B1A781E086ABDF91CF911F910F91A9
:10769000FF90EF90DF90CF90BF90AF909F908F9032
:1076A0000895EF92FF920F931F93CF93DF93F09083
:1076B000970C00E010E020E030E081E5E82E11C0FA
:1076C000FE9CE0011124CA57D84FC901B801AE0190
:1076D0006EDF8F2D8F5F803109F480E0F82E9801E6
:1076E0008E018091960CF81659F7C901B80140E057
:1076F00050E05DDFDF91CF911F910F91FF90EF90F0
:107700000895AF92BF92CF92DF92EF92FF920F93C4
:107710001F93CF93DF93EB018A016115710509F483
:1077200066C04115510509F462C0DAA4CBA4BCA41B
:10773000ADA46EA17FA188A599A52D2D3C2D4B2D23
:107740005A2D0E94D3FA882309F451C08FA98823A7
:1077500009F043C0F801E6A0F7A000A511A56D2D22
:107760007C2D8B2D9A2DA80197010E94E1FC181603
:10777000A4F5C801B701A80197010E94B3FD7B01E0
:107780008C016AA97BA98CA99DA9905820E030E0C2
:1077900040E050EC0E94B3FD2EA53FA548A959A991
:1077A0000E94B3FD9B01AC01C801B7010E94FAF928
:1077B0000E9420FE7B018C016D2D7C2D8B2D9A2D3E
:1077C0009701A8010E94D3FA882324F4ED2CFC2C05
:1077D0000B2D1A2DC701D80104C08D2D9C2DAB2D6A
:1077E000BA2D8EA39FA3A8A7B9A781E08EABDF9186
:1077F000CF911F910F91FF90EF90DF90CF90BF90AE
:10780000AF900895CF92DF92EF92FF920F93DF93A4
:10781000CF930F920F92CDB7DEB78091960C8FB7B2
:10782000F894F090970C8FBF8091960C90E0409662
:107830008F1991098F7090700497FCF00091960C4D
:1078400003500F70CC24DD2440E050E091E5E92E98
:1078500012C0802F002309F480E1082F01500E9DF3
:10786000C00111248A57984F9A838983B60149DF52
:10787000A601C980DA800F1561F70F900F90CF91A4
:10788000DF910F91FF90EF90DF90CF9008951F93BD
:1078900060918412209186129091970C8091960CA1
:1078A000981711F4122F1CC04091970C242F30E030
:1078B00081E590E0289FF001299FF00D389FF00DA1
:1078C0001124EA57F84FE85BFF4F60813496E0815E
:1078D00002C04F5F4F708091960C4817D1F71E2F52
:1078E00088E070E00E9415F486E0612F70E00E944D
:1078F00015F413DC1F9108951092960C1092970CBA
:1079000080E1E5E7F7E0DF011D928A95E9F780E085
:1079100090E0A0E0B0E080939C0C90939D0CA0932D
:107920009E0CB0939F0C8093A00C9093A10CA093FD
:10793000A20CB093A30C8093A40C9093A50CA093DD
:10794000A60CB093A70C8093A80C9093A90CA093BD
:10795000AA0CB093AB0C8093980C9093990CA093C5
:107960009A0CB0939B0C08952F923F924F925F9286
:107970006F927F928F929F92AF92BF92CF92DF923F
:10798000EF92FF920F931F93DF93CF93CDB7DEB7A4
:1079900066970FB6F894DEBF0FBECDBF9E8B8D8B62
:1079A0006A017B0148015901DC01D8966D917D91F6
:1079B0008D919C91DB970E9473FB698B7A8B8B8BEB
:1079C0009C8BA70196010E94B3FD0E94C0FA0E9401
:1079D00047FB6D837E838F83988769897A898B893A
:1079E0009C89A50194010E94B3FD0E94C0FA0E94E7
:1079F00047FB69837A838B839C832D813E814F81F2
:107A00005885283731054105510540F448E750E0D5
:107A100060E070E04D835E836F83788769817A814F
:107A20008B819C81683771058105910540F488E759
:107A300090E0A0E0B0E089839A83AB83BC83AD89FA
:107A4000BE89AC5BBF4FAD90BD90CD90DC901397DD
:107A5000A454B040BE8BAD8B6D817E818F819885A3
:107A60000E9473FB6D877E878F87988BC601B50157
:107A70000E9475FB1B012C0120E030E040E050E04B
:107A80000E94D3FA882321F4E0E070E060E028C08F
:107A900069897A898B899C899B01AC010E94B3FD1D
:107AA0007B018C016D857E858F8598899B01AC015A
:107AB0000E94B3FD9B01AC01C801B7010E94F9F916
:107AC0007B018C01C201B101A20191010E94FAF96E
:107AD0009B01AC01C801B7010E94DAFAE62F692FB9
:107AE0002E2F372F482F562FB901CA010E94C0FAF6
:107AF0000E9442FB3B014C0169817A818B819C8110
:107B00000E9473FB69877A878B879C876627772714
:107B1000CB016A197B098C099D090E9475FB5B01E9
:107B20006C0120E030E040E050E00E94D3FA88236E
:107B300021F4E0E070E060E028C069857A858B85FB
:107B40009C859B01AC010E94B3FD7B018C0169897E
:107B50007A898B899C899B01AC010E94B3FD9B01B2
:107B6000AC01C801B7010E94F9F97B018C01C60183
:107B7000B501A60195010E94FAF99B01AC01C8016B
:107B8000B7010E94DAFAE62F692F2E2F372F482FE0
:107B9000562FB901CA010E94B0FBED89FE89A08869
:107BA000B188C288D38886017501E618F7080809EC
:107BB00019090E9442FBA8019701261B370B480BAD
:107BC000590B57FF71C0C201B10120E030E040E025
:107BD00050E00E94D3FA882321F4E0E070E060E0F6
:107BE00044C0C201B101A20191010E94FAF97B01D6
:107BF0008C01C601B5010E9473FB9B01AC01C80159
:107C0000B7010E94B3FD7B018C016D857E858F8558
:107C100098899B01AC010E94B3FD9B01AC01C80196
:107C2000B7010E94F9F97B018C0169857A858B8502
:107C30009C859B01AC010E94B3FD9B01AC01C80176
:107C4000B7010E94FAF97B018C01C201B10120E069
:107C500030E040E850E40E94B3FD9B01AC01C80154
:107C6000B7010E94DAFAE62F692F2E2F372F482FFF
:107C7000562FB901CA010E94C0FA0E9442FBAC0112
:107C8000CB01DA013C014D0197FE03C06624772445
:107C900043016A147B048C049D0410F035014601F5
:107CA00020E030E040E050E09FB7F8946D897E8995
:107CB000605B7F4FDB018C91A055B040BE8BAD8BDC
:107CC000882321F5FD01648A758A868A978A260DA4
:107CD000371D481D591D58962D933D934D935C9328
:107CE0005B972D813E814F815885DC962D933D9386
:107CF0004D935C93DF97A05CBF4F29813A814B8104
:107D00005C812D933D934D935C9313979FBF669633
:107D10000FB6F894DEBF0FBECDBFCF91DF911F919C
:107D20000F91FF90EF90DF90CF90BF90AF909F901A
:107D30008F907F906F905F904F903F902F9008951D
:107D40004F925F927F928F929F92AF92BF92CF920B
:107D5000DF92EF92FF920F931F93CF93DF93709078
:107D6000970CC0E0D0E021E5422E512C45C0209771
:107D7000A9F18EA9882361F4849CF001859CF00D03
:107D8000949CF00D1124EA57F84F86A9882331F10D
:107D9000EAA0FBA00CA11DA16EA17FA188A599A5B9
:107DA000A80197010E94DAFA5B016C01849CF00142
:107DB000859CF00D949CF00D1124EA57F84F66A1B4
:107DC00077A180A591A5A80197010E94DAFA8B01FD
:107DD0009C01CE01B601A501C7DD1EAA739480E106
:107DE000781609F47724849CE001859CD00D949C3E
:107DF000D00D1124CA57D84F872C992487FC909412
:107E00008091960C90E08816990609F0B0CF2097E3
:107E1000E9F0EAA0FBA00CA11DA16EA17FA188A59D
:107E200099A5A80197010E94DAFA5B016C016DEC3B
:107E30007CEC8CE49DE3A80197010E94DAFA8B01A7
:107E40009C01CE01B601A5018FDD1EAADF91CF9165
:107E50001F910F91FF90EF90DF90CF90BF90AF9068
:107E60009F908F907F905F904F900895CBDC19DCAE
:107E700067CF2F923F924F925F926F927F928F9235
:107E80009F92AF92BF92CF92DF92EF92FF920F93A9
:107E90001F93DF93CF93CDB7DEB7CD58D0400FB649
:107EA000F894DEBF0FBECDBF5C014B012A01390142
:107EB000C657DF4FE882CA58D040C557DF4FF88217
:107EC000CB58D040C457DF4F0883CC58D040C3575D
:107ED000DF4F1883CD58D040AC96DFAECEAEAC9716
:107EE0008091960C8F5F803109F480E0282F332732
:107EF00027FD309538AB2FA706C00E94D1E00E9425
:107F000060A80E948A958091970C90E04FA558A98F
:107F10008417950791F3D5016D917D918D919C9179
:107F20002091250730912607409127075091280777
:107F30000E94B3FD0E9483FDE9966FAFE997EA9630
:107F40007FAFEA97EB968FAFEB97EC969FAFEC97EE
:107F5000F4016081718182819381209129073091A0
:107F60002A0740912B0750912C070E94B3FD0E94D5
:107F700083FDED966FAFED97EE967FAFEE97EF96A0
:107F80008FAFEF97C158DF4F9883CF57D040D201C2
:107F90006D917D918D919C9120912D0730912E07AF
:107FA00040912F07509130070E94B3FD0E9483FD3E
:107FB000C058DF4F6883C058D040CF57DF4F788319
:107FC000C158D040CE57DF4F8883C258D040CD57DC
:107FD000DF4F9883C358D040B0918212AA96BFAFAA
:107FE000AA97BB2371F4F30160817181828193812F
:107FF0002091310730913207409133075091340777
:1080000012C0AA96FFADAA97F130C1F4D3016D91C9
:108010007D918D919C91209135073091360740914B
:108020003707509138070E94B3FD0E9483FDAC01D1
:10803000CB01DA0189A79AA7ABA7BCA780918107DA
:1080400090918207A0918307B091840729A53AA552
:108050004BA55CA5281739074A075B0709F4AEC092
:10806000AA963FADAA97E32FF0E0EE0FFF1FEE0FA9
:10807000FF1FE559FB4E60817181828193812091C0
:108080009C0330919D0340919E0350919F030E9459
:10809000D3FA88237CF549A55AA56BA57CA5409306
:1080A0008107509382076093830770938407E4EA03
:1080B000F9E0949108C08091C00085FFFCCF9093B7
:1080C000C600319694919923B1F7E8ECF9E09491C8
:1080D00008C08091C00085FFFCCF9093C600319608
:1080E00094919923B1F78091C00085FFFCCF8AE07D
:1080F0008093C6008091810790918207A0918307A9
:10810000B091840729A53AA54BA55CA5281B390B7E
:108110004A0B5B0BCA01B90157FF07C090958095C8
:10812000709561957F4F8F4F9F4F0E9475FB7B012C
:108130008C016091310770913207809133079091E3
:10814000340720E030E44FE054E40E94B3FD9B018B
:10815000AC01C801B7010E94E1FC18167CF549A5E5
:108160005AA56BA57CA54093810750938207609325
:10817000830770938407E4EAF9E0949108C0809142
:10818000C00085FFFCCF9093C6003196949199234F
:10819000B1F7EAEAF9E0949108C08091C00085FF48
:1081A000FCCF9093C600319694919923B1F78091BA
:1081B000C00085FFFCCF8AE08093C6008091960CBA
:1081C000682F70E0A9967FAF6EAFA99781E590E028
:1081D000689FF001699FF00D789FF00D1124EA5718
:1081E000F84FE05BFF4F1082E055F040809175073B
:1081F00090917607A0917707B0917807A7968CAFFA
:108200009DAFAEAFBFAFA797EC962CAD3DAD4EADD9
:108210005FADEC97281B390B4A0B5B0BA3962CAF79
:108220003DAF4EAF5FAFA39720833183428353832B
:1082300057FF0DC0DA01C901B095A09590958195C1
:108240009F4FAF4FBF4F80839183A283B3834091F1
:10825000790750917A0760917B0770917C076F9640
:108260004CAF5DAF6EAF7FAF6F97C458DF4F888163
:108270009981AA81BB81CC57D040841B950BA60B5A
:10828000B70B6B968CAF9DAFAEAFBFAF6B9781E571
:1082900090E0A996AEADBFADA997A89FF001A99FA8
:1082A000F00DB89FF00D1124EA57F84F6B962CADE6
:1082B0003DAD4EAD5FAD6B972483358346835783C9
:1082C00057FF0DC0DA01C901B095A0959095819531
:1082D0009F4FAF4FBF4F84839583A683B783409151
:1082E0007D0750917E0760917F07709180076796A8
:1082F0004CAF5DAF6EAF7FAF6797C058DF4F8881DF
:108300009981AA81BB81C058D040841B950BA60BD4
:10831000B70B63968CAF9DAFAEAFBFAF639781E5F0
:1083200090E0A996AEADBFADA997A89FF001A99F17
:10833000F00DB89FF00D1124EA57F84F63962CAD5D
:108340003DAD4EAD5FAD6397208731874287538740
:1083500057FF0DC0DA01C901B095A09590958195A0
:108360009F4FAF4FBF4F80879187A287B3872090E1
:10837000810730908207409083075090840749A579
:108380005AA56BA57CA542195309640975094DA32B
:108390005EA36FA378A7AA965FADAA97E52FF0E03A
:1083A000EE0FFF1FEE0FFF1FE652FC4F6081718141
:1083B000828193812F966CAF7DAF8EAF9FAF2F9749
:1083C0008091D8039091D9032B969FAF8EAF2B97B6
:1083D0006DA17EA18FA198A597FF07C0909580956C
:1083E000709561957F4F8F4F9F4F0E9475FB2F9621
:1083F0002CAD3DAD4EAD5FAD2F970E94B3FD0E94F9
:1084000042FB2B96AEADBFAD2B979D01442737FDA8
:108410004095542F0E9485FE24E630E040E050E075
:108420000E94EDFE81E590E0A9966EAD7FADA99723
:10843000689FF001699FF00D789FF00D1124EA57B5
:10844000F84FDF011C96248711963C9311971296E2
:108450004C93129713965C93608071808280938016
:10846000A480B580C680D780E084F184028513851E
:10847000C901DA018E159F05A007B10714F4D801D0
:10848000C7018A159B05AC05BD0514F4D601C501CD
:108490009C01AD0186159705A805B90514F4A40142
:1084A000930181E590E0A996AEADBFADA997A89FD5
:1084B000B001A99F700DB89F700D11246A57784FB5
:1084C000FB01208B318B428B538B263031054105CC
:1084D000510510F40C94A04BE85BFF4F809184127F
:1084E00090918512AA2797FDA095BA2F808391833A
:1084F000A283B383FB01E45BFF4F809186129091CE
:108500008712AA2797FDA095BA2F80839183A28313
:10851000B383DB0190961C92EC962CAD3DAD4EAD35
:108520005FADEC97A7968CAD9DADAEADBFADA797F7
:10853000281739074A075B0724F481E0DB0190968E
:108540008C93C458DF4F288139814A815B81CC5795
:10855000D0406F966CAD7DAD8EAD9FAD6F972617F9
:1085600037074807590794F481E590E0A996AEAD26
:10857000BFADA997A89FF001A99FF00DB89FF00D7E
:108580001124EA57F84F80A1826080A3C058DF4FC2
:10859000288139814A815B81C058D04067966CAD93
:1085A0007DAD8EAD9FAD67972617370748075907F2
:1085B00094F481E590E0A996AEADBFADA997A89FD0
:1085C000F001A99FF00DB89FF00D1124EA57F84F64
:1085D00080A1846080A329A53AA54BA55CA522159E
:1085E00033054405550594F481E590E0A9964EAD18
:1085F0005FADA997489FF001499FF00D589FF00D7E
:108600001124EA57F84F80A1886080A381E590E0AB
:10861000A9966EAD7FADA997689FF001699FF00D97
:10862000789FF00D1124EA57F84FAC96AEADBFAD70
:10863000AC978C9181A3208131814281538129960D
:108640002CAF3DAF4EAF5FAF2997211531054105E6
:10865000510509F0179881E590E0A9964EAD5FAD00
:10866000A997489FF001499FF00D589FF00D1124E4
:10867000EA57F84F64807580868097806114710492
:108680008104910409F0169881E590E0A9966EADF9
:108690007FADA997689FF001699FF00D789FF00D5D
:1086A0001124EA57F84FA084B184C284D384A11462
:1086B000B104C104D10409F0159881E590E0A996B0
:1086C000AEADBFADA997A89FF001A99FF00DB89FCF
:1086D000F00D1124EA57F84F84859585A685B78556
:1086E0000097A105B10551F01498209049073090EA
:1086F0004A0740904B0750904C0708C020906107F4
:10870000309062074090630750906407C657DF4F70
:108710006881CA58D040C557DF4F7881CB58D040C8
:10872000C457DF4F8881CC58D040C357DF4F988162
:10873000CD58D040A20191010E94D3FA87FD16C006
:10874000C657DF4F8881CA58D040C557DF4F988140
:10875000CB58D040C457DF4FA881CC58D040C35726
:10876000DF4FB881CD58D0401C012D01A3966CADD0
:108770007DAD8EAD9FADA3970E9475FB209125071F
:108780003091260740912707509128070E94DAFA76
:10879000E5966FAFE597E6967FAFE697E7968FAFE2
:1087A000E797E8969FAFE897AC01CB01DA018983A0
:1087B0009A83AB83BC836B966CAD7DAD8EAD9FAD64
:1087C0006B970E9475FB2091290730912A074091F1
:1087D0002B0750912C070E94DAFAE1966FAFE197D0
:1087E000E2967FAFE297E3968FAFE397E4969FAF71
:1087F000E497AC01CB01DA018D839E83AF83B88708
:1088000063966CAD7DAD8EAD9FAD63970E9475FB99
:1088100020912D0730912E0740912F07509130075E
:108820000E94DAFAAD966FAFAD97AE967FAFAE9776
:10883000AF968FAFAF97E0969FAFE097AC01CB01BB
:10884000DA0189879A87AB87BC87AA96BFADAA97BA
:10885000BB2321F56DA17EA18FA198A50E9475FB78
:1088600020913107309132074091330750913407FE
:108870000E94DAFA2F962CAD3DAD4EAD5FAD2F972D
:108880000E94B3FD7B018C012B96EEADFFAD2B97C3
:10889000BF01882777FD8095982F28C0AA96FFAD45
:1088A000AA97F130A9F56DA17EA18FA198A50E948C
:1088B00075FB20913507309136074091370750916D
:1088C00038070E94DAFA2F962CAD3DAD4EAD5FAD64
:1088D0002F970E94B3FD7B018C012B962EAD3FADEF
:1088E0002B97B901882777FD8095982F0E9475FBFB
:1088F0009B01AC01C801B7010E94B3FD20E030E04C
:1089000048EC52E40E94DAFA6D877E878F87988B55
:1089100029964CAD5DAD6EAD7FAD299746305105C2
:10892000610571052CF556E065167104810491040A
:10893000FCF466E0A616B104C104D104CCF481E5D0
:1089400090E0A996AEADBFADA997A89FF001A99FF1
:10895000F00DB89FF00D1124EA57F84F8D859E85D4
:10896000AF85B889BF7786A797A7A0ABB1AB55C035
:10897000E5962FADE597E6963FADE697E7964FADC6
:10898000E797E8965FADE897B901CA010E946AFED1
:108990003B014C01E1962FADE197E2963FADE297A6
:1089A000E3964FADE397E4965FADE497B901CA0152
:1089B0000E946AFE5B016C01AD962FADAD97AE963D
:1089C0003FADAE97AF964FADAF97E0965FADE097F6
:1089D000B901CA010E946AFE7B018C01C401B30186
:1089E000A60195010E94FAF9A80197010E94FAF9DF
:1089F0000E9420FE21E530E0A9964EAD5FADA9971B
:108A0000429FF001439FF00D529FF00D1124EA5751
:108A1000F84F66A777A780AB91AB81E590E0A99668
:108A20006EAD7FADA997689FF001699FF00D789FAB
:108A3000F00D1124EA57F84F86A597A5A0A9B1A972
:108A400025968CAF9DAFAEAFBFAF259760E070E0CD
:108A500080E89FE325962CAD3DAD4EAD5FAD2597EB
:108A60000E94DAFA9B01AC01C201B1010E94B3FD80
:108A70002B013C018091960C9091970CA82FB0E0AF
:108A80005096A91BB109AF70B070BEA7ADA7A230B8
:108A9000B1050CF451C05D01CC24B7FCC094DC2CB2
:108AA000C601B5010E9475FB20E030E040E051E4D2
:108AB0000E94D3FA88230CF03FC060E074E284E7A0
:108AC00099E4A30192010E94DAFA0E9483FD7B01DE
:108AD0008C0160911107709112078091130790919A
:108AE0001407E616F7060807190730F56E197F090F
:108AF000800B910B660F771F881F991FA6019501A8
:108B00000E94CBFECA01B9010E9473FB0E9483FD43
:108B10009B01AC012E0D3F1D401F511FCA01B90121
:108B20000E9473FB9B01AC0160E074E284E799E46E
:108B30000E94DAFA2B013C0181E590E0A996EEADA6
:108B4000FFADA997E89F8001E99F100DF89F100DD8
:108B500011240A57184F25966CAD7DAD8EAD9FAD93
:108B60002597A30192010E94B3FDD80192966D93BF
:108B70007D938D939C93959750966D917D918D915A
:108B80009C9153970E9473FBA30192010E94B3FD35
:108B90000E94C0FA0E9447FBF80160AF71AF82AF3C
:108BA00093AFCC57DF4F1882C458D040CB57DF4F1C
:108BB0001882C558D040B0E82B2EAFE33A2E882457
:108BC0009924E1E0F0E0EC0FFD1FE80DF91DC30171
:108BD000B20120813181428153810E94B3FDE1E1E4
:108BE000F0E0EC0FFD1FE80DF91D608371838283B7
:108BF00093835B016C01E894D7F8F401EB5EF84FC6
:108C0000E080F18002811381C601B501A8019701BE
:108C10000E94E1FC1816CCF4C801B701A601950129
:108C20000E94DAFA6B017C01CC57DF4F6881C4588F
:108C3000D040CB57DF4F7881C558D040C101A70144
:108C400096010E94D3FA88236CF4CC57DF4F8881B9
:108C5000C458D040CB57DF4F9881C558D040D10180
:108C60006C017D0124E030E0820E931E30E183161A
:108C7000910471F0D701C601CC57DF4FC882C458A8
:108C8000D040CB57DF4F9883C558D0401D0199CFB6
:108C9000C701B60120E030E040E85FE30E94D3FA6C
:108CA00088230CF04CC08E010F5E1F4FF1E2AF2EF7
:108CB000B12CAC0EBD1ED8016D917D918D919C9112
:108CC000A70196010E94B3FDF8016193719381930E
:108CD00091938F01EA15FB0571F781E590E0A99664
:108CE0002EAD3FADA997289F8001299F100D389F79
:108CF000100D11240A57184FD80192966D917D914D
:108D00008D919C919597A70196010E94B3FDF80162
:108D100062A373A384A395A360AD71AD82AD93AD3F
:108D20000E9473FBA70196010E94B3FD0E9447FBBE
:108D3000D801D8966D937D938D939C93DB9781E5B5
:108D400090E0A996EEADFFADA997E89F8001E99F5D
:108D5000100DF89F100D11240A57184FD801509686
:108D60006D917D918D919C9153970E9473FBF801B9
:108D700026A537A540A951A90E94DAFA1B012C01AA
:108D8000F80180819181A281B3810097A105B1058D
:108D900049F584819581A681B7810097A105B10528
:108DA00009F580859185A285B3850097A105B10558
:108DB000C9F4C201B101209151073091520740918D
:108DC0005307509154070E94B3FD0E94C0FA0C5BF8
:108DD0001F4F0E9447FBD8016D937D938D939C9309
:108DE000139771C1C201B10120914D0730914E0717
:108DF00040914F07509150070E94B3FD0E94C0FA66
:108E00000E9447FB21E530E0A996EEADFFADA997A2
:108E1000E29F6001E39FD00CF29FD00C112426E862
:108E200037E0C20ED31EE4E46E2E712C6C0C7D1C58
:108E3000D3016D937D938D939C93139780906507D9
:108E400090906607A0906707B09068070E9473FB38
:108E50007B018C01F60160817181828193810E9486
:108E600075FB9B01AC01C801B7010E94B3FD7B01FA
:108E70008C01D60150966D917D918D919C91539767
:108E80000E9473FB9B01AC01C801B7010E94DAFA92
:108E90007B018C01C501B4010E9473FB9B01AC01F5
:108EA000C801B7010E94E1FC18162CF4F30180827E
:108EB0009182A282B3828090690790906A07A09005
:108EC0006B07B0906C0781E590E0A9962EAD3FADA1
:108ED000A997289F6001299FD00C389FD00C11249E
:108EE00046E857E0C40ED51E54E4652E712C6C0C78
:108EF0007D1CD3016D917D918D919C910E9473FB9E
:108F00007B018C01F60164817581868197810E94C5
:108F100075FB9B01AC01C801B7010E94B3FD7B0149
:108F20008C01D60150966D917D918D919C915397B6
:108F30000E9473FB9B01AC01C801B7010E94DAFAE1
:108F40007B018C01C501B4010E9473FB9B01AC0144
:108F5000C801B7010E94E1FC18162CF4F3018082CD
:108F60009182A282B3828090710790907207A09044
:108F70007307B090740781E590E0A9962EAD3FADE0
:108F8000A997289F6001299FD00C389FD00C1124ED
:108F900046E857E0C40ED51E44E4642E712C6C0CD8
:108FA0007D1CD3016D917D918D919C910E9473FBED
:108FB0007B018C01F60164857585868597850E9405
:108FC00075FB9B01AC01C801B7010E94B3FD7B0199
:108FD0008C01D60150966D917D918D919C91539706
:108FE0000E9473FB9B01AC01C801B7010E94DAFA31
:108FF0007B018C01C501B4010E9473FB9B01AC0194
:10900000C801B7010E94E1FC18162CF4F30180821C
:109010009182A282B38280906D0790906E07A0909B
:109020006F07B090700781E590E0A9962EAD3FAD37
:10903000A997289F6001299FD00C389FD00C11243C
:1090400046E857E0C40ED51E34E4632E712C6C0C38
:109050007D1CD3016D917D918D919C910E9473FB3C
:109060007B018C01F60160857185828593850E9464
:1090700075FB9B01AC01C801B7010E94B3FD7B01E8
:109080008C01D60150966D917D918D919C91539755
:109090000E9473FB9B01AC01C801B7010E94DAFA80
:1090A0007B018C01C501B4010E9473FB9B01AC01E3
:1090B000C801B7010E94E1FC18162CF4F30180826C
:1090C0009182A282B38281E590E0A9962EAD3FAD58
:1090D000A997289F6001299FD00C389FD00C11249C
:1090E00046E857E0C40ED51EF601EC5BFF4F6081E9
:1090F0007181828193810E9473FB7B018C01A201AB
:1091000091010E94DAFAD601D2966D937D938D93E8
:109110009C93D597C801B7012DEB37E346E051E4A6
:109120000E94B3FD0E9442FBF601648F758F868F0B
:10913000978F6090550770905607809057079090D2
:109140005807C401B30120E030E040E05FE30E9433
:10915000B3FD5B016C01298D3A8D4B8D5C8D2196A1
:109160002CAF3DAF4EAF5FAF219740915907509163
:109170005A0760915B0770915C0749AF5AAF6BAFBC
:109180007CAFCB01BA0120E030E040E05FE30E9419
:10919000B3FD7B018C0121966CAD7DAD8EAD9FAD95
:1091A00021979F77A80197010E94E1FC181644F4CB
:1091B000C601B501A80197010E94D3FA882314F4CF
:1091C000860175016D8D7E8D8F8D98A16DAB7EAB07
:1091D0008FAB98AF80915D0790915E07A0915F077C
:1091E000B091600789AB9AABABABBCABBC01CD0116
:1091F00020E030E040E05FE30E94B3FD1B012C0162
:109200006DA97EA98FA998AD9F77A20191010E94B7
:10921000E1FC181644F4C801B701A20191010E94B3
:10922000D3FA882314F41701280181E590E0A99668
:10923000AEADBFADA997A89FF001A99FF00DB89F53
:10924000F00D1124EA57F84F22A133A144A155A1F2
:1092500029A33AA34BA35CA3C201B1010E94D3FA94
:1092600087FD04C029A03AA04BA05CA04DA55EA537
:10927000423051050CF407C15091980CCA57DF4F8A
:109280005883C658D0406091990CC957DF4F688306
:10929000C758D04070919A0CC857DF4F7883C85890
:1092A000D04080919B0CC757DF4F8883C958D0406E
:1092B000652FC957DF4F7881C758D040C857DF4F57
:1092C0008881C858D040C757DF4F9881C958D040CF
:1092D00027E137EB41ED58E30E94E1FC18160CF052
:1092E000D2C069897A898B899C8920919C0C3091A4
:1092F0009D0C40919E0C50919F0C0E94F9F99B018E
:10930000AC010E94B3FD7B018C016D897E898F8940
:10931000988D2091A00C3091A10C4091A20C5091FD
:10932000A30C0E94F9F99B01AC010E94B3FD9B01C3
:10933000AC01C801B7010E94FAF90E9420FE7B012E
:109340008C01A40193010E94E1FC18165CF00F2E21
:10935000F0E06F2EF0E07F2EF0E88F2EFFE39F2EDF
:10936000F02D08C0C401B301A80197010E94DAFAE8
:109370003B014C0121966CAD7DAD8EAD9FAD21972B
:109380002091A40C3091A50C4091A60C5091A70CF3
:109390000E94F9F97B018C01E89417F9C801B70123
:1093A00029AD3AAD4BAD5CAD0E94E1FC181694F4CA
:1093B00069AD7AAD8BAD9CADA80197010E94DAFA38
:1093C0005B016C01C401B301A60195010E94D3FAAF
:1093D000882314F4640153016DA97EA98FA998AD67
:1093E0002091A80C3091A90C4091AA0C5091AB0C83
:1093F0000E94F9F97B018C01E89417F9C801B701C3
:1094000029A93AA94BA95CA90E94E1FC181694F479
:1094100069A97AA98BA99CA9A80197010E94DAFAE7
:109420007B018C01C601B501A80197010E94D3FA06
:10943000882314F48601750169A17AA18BA19CA1EE
:10944000A80197010E94B3FD7B018C01CA57DF4F31
:109450006881C658D040C957DF4F7881C758D0407F
:10946000C857DF4F8881C858D040C757DF4F988111
:10947000C958D040A80197010E94D3FA87FD19C0AE
:10948000D801C70102C0D201C101CA57DF4F88838A
:10949000C658D040C957DF4F9883C758D040C857E7
:1094A000DF4FA883C858D040C757DF4FB883C9588B
:1094B000D04081E590E0A996AEADBFADA997A89F39
:1094C0008001A99F100DB89F100D11240A57184F45
:1094D000CA57DF4F8881C658D040C957DF4F98819F
:1094E000C758D040C857DF4FA881C858D040C75789
:1094F000DF4FB881C958D040F80182A793A7A4A72D
:10950000B5A762A973A984A995A9905820E030E075
:1095100040E050EC0E94B3FDD8019E962D913D9104
:109520004D915C91D1970E94B3FD2BE037ED43E262
:109530005BE30E94FAF90E9420FEF62EE72ED82E59
:10954000C92ECA57DF4F6881C658D040C957DF4F70
:109550007881C758D040C857DF4F8881C858D0405D
:10956000C757DF4F9881C958D0402F2D3E2D4D2D24
:109570005C2D0E94D3FA87FD14C0CA57DF4FF882D2
:10958000C658D040C957DF4FE882C758D040C857A7
:10959000DF4FD882C858D040C757DF4FC882C9585C
:1095A000D04081E590E0A996EEADFFADA997E89F88
:1095B0008001E99F100DF89F100D11240A57184FD4
:1095C000CA57DF4F8881C658D040C957DF4F9881AE
:1095D000C758D040C857DF4FA881C858D040C75798
:1095E000DF4FB881C958D040F80186A397A3A0A740
:1095F000B1A762A173A184A195A12F2D3E2D4D2D60
:109600005C2D0E94D3FA18162CF081E0D801D79671
:109610008C9302C0F80117AA81E590E0A9962EADBF
:109620003FADA997289FF001299FF00D389FF00DBD
:109630001124EA57F84F81E086ABACE9BCE0FE01AB
:10964000719680E101900D928150E1F781E590E003
:10965000A9964EAD5FADA997489F6001499FD00C78
:10966000589FD00C112466E877E0C60ED71ED601AD
:109670009296ED90FD900D911C919597E092980C2B
:10968000F092990C00939A0C10939B0C96966D9106
:109690007D918D919C919997A80197010E94DAFA8A
:1096A0004B015C01C201B101A80197010E94DAFAE5
:1096B0008B019C01C601B501A4010E94B43CBFA569
:1096C000B093960C29A53AA54BA55CA520938107DC
:1096D000309382074093830750938407C058DF4F2D
:1096E000488159816A817B81C058D04040937D0771
:1096F00050937E0760937F0770938007C458DF4FB5
:10970000688179818A819B81CC57D04060937907A9
:1097100070937A0780937B0790937C07EC968CADCF
:109720009DADAEADBFADEC97809375079093760776
:10973000A0937707B09378070E94363F0E94122AC1
:10974000C357DF4F0FB6F894DEBF0FBECDBFCF912A
:10975000DF911F910F91FF90EF90DF90CF90BF901E
:10976000AF909F908F907F906F905F904F903F90C1
:109770002F900895DB010D900020E9F71197A61BAB
:10978000B70B0496AD010C94D254DF93CF930F9294
:10979000CDB7DEB769830496BE016F5F7F4F41E0AE
:1097A00050E00E94D2540F90CF91DF9108952F92F4
:1097B0003F924F925F926F927F928F929F92AF9261
:1097C000BF92CF92DF92EF92FF920F931F93DF939E
:1097D000CF93CDB7DEB7CD55D0400FB6F894DEBFEE
:1097E0000FBECDBF2F969FAF8EAF2F9761967FAFE5
:1097F0006EAF61972A0162962FAF629763960FAFA3
:1098000063976496EFAE64976896ACAEBDAECEAE8D
:10981000DFAE6897E22EFF24EE0CFF1CEE0CFF1C5F
:109820009A012E0D3F1D2D963FAF2EAF2D97D901DA
:109830006D907D908D909C90FC01EE0DFF1DC401FC
:10984000B30120813181428153810E94FAF969AFCD
:109850007AAF8BAF9CAF10E0000F111F000F111FEC
:10986000F201E00FF11F2B96FFAFEEAF2B97A08018
:10987000B180C280D3802F96EEADFFAD2F97E00F61
:10988000F11FC601B50120813181428153810E94BF
:10989000FAF96DAB7EAB8FAB98AF64962FAD649742
:1098A000E22FF0E0EE0FFF1FEE0FFF1F2F96AEAD81
:1098B000BFAD2F97AE0FBF1F4D915D916D917C9104
:1098C00029964CAF5DAF6EAF7FAF299761966EADB5
:1098D0007FAD6197E60FF71F60817181828193816F
:1098E00029962CAD3DAD4EAD5FAD29970E94F9F99B
:1098F00069AB7AAB8BAB9CAB6196AEADBFAD6197FC
:109900001C968D919D910D90BC91A02D25968CAFAC
:109910009DAFAEAFBFAF25972F96AEADBFAD2F9722
:109920001C962D913D914D915C911F9721962CAFE6
:109930003DAF4EAF5FAF2197A401930150582DA7C3
:109940003EA74FA758ABB601A501705849A75AA723
:109950006BA77CA761966EAD7FAD6197E60EF71E93
:10996000D7016D917D918D919C9129AD3AAD4BAD13
:109970005CAD0E94F9F93B014C016196EEADFFAD83
:1099800061970E0F1F1FD8016D917D918D919C9154
:109990002DA93EA94FA958AD0E94F9F95B016C01B0
:1099A0006DA57EA58FA598A9A60195010E94B3FD7E
:1099B0007B018C0169A57AA58BA59CA5A4019301C7
:1099C0000E94B3FD9B01AC01C801B7010E94F9F9E7
:1099D0001B012C016DA57EA58FA598A9A40193015B
:1099E0000E94B3FD7B018C0169A57AA58BA59CA57E
:1099F000A60195010E94B3FD9B01AC01C801B7010E
:109A00000E94FAF99B01AC01C201B1010E946DFAFA
:109A10005B016C0120E030E040E050E00E94D3FAAE
:109A2000882354F4C601B5012BED3FE049EC50E426
:109A30000E94FAF95B016C01E8968FADE8978823E4
:109A400051F0C601B5012BED3FE049EC50E40E9416
:109A5000F9F95B016C01C601B501E7962CAD3DAD8E
:109A60004EAD5FADE7970E94B3FD29A93AA94BA976
:109A70005CA95F770E94EEFC7B018C012FE632E14E
:109A800043E85AE30E94D3FA87FDF6C1C801B70143
:109A90000E94B0FB0E9447FB78A76FA3672B21F4BD
:109AA000E1E0F0E0F8A7EFA32FA138A5B90180E02D
:109AB00090E00E9473FB7B018C01C601B501A801F7
:109AC00097010E94DAFA6BA37CA38DA39EA369A9D8
:109AD0007AA98BA99CA9A80197010E94DAFA6F8F35
:109AE00078A389A39AA325966CAD7DAD8EAD9FAD6D
:109AF000259721962CAD3DAD4EAD5FAD21970E94CF
:109B0000F9F9A80197010E94DAFA6B8F7C8F8D8F8B
:109B10009E8F6BA17CA18DA19EA120E030E040E052
:109B20005FEB0E94B3FD2BA13CA14DA15EA10E9461
:109B3000B3FD20E030E040E85FE30E94FAF96F8B6C
:109B4000788F898F9A8F64963FAD6497E32FF0E00A
:109B5000EE0FFF1FEE0FFF1F9E012F5F3F4FE20F23
:109B6000F31F29964CAD5DAD6EAD7FAD2997408357
:109B70005183628373832F96AEADBFAD2F971C9632
:109B80004D915D916D917C911F974D875E876F8799
:109B9000788B41E050E05A8B498B662462967FAD0A
:109BA0006297672F70E0660F771F660F771FC901F6
:109BB000860F971F6A969FAF8EAF6A976396BFAD69
:109BC0006397AB2FB0E0AA0FBB1FAA0FBB1F21E00A
:109BD00030E02C0F3D1F2A0F3B1F6C963FAF2EAF7E
:109BE0006C976E96FFAFEEAF6E971AC138E13615DF
:109BF0000CF446C06DA57EA58FA598A92BA13CA10C
:109C00004DA15EA10E94B3FD7B018C0169A57AA5DF
:109C10008BA59CA52F89388D498D5A8D0E94B3FD47
:109C20009B01AC01C801B7010E94FAF97B018C01CC
:109C30006DA57EA58FA598A92F89388D498D5A8D40
:109C40000E94B3FD5B016C0169A57AA58BA59CA55B
:109C50002BA13CA14DA15EA10E94B3FD9B01AC01D3
:109C6000C601B5010E94F9F96DA77EA78FA798AB31
:109C70006394C701D80189A79AA7ABA7BCA765C001
:109C800049895A89BA0180E090E00E9473FB2BA1B8
:109C90003CA14DA15EA10E94B3FD7B018C01C801D6
:109CA0000E94D7FA6B8B7C8B8D8B9E8BB701C80182
:109CB0000E9416FE3B014C012D96AEADBFAD2D9717
:109CC000ED90FD900D911C9117FB109517F91095D3
:109CD0002B96EEADFFAD2B972080318042805380D4
:109CE000C801B7012B893C894D895E890E94B3FD6B
:109CF0005B016C01C201B101A40193010E94B3FD9B
:109D00009B01AC01C601B5010E94FAF96DA77EA7BF
:109D10008FA798ABC801B701A40193010E94B3FDBE
:109D20007B018C01C201B1012B893C894D895E897F
:109D30000E94B3FD9B01AC01C801B7010E94F9F973
:109D400069A77AA78BA79CA7662469AD7AAD8BAD6E
:109D50009CAD2DA53EA54FA558A90E94FAF96A967B
:109D6000AEADBFAD6A976D937D938D939C93139722
:109D70006DA97EA98FA998AD29A53AA54BA55CA58B
:109D80000E94FAF96C96EEADFFAD6C97608371831B
:109D9000828393836E96AEADBFAD6E976D917D91CC
:109DA0008D919C912F8D38A149A15AA10E94FAF959
:109DB0006E96EEADFFAD6E97608371838283938361
:109DC0006D857E858F8598892B8D3C8D4D8D5E8D23
:109DD0000E94FAF96D877E878F87988BCE01019656
:109DE0000E9426A6CE010196BE016B5F7F4FAE0199
:109DF000475F5F4F9E01235F3F4F6896ECACFDAC21
:109E00000EAD1FAD6897F8E7CF2ED12CCC0EDD1E1E
:109E10000E94393F29893A892F5F3F4F3A8B298B1E
:109E200049895A896FA178A54617570708F4DECEED
:109E300061964EAD5FAD6197485F5F4F61962EAD05
:109E40003FAD6197245F3F4F61968EAD9FAD6197A7
:109E5000DC0114966196BFAFAEAF6197BD01689605
:109E6000ECACFDAC0EAD1FAD6897E8E7CE2ED12C63
:109E7000CC0EDD1E0E94393FC35ADF4F0FB6F89457
:109E8000DEBF0FBECDBFCF91DF911F910F91FF902D
:109E9000EF90DF90CF90BF90AF909F908F907F908A
:109EA0006F905F904F903F902F900895CF93DF93E6
:109EB000EB01DC0190E020E03EE28C91803269F021
:109EC000283029F4FE01E90FF11D30839F5FFE0168
:109ED000E90FF11D8C9180839F5F2F5F11962B30CE
:109EE00061F7C90FD11D1882DF91CF9108950F93AB
:109EF0001F93CF93DF93DC01EB018A0180E090E0B8
:109F000020E2FE01E80FF91F208301968B309105B6
:109F1000C1F757E040E024C0622F2E3219F082EEE4
:109F200099E007C05A3051F15AE048E018C03217A2
:109F300029F1FC01019634913323C9F75417F0F04D
:109F40002132E0F02F37D0F4822F81568A3110F47D
:109F5000622F6052FE01E40FF11D60834F5F119686
:109F60002C91222311F02F32B9F6F801B183A0838E
:109F700090E08881803219F091E001C090E0892F53
:109F8000DF91CF911F910F9108956F927F928F92E1
:109F90009F92AF92BF92CF92DF92EF92FF920F9378
:109FA0001F93CF93DF93EC017A018B012B81222346
:109FB00009F480C089899A89AB89BC89841795077F
:109FC000A607B70708F476C085C0E114F1040105BF
:109FD000110551F41C821D821E821F82188619866B
:109FE0001A861B8681E067C0288539854A855B858E
:109FF000E98DFA8D858590E00996215030404040EA
:10A00000504039014A01082E04C0969487947794F1
:10A0100067940A94D2F72F5F3F4F4F4F5F4F0894DA
:10A02000E108F108010911095701680104C0D6943B
:10A03000C794B794A7948A95D2F70894E11CF11CB1
:10A04000011D111DA614B704C804D90428F0211558
:10A0500031054105510549F48D899E89AF89B88D37
:10A060008C839D83AE83BF8316C0A618B708C8082B
:10A07000D90811C04C815D816E817F81898D9A8D57
:10A0800094010E9446360894A108B108C108D1087D
:10A09000882331F40FC084E0882E912C8C0E9D1EF5
:10A0A000A114B104C104D10429F7E886F9860A870E
:10A0B0001B8798CF80E0DF91CF911F910F91FF9088
:10A0C000EF90DF90CF90BF90AF909F908F907F9058
:10A0D0006F900895223009F078CFE7CFCF93DF93C8
:10A0E000EC018C859D85AE85BF8540E0611141E026
:10A0F000BC01CD010E942034882319F420E030E017
:10A100000AC08889282F30E095E0220F331F9A95E6
:10A11000E1F7265F3A4FC901DF91CF9108950F9380
:10A120001F93CF93DF938C01FC0183818823D9F1A6
:10A13000818187FF35C0C80161E0D0DFEC01009765
:10A1400091F18881853E79F1F8018381823040F474
:10A1500081899289A389B4898C8F9D8FAE8FBF8F9F
:10A16000F80185899689A789B08D9B8F8A8FCD014B
:10A17000AA27BB279D8B8C8BE091B00CF091B10C82
:10A18000309751F0BE016A5E7F4FCE014896199517
:10A19000888D998D9B8B8A8BF80181818F77818344
:10A1A0000E94E53304C081E0F801808380E0DF9104
:10A1B000CF911F910F9108950F931F938C01AFDFE3
:10A1C000F80113821F910F910895FC018381882368
:10A1D00011F0CF01F1CF0895CF93DF93FC01EB0194
:10A1E0008381882381F08250823020F48FE288833B
:10A1F000198207C0CF0160E071DF009721F0BE0136
:10A2000055DE81E001C080E0DF91CF9108956F922B
:10A210007F928F929F92AF92BF92CF92DF92EF92F6
:10A22000FF920F931F93DF93CF9300D00F92CDB780
:10A23000DEB77C015A016B01DC0113968C911397F8
:10A24000813009F08EC011968C9181FF8AC09DC02B
:10A250000097A105B10511F481E084C0F701608485
:10A26000718482849384C701B601A5018EDE8823A0
:10A2700009F477C0D70159968D919C915A97A114F2
:10A28000B104C104D10489F455964D915D916D914D
:10A290007C9158970E94BB36882309F462C0F7016D
:10A2A000158A168A178A108E44C0D70114964D91CC
:10A2B0005D916D917C9117979E012F5F3F4F0E949A
:10A2C0004636882309F44DC0D7015996ED91FC918B
:10A2D0005A9749815A816B817C818789803149F401
:10A2E000483FBFEF5B07B0E06B07B0E07B0748F08B
:10A2F00020C0483F8FEF58078FEF68078FE078073F
:10A30000C0F4CF010E94BB36882359F1D7011496BF
:10A310004D915D916D917C91179759968D919C917E
:10A320005A970FEF1FEF2FEF3FE00E94C0358823B1
:10A33000C1F0F701A18AB28AC38AD48A8181806878
:10A340008183C701ECDE882361F0B601A5016A14A0
:10A350007B048C049D0410F4B401A301C70115DE35
:10A3600001C080E00F900F900F900F90CF91DF9180
:10A370001F910F91FF90EF90DF90CF90BF90AF9023
:10A380009F908F907F906F900895F70181899289B7
:10A39000A389B48984179507A607B70708F058CF93
:10A3A000E0CFCF93DF93EC0140E050E060E070E05D
:10A3B0002EDF882361F0CE0161E090DEFC01009782
:10A3C00031F085EE80831B820E94E53301C080E07E
:10A3D000DF91CF9108952F923F924F925F926F92AB
:10A3E0007F928F929F92AF92BF92CF92DF92EF9225
:10A3F000FF920F931F93CF93DF93EC012A018B8180
:10A40000882309F4B6C0898180FFB3C0C8C0250184
:10A410004E185F083B0174E0272E312C2C0E3D1E98
:10A420004201A1C0288539854A855B856FEFA62E3C
:10A4300061E0B62EA222B3228B8179018A0199E0D4
:10A4400016950795F794E7949A95D1F7E98DFA8DCB
:10A45000823049F4428D538D648D758D4E0D5F1D94
:10A46000601F711F3FC0D480DA94DE20A114B104B4
:10A47000D9F4DD20C9F4211531054105510549F410
:10A480008D899E89AF89B88D8C839D83AE83BF8370
:10A490000BC04C815D816E817F81CF0191010E9453
:10A4A0004636882309F465C0E98DFA8D4C815D81BB
:10A4B0006E817F814250504060407040058404C0EE
:10A4C000440F551F661F771F0A94D2F7868597851C
:10A4D000A089B189480F591F6A1F7B1F4D0D511D5F
:10A4E000611D711D80E092E08A199B098401881525
:10A4F000990508F48C0182E00030180709F067C064
:10A500008091060590910705A0910805B091090575
:10A51000481759076A077B0709F459C080910A0751
:10A5200090910B0793010E949AE9882349F421C076
:10A530009501265F3A4FC301B901A8010E94322755
:10A54000600E711E980140E050E088859985AA85CB
:10A55000BB85820F931FA41FB51F88879987AA8781
:10A56000BB87801A910A8114910409F05BCFA20184
:10A5700002C04FEF5FEFCA01DF91CF911F910F91A2
:10A58000FF90EF90DF90CF90BF90AF909F908F9013
:10A590007F906F905F904F903F902F900895A98883
:10A5A000BA88CB88DC88E884F9840A851B859A01FF
:10A5B00040E050E0D601C5018E199F09A00BB10BF8
:10A5C000281739074A075B0708F021CF23CFCB01B3
:10A5D000BA0140E00E942034882309F0A9CFC9CFF6
:10A5E000CF92DF92EF92FF920F931F93CF93DF935F
:10A5F0007C01EB018A01FC018381823008F46EC08A
:10A6000080859185A285B3858F719070A070B070A0
:10A610000097A105B10509F061C06CC0F801108276
:10A62000EDE0CE2ED12CC701BE0140E250E0D3DEDA
:10A630009C018032910521F0009709F04FC050C075
:10A640004881442309F44CC0453E69F34E3259F326
:10A650008B858F738F30E9F501151105D1F18A8D46
:10A660009B8D892BB1F5842F90E08F7190700097AE
:10A6700081F1833091056CF58C9D90018D9D300D9D
:10A680009C9D300D11242D503040F801E20FF31F36
:10A69000898180838B8181838D8182838F81838374
:10A6A000898584838E858583888986838A89878343
:10A6B0008C8980878E898187888D82878C8D83871E
:10A6C0008E8D8487888186FF04C0F801E20FF31F16
:10A6D00015868B8583FDA7CF822F03C08FEF01C026
:10A6E00080E0DF91CF911F910F91FF90EF90DF906D
:10A6F000CF9008954115510509F090CF91CFDF9388
:10A70000CF930F92CDB7DEB7BE016F5F7F4F41E0B1
:10A7100050E061DE019719F02FEF3FEF03C0898110
:10A72000282F30E0C9010F90CF91DF910895EF926B
:10A73000FF920F931F93CF93DF93EC018B818230B5
:10A7400030F1E884F9840A851B85CE01D8DF97FDB6
:10A750001EC088859985AA85BB854F96A11DB11D10
:10A7600088879987AA87BB87A5E016950795F794F0
:10A77000E794AA95D1F72E2D30E02F703070F5E0D8
:10A78000220F331FFA95E1F7265F3A4F02C020E00F
:10A7900030E0C901DF91CF911F910F91FF90EF90B1
:10A7A00008950F931F93CF93DF93EC018B018B815F
:10A7B000882309F040C0FB018789803109F041C03E
:10A7C00082E08B831D8A1E8A1F8A188E808D918D50
:10A7D000A0E0B0E045E0880F991FAA1FBB1F4A9573
:10A7E000D1F7898B9A8BAB8BBC8B13C083E08B83A7
:10A7F000F801428D538D648D758D4D8B5E8B6F8B03
:10A80000788F9E012F5E3F4FC8010E941737882323
:10A8100091F01A8F098F81E089831C821D821E822C
:10A820001F82188619861A861B861C861D861E8620
:10A830001F86188A01C080E0DF91CF911F910F9190
:10A8400008958032C1F7D2CF1F93CF93DF93EC01ED
:10A85000142F262F30E0F90175E0EE0FFF1F7A95D7
:10A86000E1F7E65FFA4F8385817121F0842F8271D1
:10A8700009F067C08091060590910705A091080531
:10A88000B09109058C879D87AE87BF87688BF901DA
:10A8900065E0EE0FFF1F6A95E1F7E65FFA4F8489E6
:10A8A0009589A0E0B0E0DC01992788278D8B9E8BED
:10A8B000AF8BB88F228D338DA90160E070E0482BFB
:10A8C000592B6A2B7B2B4D8B5E8B6F8B788F8385FF
:10A8D00090E088719070009751F4848D958DA68DCD
:10A8E000B78D898B9A8BAB8BBC8B81E00CC040976A
:10A8F00041F59E012F5E3F4F898D9A8D0E9417373B
:10A900008823F9F084E08B83812F8F7089831C82E8
:10A910001D821E821F82188619861A861B8614FFC6
:10A9200016C0CE0140E050E060E070E070DC8823AB
:10A9300071F409C049895A896B897C89CE0125DB6C
:10A9400002C01B8280E0DF91CF911F91089515FD19
:10A95000F1CF81E0F8CFCF93DF93EC019C012C5F26
:10A960003F4F898D9A8D41E050E060E070E00E9499
:10A9700082378823A1F08D899E89AF89B88D009791
:10A98000A105B10559F48C819D81AE81BF818D8B6C
:10A990009E8BAF8BB88F89818068898381E0DF913E
:10A9A000CF9108952F923F924F925F927F928F9214
:10A9B0009F92AF92BF92CF92DF92EF92FF920F934E
:10A9C0001F93DF93CF9300D000D0CDB7DEB76C01DB
:10A9D000162F072F5E834D83DC0113968C911397FE
:10A9E000813009F06CC111968C9181FF68C185C1DD
:10A9F000F601418952896389748980859185A28590
:10AA0000B38584179507A607B70729F0C601BDDAF5
:10AA1000882309F454C1812F902F9C0119014D8086
:10AA20005E8012C1D6015996ED91FC915A97DA01D8
:10AA3000C90149E0B695A795979587954A95D1F7AD
:10AA400074807A9478228FEF882E81E0982E82226B
:10AA50009322772009F052C08114910409F04EC06E
:10AA6000D60114964D915D916D917C91179741158A
:10AA700051056105710581F455968D919D910D905B
:10AA8000BC91A02D0097A105B10561F1F601848369
:10AA90009583A683B78332C0CF019E012F5F3F4FBE
:10AAA0000E944636882309F40AC129813A814B81E4
:10AAB0005C81D6015996ED91FC915A978789803136
:10AAC00049F4283FBFEF3B07B0E04B07B0E05B071E
:10AAD00070F008C0283FEFEF3E07EFEF4E07EFE0C2
:10AAE0005E0728F0C60137DF882341F4E8C0D601AD
:10AAF00014962D933D934D935C93179780E092E0CD
:10AB00008819990952018415950508F45C01D6014C
:10AB10005996ED91FC915A971496ED90FD900D91F8
:10AB20001C9117978EEF9FEFAFEFBFEFE80EF91E66
:10AB30000A1F1B1F058404C0EE0CFF1C001F111F01
:10AB40000A94D2F786859785A089B189E80EF91E07
:10AB50000A1F1B1FE70CF11C011D111D90E0A91617
:10AB600092E0B90639F58091060590910705A0910C
:10AB70000805B09109058E159F05A007B10771F46E
:10AB800010920C078FEF9FEFAFEFBFEF809306059A
:10AB900090930705A0930805B093090580910A07D3
:10ABA00090910B07B801A70191010E94E7E8882363
:10ABB000B9F585C08114910419F5D60118962D9127
:10ABC0003D914D915C911B9751968D919D910D906A
:10ABD000BC91A02D281739074A075B0788F00E940F
:10ABE000E533882309F46BC081E080930C07E09281
:10ABF0000605F0920705009308051093090508C0A3
:10AC0000C801B70141E00E942034882309F457C0ED
:10AC10009401265F3A4FC901B101A5010E94322774
:10AC2000950140E050E0F60180859185A285B385CD
:10AC3000820F931FA41FB51F80879187A287B387B8
:10AC40002A0C3B1C4A185B08D60118962D913D91A1
:10AC50004D915C911B974114510409F0E3CE51963C
:10AC60008D919D910D90BC91A02D82179307A40703
:10AC7000B50748F4F601218B328B438B548B8181CD
:10AC80008068818311C08091B00C9091B10C892BA8
:10AC900059F08D819E81892B39F0D60111968C91C6
:10ACA0001197806811968C93F601818183FF04C00F
:10ACB000C60135DA882319F04D815E8105C081E037
:10ACC000D6018C934FEF5FEFCA0126960FB6F8942A
:10ACD000DEBF0FBECDBFCF91DF911F910F91FF90CF
:10ACE000EF90DF90CF90BF90AF909F908F907F902C
:10ACF0005F904F903F902F90089582FD79CE8BCE3C
:10AD0000DF92EF92FF920F931F93CF93DF93EC01AB
:10AD100089899A89AB89BC89805E9F4FAF41B040D9
:10AD200008F070C0CE0117DE882309F46BC00E94C2
:10AD3000E533882309F466C0E98DFA8DEC80FD8047
:10AD40000E811F818EEF9FEFAFEFBFEFE80EF91E70
:10AD50000A1F1B1F058404C0EE0CFF1C001F111FDF
:10AD60000A94D2F786859785A089B189E80EF91EE5
:10AD70000A1F1B1F81E080930C07E0920605F092EA
:10AD80000705009308051093090580E092E0EAE0CA
:10AD9000F5E0DF019C011D9221503040E1F7DD24F8
:10ADA000D39411C0B801A7014D0D511D611D711D36
:10ADB00080910A0790910B072AE035E00E94E7E8AE
:10ADC000882301F1D394E98DFA8D8481D81650F34C
:10ADD00020E032E040E050E0058404C0220F331F41
:10ADE000441F551F0A94D2F789899A89AB89BC8977
:10ADF000820F931FA41FB51F898B9A8BAB8BBC8BC3
:10AE000081E001C080E0DF91CF911F910F91FF9011
:10AE1000EF90DF9008958F929F92AF92BF92CF9262
:10AE2000DF92EF92FF920F931F93CF93DF936C010A
:10AE3000EB01942E852EA22E898D9A8DD6015A96DD
:10AE40009C938E935997CB0140E050E060E070E016
:10AE50009CD8BB2437C0CE016ADCFC01009709F402
:10AE600090C055E016950795F794E7945A95D1F759
:10AE70001E2D1F708081882311F0853EC9F4BB20F0
:10AE800099F42091060530910705409108055091ED
:10AE90000905D6011C962D933D934D935C931F9706
:10AEA00050961C93BB24B3948081882359F418C016
:10AEB000892D982DBF014BE050E00E942527009777
:10AEC00009F46DC0E884F9840A851B8589899A890B
:10AED000AB89BC89E816F9060A071B0708F4BBCF43
:10AEE000A6FE4FC0A1FE4DC0BB2049F0F60110895F
:10AEF000C60161E0F3D8EC01009761F442C08B8198
:10AF0000823009F43EC0CE01FBDE8823D1F110E08F
:10AF1000CAE0D5E080E2DE011D928A95E9F7DE0104
:10AF2000292D382DC901FC018BE001900D92815033
:10AF3000E1F7E091B00CF091B10C309739F0BE011F
:10AF4000625F7F4FCE014096199508C081E298E27A
:10AF5000998B888B80E098E09F878E878889998974
:10AF60009B8B8A8B998F888F8E859F859F8B8E8BED
:10AF70000E94E533882329F0C601612F4A2D64DC45
:10AF800001C080E0DF91CF911F910F91FF90EF9072
:10AF9000DF90CF90BF90AF909F908F900895A7FEC5
:10AFA000EBCFEFCF2F923F924F925F926F927F92B3
:10AFB0008F929F92AF92BF92CF92DF92EF92FF92C9
:10AFC0000F931F93DF93CF93CDB7DEB7C654D04016
:10AFD0000FB6F894DEBF0FBECDBF3C016B01DE01A2
:10AFE000AE5BBF4F11965C934E9325962FAF25977E
:10AFF0001C861F861FA21AA66115710509F47CC064
:10B00000FC018381882309F077C0FA0180818F32A7
:10B01000F1F08601ECE0EE2EF12CEC0EFD1E72E458
:10B02000A72EB12CAC0EBD1E4E010894811C911CA4
:10B030002796FFAEEEAE279767E2262E312C2C0E18
:10B040003D1E270123C01196B183A08301C0FD01DD
:10B05000A081B1818C918F32B1F3D60113968C917E
:10B06000139782508230A8F28E01095D1F4F5996C6
:10B070006D917C915A97C80194DB882359F63CC0A6
:10B08000342D252D8701832F922F7C01F50180819E
:10B090009181B401A5010E94774F882329F42CC027
:10B0A0003196D501ED93FC93D501ED91FC91808112
:10B0B0008F32B1F38823B9F0C701B801A40121E0B0
:10B0C000AADE8823C9F00C151D0511F0C80174D83B
:10B0D0002796EEADFFAD2797EE16FF0689F6C10164
:10B0E000322D292FCFCFC301B801A40125962FAD52
:10B0F000259791DE182F01C010E0CE01879665D804
:10B10000CE010C9662D8812FCA5BDF4F0FB6F89440
:10B11000DEBF0FBECDBFCF91DF911F910F91FF908A
:10B12000EF90DF90CF90BF90AF909F908F907F90E7
:10B130006F905F904F903F902F9008950F931F93C3
:10B14000DF93CF93CDB7DEB76B970FB6F894DEBF22
:10B150000FBECDBF9C01AB0119821C828E010F5F17
:10B160001F4FC801B90122E01DDF882311F410E050
:10B1700003C0C80116D9182FCE01019626D8812FF9
:10B180006B960FB6F894DEBF0FBECDBFCF91DF91A7
:10B190001F910F910895382F20E09FB7F894809168
:10B1A00005018B7F809305019FBF37FF02C0A39AE3
:10B1B00001C0A3989FB7F8948091050184608093A3
:10B1C00005019FBF2F5F283011F0330FE6CF0895A0
:10B1D0001092BF0C08958091FE0E90E09695879591
:10B1E0009695879581700895FC012081822F90E0CB
:10B1F0006AE070E00E94B8FECB016AE070E00E9455
:10B20000B8FE805D80932D0F822F90E06AE070E0A1
:10B210000E94B8FE805D80932E0F10922F0F8DE25A
:10B220009FE00895FC01608171818281938120E01B
:10B2300030E040E251E40E94B3FD0E9442FB9B01DA
:10B2400077FF02C08DE201C08BE280932D0F37FFA4
:10B2500003C0309521953F4FC90168EE73E00E940D
:10B26000B8FECB016AE070E00E94B8FE805D80937A
:10B270002E0FC90164E670E00E94B8FECB016AE0BF
:10B2800070E00E94B8FE805D80932F0FC9016AE0D4
:10B2900070E00E94B8FECB016AE070E00E94B8FE48
:10B2A000805D8093300F8EE28093310FC9016AE098
:10B2B00070E00E94B8FE805D8093320F1092330FD1
:10B2C0008DE29FE00895FC0160817181828193810C
:10B2D00020E030E040E251E40E94B3FD0E9442FBD6
:10B2E0009B0177FF03C0309521953F4FC90168EE60
:10B2F00073E00E94B8FECB016AE070E00E94B8FEE5
:10B30000805D80932D0FC90164E670E00E94B8FE55
:10B31000CB016AE070E00E94B8FE805D80932E0F42
:10B32000C9016AE070E00E94B8FECB016AE070E0FB
:10B330000E94B8FE805D80932F0F8EE28093300FC5
:10B34000C9016AE070E00E94B8FE805D8093310F11
:10B350001092320F8DE29FE00895EF92FF920F93CB
:10B360001F93FC01608171818281938120E030E034
:10B3700048EC52E40E94B3FD0E9442FB7B018C0129
:10B3800097FD12C020E137E240E050E00E94EDFE60
:10B39000CA01B9012AE030E040E050E00E94EDFE31
:10B3A000605D60932D0F03C08DE280932D0F17FF1A
:10B3B00008C010950095F094E094E11CF11C011D6B
:10B3C000111DC801B70128EE33E040E050E00E94B3
:10B3D000EDFECA01B9012AE030E040E050E00E94F1
:10B3E000EDFE605D60932E0FC801B70124E630E0EA
:10B3F00040E050E00E94EDFECA01B9012AE030E0D1
:10B4000040E050E00E94EDFE605D60932F0F8EE201
:10B410008093300FC801B7012AE030E040E050E0EF
:10B420000E94EDFECA01B9012AE030E040E050E0A0
:10B430000E94EDFE605D6093310FC801B7012AE004
:10B4400030E040E050E00E94EDFE605D6093320F1E
:10B450001092330F8DE29FE01F910F91FF90EF90BC
:10B460000895FC0180819181843691055CF064E649
:10B4700070E00E94B8FECB016AE070E00E94B8FE66
:10B48000805D01C080E280932D0F808191818A30A0
:10B4900091055CF06AE070E00E94B8FECB016AE0C2
:10B4A00070E00E94B8FE805D01C080E280932E0FA4
:10B4B000808191816AE070E00E94B8FE805D809397
:10B4C0002F0F1092300F8DE29FE00895DF93CF93FE
:10B4D0000F920F92CDB7DEB7FC016081718182813E
:10B4E00093810E9442FB7A836983CE010196B9DF82
:10B4F0000F900F90CF91DF910895EF92FF920F93ED
:10B500001F93FC01E080F18002811381C801B70123
:10B5100020E030E040E050E00E94E1FC18161CF40E
:10B52000C801B70103C0C801B70190580E9442FB8F
:10B530007B018C0180E1E81687E2F80680E00807CD
:10B5400080E01807A4F0C801B70120E137E240E02D
:10B5500050E00E94EDFECA01B9012AE030E040E06F
:10B5600050E00E94EDFE605D60932D0F0CC080E204
:10B5700080932D0F98EEE91693E0F90690E0090705
:10B5800090E01907A4F0C801B70128EE33E040E0CD
:10B5900050E00E94EDFECA01B9012AE030E040E02F
:10B5A00050E00E94EDFE605D60932E0F08C0809316
:10B5B0002E0F94E6E916F10401051105A4F0C80167
:10B5C000B70124E630E040E050E00E94EDFECA0101
:10B5D000B9012AE030E040E050E00E94EDFE605DFD
:10B5E00060932F0F08C080932F0F9AE0E916F104A3
:10B5F00001051105A4F0C801B7012AE030E040E0E0
:10B6000050E00E94EDFECA01B9012AE030E040E0BE
:10B6100050E00E94EDFE605D6093300F02C08093A9
:10B62000300FC801B7012AE030E040E050E00E944E
:10B63000EDFE605D6093310F1092320F8DE29FE05E
:10B640001F910F91FF90EF900895EF92FF920F934B
:10B650001F93FC01608171818281938120E030E041
:10B6600040E251E40E94B3FD0E9442FB97FF02C0FA
:10B670002DE201C02BE220932D0F7B018C0197FF5F
:10B6800008C010950095F094E094E11CF11C011D98
:10B69000111DC801B70120E137E240E050E00E94EF
:10B6A000EDFECA01B9012AE030E040E050E00E941E
:10B6B000EDFE605D60932E0FC801B70128EE33E008
:10B6C00040E050E00E94EDFECA01B9012AE030E0FE
:10B6D00040E050E00E94EDFE605D60932F0FC801D6
:10B6E000B70124E630E040E050E00E94EDFECA01E0
:10B6F000B9012AE030E040E050E00E94EDFE605DDC
:10B700006093300FC801B7012AE030E040E050E01C
:10B710000E94EDFECA01B9012AE030E040E050E0AD
:10B720000E94EDFE605D6093310F8EE28093320FD8
:10B73000C801B7012AE030E040E050E00E94EDFE91
:10B74000605D6093330F1092340F8DE29FE01F9184
:10B750000F91FF90EF900895EF92FF920F931F9338
:10B76000FC01608171818281938120E030E048ECAE
:10B7700052E40E94B3FD0E9442FB97FF02C02DE2FB
:10B7800001C02BE220932D0F7B018C0197FF08C095
:10B7900010950095F094E094E11CF11C011D111D21
:10B7A000C801B70120E137E240E050E00E94EDFE21
:10B7B000CA01B9012AE030E040E050E00E94EDFE0D
:10B7C000605D60932E0FC801B70128EE33E040E0C2
:10B7D00050E00E94EDFECA01B9012AE030E040E0ED
:10B7E00050E00E94EDFE605D60932F0FC801B7012D
:10B7F00024E630E040E050E00E94EDFECA01B901CD
:10B800002AE030E040E050E00E94EDFE605D609391
:10B81000300F8EE28093310FC801B7012AE030E08B
:10B8200040E050E00E94EDFECA01B9012AE030E09C
:10B8300040E050E00E94EDFE605D6093320FC80171
:10B84000B7012AE030E040E050E00E94EDFE605D8C
:10B850006093330F1092340F8DE29FE01F910F9190
:10B86000FF90EF9008950F93DF93CF9300D00F9246
:10B87000CDB7DEB7009103010295069507700095DC
:10B8800001708091030186FF02602091000F3091CA
:10B89000010F4091020F5091030F29833A834B838C
:10B8A0005C830E943BF529813A814B815C8126179C
:10B8B00037074807590710F4629B04600093FE0E97
:10B8C0009091FE0E91708091FE0E81FD92608091AC
:10B8D000040F981729F19130B1F0913028F092308F
:10B8E00041F09330E9F40AC0813079F08230C1F43C
:10B8F00012C0882351F0833099F40DC0823029F0B2
:10B90000813071F408C0833021F48091B20C8F5FD4
:10B9100005C0882329F48091B20C81508093B20C29
:10B920009093040F0F900F900F900F90CF91DF9195
:10B930000F910895CF93DF93EC0104C082EC9EE059
:10B940000E942EF6FE01219664916623B9F7DF91DD
:10B95000CF910895EF92FF920F931F93CF93DF93B0
:10B96000F82EEB01142FE22E4E3311F04B3FA9F4C9
:10B9700086EC9EE061E00E94A4F14CE0F49EA00100
:10B9800011244D5F86EC9EE060E020E80CE00E9410
:10B99000A3ED86EC9EE060E003C086EC9EE061E0F3
:10B9A0000E94A4F11092FB0E2F2D30E02F5F3F4F2D
:10B9B000C901880F991F820F931F880F991F880F45
:10B9C000991F8093FC0E1E3321F082EC9EE0612FC4
:10B9D00003C082EC9EE060E20E942EF601E106C008
:10B9E00082EC9EE00E942EF621960150FE016491A9
:10B9F0006623B1F706C082EC9EE060E20E942EF65C
:10BA000001500023C1F782EC9EE06E2D0E942EF6BD
:10BA100082EC9EE060E20E942EF686EC9EE061E001
:10BA20000E94A4F1DF91CF911F910F91FF90EF90B1
:10BA30000895EF92FF920F931F93DF93CF93CDB7AB
:10BA4000DEB72C970FB6F894DEBF0FBECDBF86ECE5
:10BA50009EE061E00E94A4F18091350F80FF11C04B
:10BA60008091841290918512892B59F086EC9EE08A
:10BA700069E041E02FE003E177E2E72E7DE1F72E78
:10BA80000AC086EC9EE069E041E02FE003E154E467
:10BA9000E52E5EE1F52E0E9413EE86EC9EE06AE252
:10BAA0004AE228E007E00E94A3ED86EC9EE062E314
:10BAB0004CE222E005E00E94A3ED86EC9EE06AE203
:10BAC00041E32AE004E00E94BEED86EC9EE062E3E2
:10BAD0004BE20E948DF186EC9EE066E341E329E4AF
:10BAE0000E94BEED86EC9EE062EF79E00E948BEF53
:10BAF0008091C10F8823B9F180919011882311F1B1
:10BB000060913A1270913B1280913C1290913D12DB
:10BB10006115710581059105A9F06D597F4F8F4F12
:10BB20009F4F24E630E040E050E00E94CBFE609161
:10BB300042127091431280914412909145120E94DA
:10BB4000CBFE01C020E087E4289FC001112464E6F9
:10BB500070E00E94B8FE262F86EC9EE067E342E389
:10BB600002E00E94A3ED80E58093FB0E8FE28093BC
:10BB7000FC0E8091881290918912A0918A12B09146
:10BB80008B120097A105B105E1F10E943BF520E67B
:10BB90003AEE40E050E00E94CBFE79018A016091CC
:10BBA00088127091891280918A1290918B1220E6EE
:10BBB0003AEE40E050E00E94CBFEE21AF30AC701E1
:10BBC0006CE370E00E94A4FE6983CE0101960CDB59
:10BBD000BC0182EC9EE00E9452F682EC9EE06AE399
:10BBE0000E942EF6C7016CE370E00E94A4FE8A83D7
:10BBF000CE010296F9DABC0182EC9EE00E9452F678
:10BC000003C08FE69FE196DE86EC9EE062EF79E06E
:10BC10000E948BEF16E01093FB0E1093FC0E6091C8
:10BC2000651470916614882777FD8095982F0E947F
:10BC300075FB20E030E040E05FE30E94FAF90E94EB
:10BC400042FB7C836B83CE0103960BDCBC0182EC50
:10BC50009EE00E9452F68CE69FE16CDE1093FB0E94
:10BC60008BE18093FC0E60916B1470916C14809149
:10BC70006D1490916E1420E030E040E05FE30E948C
:10BC8000FAF90E9442FB7E836D83CE010596E9DBC3
:10BC9000BC0182EC9EE00E9452F689E69FE14ADEFA
:10BCA0006091651470916614882777FD8095982FB0
:10BCB0000E9475FB20916B1430916C1440916D14AF
:10BCC00050916E140E94E1FC18164CF086EC9EE038
:10BCD0006DE041E122E002E00E94A3ED12C086EC9B
:10BCE0009EE060E00E94A4F186EC9EE06DE041E100
:10BCF00022E002E00E94A3ED86EC9EE061E00E945B
:10BD0000A4F186EC9EE062EF79E00E948BEF8FE178
:10BD10008093FB0E1BE11093FC0E82EC9EE065E12C
:10BD200072E00E9452F686EC9EE062EF79E00E949B
:10BD30008BEF87E38093FB0E1093FC0E82EC9EE06A
:10BD400065E172E00E9452F686EC9EE062EF79E0D7
:10BD50000E948BEF01E50093FB0E86E08093FC0EC2
:10BD60006091671470916814882777FD8095982FEB
:10BD70000E9475FB20E030E040E05FE30E94FAF9AA
:10BD80000E9442FB78876F83CE0107966ADBBC0175
:10BD900082EC9EE00E9452F686E69FE1CBDD0093A6
:10BDA000FB0E1093FC0E60917114709172148091CF
:10BDB00073149091741420E030E040E05FE30E943F
:10BDC000FAF90E9442FB7A876987CE01099649DB1E
:10BDD000BC0182EC9EE00E9452F683E69FE1AADD60
:10BDE0006091671470916814882777FD8095982F6B
:10BDF0000E9475FB2091711430917214409173145C
:10BE0000509174140E94E1FC18164CF086EC9EE0F0
:10BE100068E542E122E002E00E94A3ED12C086EC58
:10BE20009EE060E00E94A4F186EC9EE068E542E1BD
:10BE300022E002E00E94A3ED86EC9EE061E00E9419
:10BE4000A4F186EC9EE062EF79E00E948BEF88E639
:10BE50008093FB0E8BE18093FC0E20918412309135
:10BE6000851284E690E0AC01249FC001259F900DCF
:10BE7000349F900D112460E071E00E94B8FE6F5F66
:10BE80007F4F7C876B87CE010B96EBDABC0182EC8F
:10BE90009EE00E9452F682EC9EE069E172E00E9410
:10BEA00052F686EC9EE062EF79E00E948BEF86EC22
:10BEB0009EE060E04DE120E80AE00E94A3ED86EC00
:10BEC0009EE060E00E94A4F182E08093FB0E15E208
:10BED0001093FC0E82EC9EE06BE172E00E9452F641
:10BEE00086EC9EE068E041E20E948DF186EC9EE0E7
:10BEF00068E043E20E948DF18AE08093FB0E10938C
:10BF0000FC0E83E592E1DFD9BC0182EC9EE00E9449
:10BF100052F68BE28093FB0E1093FC0E81E69FE1BC
:10BF200009DD86EC9EE061E341E20E948DF186EC42
:10BF30009EE061E343E20E948DF183E38093FB0E78
:10BF40001093FC0E87E592E1BED9BC0182EC9EE025
:10BF50000E9452F683E58093FB0E1093FC0E82EC58
:10BF60009EE06DE172E00E9452F686EC9EE069E58B
:10BF700041E20E948DF186EC9EE069E543E20E9479
:10BF80008DF18BE58093FB0E1093FC0E8BE592E117
:10BF900049D9BC0182EC9EE00E9452F686EC9EE0FC
:10BFA00061E00E94A4F186EC9EE06EEE72E10E94D8
:10BFB0008BEF83E08093FB0E81E38093FC0E82EC99
:10BFC0009EE06DEF0E942EF686EC9EE062EF79E037
:10BFD0000E948BEF8CE08093FB0E80E38093FC0E3D
:10BFE00086ED93E03EDABC0182EC9EE00E9452F6C0
:10BFF00082EC9EE065E20E942EF686EC9EE062EF07
:10C0000079E00E948BEF1092FB0E8DE38093FC0E83
:10C0100082EC9EE060EA73E00E9452F62C960FB626
:10C02000F894DEBF0FBECDBFCF91DF911F910F916E
:10C03000FF90EF90089582E08093C5030E943BF546
:10C040006C507E4F8F4F9F4F6093000F7093010F86
:10C050008093020F9093030F6E9A8FE467E174E070
:10C0600020E030E040E050E00E94FBF66AE070E043
:10C0700080E090E00E9449F58FE40C9487F680916F
:10C080000E0F882321F0815080930E0F03C081E0B2
:10C090008093C5038091C503882321F0CADC8AE020
:10C0A00080930E0F8091FE0E82FF0FC081EE97E607
:10C0B0009093C4038093C3031092050F1092060F50
:10C0C0001092070F1092080FB6DF2091D60330911F
:10C0D000D7032436310554F48091050F9091060F53
:10C0E000280F391F253631056CF41AC02536310565
:10C0F000BCF08091050F9091060F280F391F243650
:10C10000310574F41092050F1092060F1092070F6C
:10C110001092080F84E690E09093D7038093D603A3
:10C120002091D6033091D7032436310589F48091CC
:10C13000050F9091060F8B3091051CF0865A9F4F8A
:10C140000DC02FEF863F9207ACF482599F4F06C077
:10C150008091050F9091060F820F931F9093D70344
:10C160008093D6031092050F1092060F1092070FBE
:10C170001092080F8091D6039091D7030A9734F458
:10C180008AE090E09093D7038093D6038091D60302
:10C190009091D703885E934034F087EE93E09093BC
:10C1A000D7038093D6030895AF92BF92CF92DF92C8
:10C1B000EF92FF920F931F938091050F9091060FBE
:10C1C000A091070FB091080F81509048A040B04057
:10C1D00040F01092050F1092060F1092070F109268
:10C1E000080F6091050F7091060F8091070F9091D5
:10C1F000080F25E030E040E050E00E94CBFE7901DE
:10C200008A018091FF0E90E0A0E0B0E0E816F90608
:10C210000A071B0710F42093FF0E0091FF0E809178
:10C22000FE0E90E09695879596958795FF24F3945A
:10C23000F82210E0E3E1AE2EB12CC12CD12CEE247B
:10C24000E394002379F58091C5038823B9F08091A8
:10C25000050F9091060FA091070FB091080F059759
:10C26000A105B10528F4812F60E673E24BEF04C00D
:10C27000812F60E673E240E22BEF6CDBFF2009F4D4
:10C28000DBC08091050F9091060FA091070FB09130
:10C29000080F0597A105B10508F0CEC0CCDE85E3F7
:10C2A00098E9BDC0013009F03DC08091C5038823E5
:10C2B000F1F06091050F7091060F8091070F90913A
:10C2C000080F25E030E040E050E00E94CBFE213036
:10C2D00031054105510529F4812F66E573E24EE3EE
:10C2E00004C0812F66E573E240E22AEF33DBFF20D2
:10C2F00009F4A2C06091050F7091060F8091070F9D
:10C300009091080F25E030E040E050E00E94CBFE25
:10C31000213031054105510509F08EC08CDE81E6E2
:10C3200094E67DC0023009F03DC08091C5038823AA
:10C33000F1F06091050F7091060F8091070F9091B9
:10C34000080F25E030E040E050E00E94CBFE2230B4
:10C3500031054105510529F4812F6DE473E24EE367
:10C3600004C0812F6DE473E240E22AEFF3DAFF208C
:10C3700009F462C06091050F7091060F8091070F5C
:10C380009091080F25E030E040E050E00E94CBFEA5
:10C39000223031054105510509F04EC04CDE84E5DF
:10C3A00094E63DC0033009F047C08091C50388235F
:10C3B000F1F06091050F7091060F8091070F909139
:10C3C000080F25E030E040E050E00E94CBFE233033
:10C3D00031054105510529F4812F62E473E24EE3F2
:10C3E00004C0812F62E473E240E22AEFB3DAFF2057
:10C3F00019F16091050F7091060F8091070F9091D0
:10C40000080F25E030E040E050E00E94CBFE2330F2
:10C4100031054105510581F40EDE87E494E69093E1
:10C42000C4038093C3031092050F1092060F10925D
:10C43000070F1092080F38C08091050F9091060FDA
:10C44000A091070FB091080F4497A105B10540F0E6
:10C45000A092050FB092060FC092070FD092080F5E
:10C460006091050F7091060F8091070F9091080F52
:10C4700025E030E040E050E00E94CBFE422F80916A
:10C48000FF0E90E0049630E08217930744F4445086
:10C490004093FF0EE092C503042F01501FEF1F5F72
:10C4A000153010F40F5FCDCE1F910F91FF90EF90DC
:10C4B000DF90CF90BF90AF900895CF92DF92EF9230
:10C4C000FF920F931F938091050F9091060FA091FB
:10C4D000070FB091080F81509048A040B04040F045
:10C4E0001092050F1092060F1092070F1092080F6E
:10C4F0006091050F7091060F8091070F9091080FC2
:10C5000025E030E040E050E00E94CBFE79018A0156
:10C510008091FF0E90E0A0E0B0E0E816F9060A076F
:10C520001B0710F42093FF0EF090FF0E8091FE0E7B
:10C5300090E09695879596958795EE24E394E8226A
:10C5400000E0A5E0DA2ECC24C394FF2079F5809199
:10C55000C5038823B9F08091050F9091060FA09133
:10C56000070FB091080F0597A105B10528F4802F9A
:10C5700066E873E24BEF04C0802F66E873E240E2A6
:10C580002BEFE8D9EE2009F490C08091050F90912F
:10C59000060FA091070FB091080F0597A105B105EF
:10C5A00008F083C048DD84ED90E60FC181E0F81605
:10C5B00009F03DC08091C5038823F1F06091050F1B
:10C5C0007091060F8091070F9091080F25E030E0E1
:10C5D00040E050E00E94CBFE21303105410551057D
:10C5E00029F4802F6FE773E24EE304C0802F6FE7DA
:10C5F00073E240E22AEFAED9EE2009F456C0609112
:10C60000050F7091060F8091070F9091080F25E09C
:10C6100030E040E050E00E94CBFE21303105410582
:10C62000510509F042C007DD8BE793E9CEC022E057
:10C63000F216D9F58091C5038823F1F06091050FBA
:10C640007091060F8091070F9091080F25E030E060
:10C6500040E050E00E94CBFE2230310541055105FB
:10C6600029F4802F68E773E24EE304C0802F68E767
:10C6700073E240E22AEF6ED9EE20B9F06091050F27
:10C680007091060F8091070F9091080F25E030E020
:10C6900040E050E00E94CBFE2230310541055105BB
:10C6A00021F4C9DC89EC92E990C06091290F709166
:10C6B0002A0F80912B0F90912C0F20E030E040E268
:10C6C00051E40E94D3FA88230CF08CC083E0F81662
:10C6D00009F03DC08091C5038823F1F06091050FFA
:10C6E0007091060F8091070F9091080F25E030E0C0
:10C6F00040E050E00E94CBFE23303105410551055A
:10C7000029F4802F61E773E24EE304C0802F61E7D4
:10C7100073E240E22AEF1ED9EE2009F465C0609171
:10C72000050F7091060F8091070F9091080F25E07B
:10C7300030E040E050E00E94CBFE2330310541055F
:10C74000510509F051C077DC87E192E93EC024E051
:10C75000F21609F049C08091C5038823F1F0609179
:10C76000050F7091060F8091070F9091080F25E03B
:10C7700030E040E050E00E94CBFE2430310541051E
:10C78000510529F4802F68E673E24EE304C0802F40
:10C7900068E673E240E22AEFDDD8EE2029F16091ED
:10C7A000050F7091060F8091070F9091080F25E0FB
:10C7B00030E040E050E00E94CBFE243031054105DE
:10C7C000510591F438DC83E991E99093C403809397
:10C7D000C3031092050F1092060F1092070F1092CC
:10C7E000080F4EC013E001C015E06091050F709175
:10C7F000060F8091070F9091080F25E030E040E090
:10C8000050E00E94CBFE812F90E0A0E0B0E028171E
:10C8100039074A075B0780F01D9DC001112401976D
:10C82000AA2797FDA095BA2F8093050F9093060F26
:10C83000A093070FB093080F6091050F7091060F3A
:10C840008091070F9091080F25E030E040E050E024
:10C850000E94CBFE422F8091FF0E90E0049630E0C4
:10C860008217930744F444504093FF0EC092C503CF
:10C87000F42EFA940FEF0F5F053010F4F39465CEA9
:10C880001F910F91FF90EF90DF90CF9008958DEC66
:10C890009CECACECBDE38093290F90932A0FA093FE
:10C8A0002B0FB0932C0F09CE80E090E0A0E8BFE3FF
:10C8B0008093290F90932A0FA0932B0FB0932C0FE6
:10C8C000FCCD80E090E0A0E2B1E48093290F90934A
:10C8D0002A0FA0932B0FB0932C0FEFCD0F931F9324
:10C8E000DF93CF93CDB7DEB76E970FB6F894DEBF68
:10C8F0000FBECDBF00D000D0EDB7FEB731969E0180
:10C900002F5F3F4FADB7BEB712963C932E93119752
:10C910002DED3FE133832283958384830E94752725
:10C920008E010B5F1F4FEDB7FEB736960FB6F8942A
:10C93000FEBF0FBEEDBF08C0992787FD90950E94EE
:10C9400016FFD8018D938D01F80180818823A1F70E
:10C95000CE0101960E9467CD89ED9FE10E94EECC49
:10C960001092050F1092060F1092070F1092080FE9
:10C970008FE390E69093C4038093C3036E960FB643
:10C98000F894DEBF0FBECDBFCF91DF911F910F9105
:10C9900008958FEB9FE00E94F0CD1092FF0E089556
:10C9A0003F924F925F926F927F928F929F92AF923F
:10C9B000BF92CF92DF92EF92FF920F931F93CF938C
:10C9C000DF938091C503882309F097C28091FE0E02
:10C9D00082FD93C2A6C21092050F1092060F10920C
:10C9E000070F1092080F6091050F7091060F80914C
:10C9F000070F9091080F25E030E040E050E00E94E2
:10CA0000CBFE79018A018091FF0E90E0A0E0B0E0BA
:10CA1000E816F9060A071B0710F42093FF0EA090F2
:10CA2000FF0E8091FE0E90E09695879596958795DE
:10CA3000992493949822EE2433243394562C5A94B8
:10CA400075E0472EAA2091F58091C5038823C1F097
:10CA50008091050F9091060FA091070FB091080FDC
:10CA60000597A105B10528F48E2D64ED7FE14BEF0C
:10CA700004C08E2D64ED7FE140E22BEF0E94AA5CA2
:10CA80009920A1F08091050F9091060FA091070FBA
:10CA9000B091080F0597A105B10540F4CCDA81EEFD
:10CAA00097E69093C4038093C30326C183E190E18A
:10CAB00063EC7FE00E94EC508091C30F8F3219F439
:10CAC000FF24F3942AC021E0A21629F58091C50322
:10CAD0008823F9F06091050F7091060F8091070F80
:10CAE0009091080F25E030E040E050E00E94CBFE3E
:10CAF000213031054105510529F48E2D60ED7FE18E
:10CB00004EE304C08E2D60ED7FE140E220E20E9402
:10CB1000AA5C9920E1F462E0F62E8E2D90E09C0153
:10CB2000220F331F280F391F220F331F220F331FED
:10CB300003E0802E820E01969C01220F331F280FE6
:10CB4000391FB22EBB0CBB0CCC24DD2485C16091F7
:10CB5000050F7091060F8091070F9091080F25E047
:10CB600030E040E050E00E94CBFE2130310541052D
:10CB7000510589F660DA0DDFD4C1FA1409F068C1F5
:10CB8000652D6C198FEB9FE00E9411DA8091EB0FFD
:10CB90009091C503882309F4B8C0992309F48AC089
:10CBA0006091050F7091060F8091070F9091080F0B
:10CBB00025E030E040E050E00E94CBFE8F2D90E079
:10CBC000A0E0B0E0281739074A075B0709F045C025
:10CBD0008091D00F882319F4C3ECDFE004C01092D9
:10CBE000E20FC0EDDFE086EC9EE061E00E94A4F180
:10CBF00086EC9EE060E0482D20E80CE00E94A3ED6A
:10CC000086EC9EE060E00E94A4F11092FB0EB092D0
:10CC1000FC0E82EC9EE060E20E942EF682EC9EE02A
:10CC200069EF0E942EF612E106C082EC9EE00E949F
:10CC30002EF62196115068816623B9F706C082EC62
:10CC40009EE060E20E942EF611501123C1F786EC9F
:10CC50009EE061E00E94A4F12DC08091D00F882356
:10CC600019F4C3ECDFE004C01092E20FC0EDDFE086
:10CC70001092FB0EB092FC0E82EC9EE060E20E94ED
:10CC80002EF682EC9EE069EF0E942EF612E106C0BD
:10CC900082EC9EE00E942EF6219611506881662358
:10CCA000B9F706C082EC9EE060E20E942EF61150B9
:10CCB0001123C1F7992009F4CBC06091050F709141
:10CCC000060F8091070F9091080F25E030E040E0BB
:10CCD00050E00E94CBFE8F2D90E0A0E0B0E028173E
:10CCE00039074A075B0709F0B3C0A5D98FEB9FE06E
:10CCF00063EC7FE00E9443CE1092050F1092060F66
:10CD00001092070F1092080F0CC1992309F480C0EC
:10CD10006091050F7091060F8091070F9091080F99
:10CD200025E030E040E050E00E94CBFE8F2D90E007
:10CD3000A0E0B0E0281739074A075B0709F040C0B8
:10CD40008091D00F882319F4C3ECDFE004C0109267
:10CD5000E30FC0EDDFE086EC9EE061E00E94A4F10D
:10CD600086EC9EE060E0482D20E80CE00E94A3EDF8
:10CD700086EC9EE060E00E94A4F11092FB0EB0925F
:10CD8000FC0E82EC9EE060E20E942EF613E106C0EB
:10CD900082EC9EE00E942EF6219611506881662357
:10CDA000B9F706C082EC9EE060E20E942EF61150B8
:10CDB0001123C1F786EC9EE061E00E94A4F128C037
:10CDC0008091D00F882319F4C3ECDFE004C01092E7
:10CDD000E30FC0EDDFE01092FB0EB092FC0E82EC90
:10CDE0009EE060E20E942EF613E106C082EC9EE017
:10CDF0000E942EF62196115068816623B9F706C06D
:10CE000082EC9EE060E20E942EF611501123C1F7E1
:10CE10009920F1F06091050F7091060F8091070F36
:10CE20009091080F25E030E040E050E00E94CBFEFA
:10CE30008F2D90E0A0E0B0E0281739074A075B0784
:10CE400039F4F9D883EC9FE060ED7FE047DD69C0FD
:10CE5000F3940894C11CD11CC614D70408F48DCED9
:10CE60006091050F7091060F8091070F9091080F48
:10CE700025E030E040E050E00E94CBFE8F2D90E0B6
:10CE8000A0E0B0E0281739074A075B0780F0F49C60
:10CE9000C00111240197AA2797FDA095BA2F80936E
:10CEA000050F9093060FA093070FB093080F6091A2
:10CEB000050F7091060F8091070F9091080F25E0E4
:10CEC00030E040E050E00E94CBFE422F8091FF0E08
:10CED00090E0049630E0821793074CF4445040935E
:10CEE000FF0E3092C503A42EAA94EE24EA94E39494
:10CEF00084E08E15B0F0A394A5CD8FEB9FE00E9447
:10CF0000B1D93C018091050F9091060FA091070FB8
:10CF1000B091080F81509048A040B04008F05BCD20
:10CF200062CDDF91CF911F910F91FF90EF90DF9035
:10CF3000CF90BF90AF909F908F907F906F905F90B9
:10CF40004F903F900895CF93DF931092C10F8FEBD6
:10CF50009FE060E00E9417CF0E94752A84EE9FE157
:10CF60000E94EECC80918507882301F110928507FD
:10CF700080918212C82FD0E0CC0FDD1FCB59DB4E41
:10CF800068817981882777FD8095982F0E9475FBAD
:10CF9000209194033091950340919603509197030B
:10CFA0000E94E1FC181614F419821882DF91CF91C7
:10CFB00008958FEB9FE00C94E4CD8FEB9FE00C94F1
:10CFC000EBCDCF92DF92EF92FF920F931F93809160
:10CFD000050F9091060FA091070FB091080F815097
:10CFE0009048A040B04040F01092050F1092060FFC
:10CFF0001092070F1092080F6091050F7091060FA5
:10D000008091070F9091080F25E030E040E050E05C
:10D010000E94CBFE79018A018091FF0E90E0A0E092
:10D02000B0E0E816F9060A071B0710F42093FF0E7C
:10D03000F090FF0E8091FE0E90E096958795969564
:10D040008795EE24E394E82200E0A5E0CA2EDD24D3
:10D05000D394FF2079F58091C5038823C1F0809196
:10D06000050F9091060FA091070FB091080F05973B
:10D07000A105B10528F4802F64EC7FE14BEF04C0DB
:10D08000802F64EC7FE140E22BEF0E94AA5CEE204F
:10D0900089F08091050F9091060FA091070FB09134
:10D0A000080F0597A105B10528F40E941B608FE3C6
:10D0B00090E604C20E94AB39882329F48091C10F05
:10D0C000882309F456C281E0F81609F07EC08091E9
:10D0D000C5038823F9F06091050F7091060F8091C8
:10D0E000070F9091080F25E030E040E050E00E94EB
:10D0F000CBFE213031054105510529F4802F6FEB1E
:10D100007FE14EE304C0802F6FEB7FE140E22AEF26
:10D110000E94AA5CEE2009F498C06091050F7091FE
:10D12000060F8091070F9091080F25E030E040E056
:10D1300050E00E94CBFE213031054105510509F038
:10D1400084C00E941B6081ED9FE7B8C18091C50338
:10D150008823F9F06091050F7091060F8091070FF9
:10D160009091080F25E030E040E050E00E94CBFEB7
:10D17000213031054105510529F4802F67EB7FE10E
:10D180004EE304C0802F67EB7FE140E22AEF0E946C
:10D19000AA5CEE2009F459C06091050F7091060F4A
:10D1A0008091070F9091080F25E030E040E050E0BB
:10D1B0000E94CBFE213031054105510509F045C0E3
:10D1C0000E941B6085E398E979C122E0F216E9F537
:10D1D0008091C5038823F9F06091050F7091060FC7
:10D1E0008091070F9091080F25E030E040E050E07B
:10D1F0000E94CBFE223031054105510529F4802FD4
:10D200006FEA7FE14EE304C0802F6FEA7FE140E2E6
:10D210002AEF0E94AA5CEE20C1F06091050F709188
:10D22000060F8091070F9091080F25E030E040E055
:10D2300050E00E94CBFE223031054105510529F412
:10D240000E941B6085EC9AE639C18091C20F882349
:10D2500009F4F4C080919011882309F4CBC0809127
:10D26000C10F882309F442C083E0F81609F080C09A
:10D270008091C5038823F9F06091050F7091060F26
:10D280008091070F9091080F25E030E040E050E0DA
:10D290000E94CBFE233031054105510529F4802F32
:10D2A00063EA7FE14EE304C0802F63EA7FE140E25E
:10D2B00020E20E94AA5CEE2009F40FC16091050FE4
:10D2C0007091060F8091070F9091080F25E030E0D4
:10D2D00040E050E00E94CBFE23303105410551056E
:10D2E00009F0FBC00E941B6068DE48C123E0F21613
:10D2F00009F03EC08091C5038823F9F06091050FC5
:10D300007091060F8091070F9091080F25E030E093
:10D3100040E050E00E94CBFE23303105410551052D
:10D3200029F4802F66E97FE14EE304C0802F66E98F
:10D330007FE140E220E20E94AA5CEE2009F4CDC029
:10D340006091050F7091060F8091070F9091080F63
:10D3500025E030E040E050E00E94CBFE2330310574
:10D360004105510509F0B9C00E941B6022DE06C1CB
:10D3700084E0F81609F0B1C08091C5038823F9F064
:10D380006091050F7091060F8091070F9091080F23
:10D3900025E030E040E050E00E94CBFE2430310533
:10D3A0004105510529F4802F6BE87FE14EE304C06D
:10D3B000802F6BE87FE140E220E20E94AA5CEE2031
:10D3C00009F48BC06091050F7091060F8091070FD3
:10D3D0009091080F25E030E040E050E00E94CBFE45
:10D3E000243031054105510509F077C00E941B60CA
:10D3F000AADDC4C023E0F21609F06DC08091C50318
:10D40000882309F442C06091050F7091060F809146
:10D41000070F9091080F25E030E040E050E00E94B7
:10D42000CBFE233031054105510521F4802F6DE7F6
:10D430007FE122C0802F6DE77FE123C083E0F816F3
:10D4400009F049C08091C5038823F9F06091050F68
:10D450007091060F8091070F9091080F25E030E042
:10D4600040E050E00E94CBFE2330310541055105DC
:10D4700029F4802F65E77FE14EE304C0802F65E744
:10D480007FE140E22AEF0E94AA5CEE2021F1609148
:10D49000050F7091060F8091070F9091080F25E0FE
:10D4A00030E040E050E00E94CBFE233031054105E2
:10D4B000510589F40E941B6080ED94E69093C403AB
:10D4C0008093C3031092050F1092060F1092070F5E
:10D4D0001092080F53C014E001C015E06091050FD1
:10D4E0007091060F8091070F9091080F25E030E0B2
:10D4F00040E050E00E94CBFE812F90E0A0E0B0E041
:10D50000281739074A075B0780F01C9DC0011124CA
:10D510000197AA2797FDA095BA2F8093050F9093A6
:10D52000060FA093070FB093080F6091050F70913D
:10D53000060F8091070F9091080F25E030E040E042
:10D5400050E00E94CBFE422F8091FF0E90E00496A7
:10D5500030E08217930744F444504093FF0ED0927A
:10D56000C503F42EFA940FEF0F5F053038F4F394EF
:10D5700070CD21E0F21609F028CEE8CD1F910F9171
:10D58000FF90EF90DF90CF900895AF92BF92CF922F
:10D59000DF92EF92FF920F931F938091050F90916E
:10D5A000060FA091070FB091080F81509048A0403E
:10D5B000B04040F01092050F1092060F1092070F26
:10D5C0001092080F6091050F7091060F8091070F60
:10D5D0009091080F25E030E040E050E00E94CBFE43
:10D5E00079018A018091FF0E90E0A0E0B0E0E8169A
:10D5F000F9060A071B0710F42093FF0E0091FF0E97
:10D600008091FE0E90E09695879596958795FF24DC
:10D61000F394F82210E08DE1A82EB12CC12CD12C6E
:10D62000EE24E394002389F58091C5038823C1F09B
:10D630008091050F9091060FA091070FB091080FF0
:10D640000597A105B10528F4812F6DE270E24BEF3B
:10D6500004C0812F6DE270E240E22BEF0E94AA5CD1
:10D66000FF2009F465C18091050F9091060FA091EC
:10D67000070FB091080F0597A105B10508F058C133
:10D680000E941B6081EE97E641C0013009F04BC05B
:10D690008091C5038823F9F06091050F7091060F02
:10D6A0008091070F9091080F25E030E040E050E0B6
:10D6B0000E94CBFE213031054105510529F4812F0F
:10D6C00061E270E24EE304C0812F61E270E240E269
:10D6D0002AEF0E94AA5CFF2009F42AC16091050F7D
:10D6E0007091060F8091070F9091080F25E030E0B0
:10D6F00040E050E00E94CBFE21303105410551054C
:10D7000009F016C10E941B6083EA99E89093C40354
:10D710008093C3031092050F1092060F1092070F0B
:10D720001092080F3DC1023009F03FC08091C5033F
:10D730008823F9F06091050F7091060F8091070F13
:10D740009091080F25E030E040E050E00E94CBFED1
:10D75000223031054105510529F4812F6AE170E23B
:10D760004EE304C0812F6AE170E240E22AEF0E949A
:10D77000AA5CFF2009F4DCC06091050F7091060FD0
:10D780008091070F9091080F25E030E040E050E0D5
:10D790000E94CBFE223031054105510509F0C8C079
:10D7A0000E941B6083E29DE6B1CF033009F03FC0C9
:10D7B0008091C5038823F9F06091050F7091060FE1
:10D7C0008091070F9091080F25E030E040E050E095
:10D7D0000E94CBFE233031054105510529F4812FEC
:10D7E0006DE070E24EE304C0812F6DE070E240E234
:10D7F00020E20E94AA5CFF2009F49AC06091050F04
:10D800007091060F8091070F9091080F25E030E08E
:10D8100040E050E00E94CBFE233031054105510528
:10D8200009F086C00E941B600E94F19CB9C00430C0
:10D8300009F03FC08091C5038823F9F06091050F7E
:10D840007091060F8091070F9091080F25E030E04E
:10D8500040E050E00E94CBFE2430310541055105E7
:10D8600029F4812F61E070E24EE304C0812F61E072
:10D8700070E240E220E20E94AA5CFF2009F458C056
:10D880006091050F7091060F8091070F9091080F1E
:10D8900025E030E040E050E00E94CBFE243031052E
:10D8A0004105510509F044C00E941B600E940BA174
:10D8B00077C00530E9F58091C5038823F9F06091C0
:10D8C000050F7091060F8091070F9091080F25E0CA
:10D8D00030E040E050E00E94CBFE253031054105AC
:10D8E000510529F4812F60EF7FE14EE304C0812FC1
:10D8F00060EF7FE140E220E20E94AA5CFF20C1F0DD
:10D900006091050F7091060F8091070F9091080F9D
:10D9100025E030E040E050E00E94CBFE25303105AC
:10D920004105510529F40E941B600E944C9F38C09C
:10D930008091050F9091060FA091070FB091080FED
:10D940004E97A105B10540F0A092050FB092060FC9
:10D95000C092070FD092080F6091050F7091060FCB
:10D960008091070F9091080F25E030E040E050E0F3
:10D970000E94CBFE422F8091FF0E90E0049630E093
:10D980008217930744F444504093FF0EE092C5037E
:10D99000042F01501FEF1F5F153010F40F5F42CEB0
:10D9A0001F910F91FF90EF90DF90CF90BF90AF90BD
:10D9B0000895FF920F931F93CF93DF93EB01022FF4
:10D9C000F32EE22FF32FDF010D900020E9F7122F45
:10D9D0001A1B1C5E1092FB0E90E001969C01220F18
:10D9E000331F280F391F220F331F220F331F20939D
:10D9F000FC0E82EC9EE0642F0E942EF606C082ECA4
:10DA00009EE00E942EF621961150FE01649166233D
:10DA1000B1F782EC9EE06AE30E942EF606C082EC2B
:10DA20009EE060E20E942EF611501123C1F782ECB5
:10DA30009EE0602F7F2D0E9452F6DF91CF911F91C3
:10DA40000F91FF9008952F923F924F925F926F92A5
:10DA50007F928F929F92AF92BF92CF92DF92EF927E
:10DA6000FF920F931F93DF93CF93CDB7DEB7A097AD
:10DA70000FB6F894DEBF0FBECDBF8091050F909119
:10DA8000060FA091070FB091080F81509048A04059
:10DA9000B04040F01092050F1092060F1092070F41
:10DAA0001092080F6091050F7091060F8091070F7B
:10DAB0009091080F25E030E040E050E00E94CBFE5E
:10DAC00079018A018091FF0E90E0A0E0B0E0E816B5
:10DAD000F9060A071B0710F42093FF0E0091FF0EB2
:10DAE0008091FE0E90E09695879596958795FF24F8
:10DAF000F394F82210E08DE1C82ED12CCC0EDD1E5F
:10DB0000B9E1AB2EB12CAC0EBD1EA5E18A2E912C35
:10DB10008C0E9D1EF1E16F2E712C6C0E7D1EEDE0C2
:10DB20004E2E512C4C0E5D1E79E0272E312C2C0EE2
:10DB30003D1E002309F040C08091C5038823C1F039
:10DB40008091050F9091060FA091070FB091080FDB
:10DB50000597A105B10528F4812F68E871E24BEF24
:10DB600004C0812F68E871E240E22BEF0E94AA5CBA
:10DB7000FF2011F40C94237A8091050F9091060FE9
:10DB8000A091070FB091080F0597A105B10510F0FE
:10DB90000C94237A0E941B6085EC9AE69093C40350
:10DBA0008093C3031092050F1092060F1092070F77
:10DBB0001092080F0C94627A013009F08DC08091A8
:10DBC000C503882339F16091050F7091060F80918C
:10DBD000070F9091080F25E030E040E050E00E94F0
:10DBE000CBFE213031054105510551F48EE792E11C
:10DBF0000E94AD599C01812F6FE771E24EE309C08D
:10DC00008EE792E10E94AD599C01812F6FE771E28E
:10DC100040E2CFDEFF2011F40C94237A6091050FCF
:10DC20007091060F8091070F9091080F25E030E06A
:10DC300040E050E00E94CBFE213031054105510506
:10DC400011F00C94237A0E941B608091C303909181
:10DC5000C4039093100F80930F0F8091050F909144
:10DC6000060F9093120F8093110F82E08093C503EB
:10DC700089E997E89093C4038093C30386E791E210
:10DC80009093140F8093130F8EE792E19093160FE9
:10DC90008093150F82E390E0A0E0B0E08093170F2F
:10DCA0009093180FA093190FB0931A0F88E893E17F
:10DCB000A0E0B0E080931B0F90931C0FA0931D0F6A
:10DCC000B0931E0F60917E1270917F12809180122E
:10DCD000909181120C946478023009F08DC080918B
:10DCE000C503882339F16091050F7091060F80916B
:10DCF000070F9091080F25E030E040E050E00E94CF
:10DD0000CBFE223031054105510551F48DE497E0F9
:10DD10000E947D5A9C01812F60E771E24EE309C0A9
:10DD20008DE497E00E947D5A9C01812F60E771E2AB
:10DD300040E23FDEFF2011F40C94237A6091050F3E
:10DD40007091060F8091070F9091080F25E030E049
:10DD500040E050E00E94CBFE2230310541055105E4
:10DD600011F00C94237A0E941B608091C303909160
:10DD7000C4039093100F80930F0F8091050F909123
:10DD8000060F9093120F8093110F82E08093C503CA
:10DD900086EF96E89093C4038093C3038AE691E2EA
:10DDA0009093140F8093130F8DE497E09093160FC8
:10DDB0008093150F85E090E0A0E0B0E08093170F0E
:10DDC0009093180FA093190FB0931A0F8EED93E054
:10DDD000A0E0B0E080931B0F90931C0FA0931D0F49
:10DDE000B0931E0F60914D0770914E0780914F07C1
:10DDF000909150070C944477033009F08DC08091C6
:10DE0000C503882339F16091050F7091060F809149
:10DE1000070F9091080F25E030E040E050E00E94AD
:10DE2000CBFE233031054105510551F485E597E0DE
:10DE30000E94665A9C01812F61E671E24EE309C09F
:10DE400085E597E00E94665A9C01812F61E671E2A8
:10DE500040E2AFDDFF2011F40C94237A6091050FAE
:10DE60007091060F8091070F9091080F25E030E028
:10DE700040E050E00E94CBFE2330310541055105C2
:10DE800011F00C94237A0E941B608091C30390913F
:10DE9000C4039093100F80930F0F8091050F909102
:10DEA000060F9093120F8093110F82E08093C503A9
:10DEB0008CE398E89093C4038093C30388E591E2D0
:10DEC0009093140F8093130F85E597E09093160FAE
:10DED0008093150F81E090E0A0E0B0E08093170FF1
:10DEE0009093180FA093190FB0931A0F8EED93E033
:10DEF000A0E0B0E080931B0F90931C0FA0931D0F28
:10DF0000B0931E0F60915507709156078091570787
:10DF1000909158070C94187A043009F08DC08091C4
:10DF2000C503882339F16091050F7091060F809128
:10DF3000070F9091080F25E030E040E050E00E948C
:10DF4000CBFE243031054105510551F489E597E0B8
:10DF50000E94AC5B9C01812F60E571E24EE309C039
:10DF600089E597E00E94AC5B9C01812F60E571E23E
:10DF700040E21FDDFF2011F40C94237A6091050F1D
:10DF80007091060F8091070F9091080F25E030E007
:10DF900040E050E00E94CBFE2430310541055105A0
:10DFA00011F00C94237A0E941B608091C30390911E
:10DFB000C4039093100F80930F0F8091050F9091E1
:10DFC000060F9093120F8093110F82E08093C50388
:10DFD00080EB95E89093C4038093C30388E491E2B7
:10DFE0009093140F8093130F89E597E09093160F89
:10DFF0008093150F8AE090E0A0E0B0E08093170FC7
:10E000009093180FA093190FB0931A0F88EB92E812
:10E01000A1E0B0E080931B0F90931C0FA0931D0F05
:10E02000B0931E0F6091590770915A0780915B075A
:10E0300090915C070C946478053009F08DC0809154
:10E04000C503882339F16091050F7091060F809107
:10E05000070F9091080F25E030E040E050E00E946B
:10E06000CBFE253031054105510551F48DE597E092
:10E070000E94665A9C01812F60E471E24EE309C060
:10E080008DE597E00E94665A9C01812F60E471E261
:10E0900040E28FDCFF2011F40C94237A6091050F8D
:10E0A0007091060F8091070F9091080F25E030E0E6
:10E0B00040E050E00E94CBFE25303105410551057E
:10E0C00011F00C94237A0E941B608091C3039091FD
:10E0D000C4039093100F80930F0F8091050F9091C0
:10E0E000060F9093120F8093110F82E08093C50367
:10E0F0008CE398E89093C4038093C30388E391E290
:10E100009093140F8093130F8DE597E09093160F63
:10E110008093150F81E090E0A0E0B0E08093170FAE
:10E120009093180FA093190FB0931A0F8EED93E0F0
:10E13000A0E0B0E080931B0F90931C0FA0931D0FE5
:10E14000B0931E0F60915D0770915E0780915F072D
:10E15000909160070C94187A063009F08DC0809178
:10E16000C503882339F16091050F7091060F8091E6
:10E17000070F9091080F25E030E040E050E00E944A
:10E18000CBFE263031054105510551F485E197E07C
:10E190000E94665A9C01812F61E371E24EE309C03F
:10E1A00085E197E00E94665A9C01812F61E371E24C
:10E1B00040E2FFDBFF2011F40C94237A6091050FFD
:10E1C0007091060F8091070F9091080F25E030E0C5
:10E1D00040E050E00E94CBFE26303105410551055C
:10E1E00011F00C94237A0E941B608091C3039091DC
:10E1F000C4039093100F80930F0F8091050F90919F
:10E20000060F9093120F8093110F82E08093C50345
:10E210008CE398E89093C4038093C3038AE291E26D
:10E220009093140F8093130F85E197E09093160F4E
:10E230008093150F81E090E0A0E0B0E08093170F8D
:10E240009093180FA093190FB0931A0F87EE93E0D5
:10E25000A0E0B0E080931B0F90931C0FA0931D0FC4
:10E26000B0931E0F609115077091160780911707E4
:10E27000909118070C94187A073009F08DC080919E
:10E28000C503882339F16091050F7091060F8091C5
:10E29000070F9091080F25E030E040E050E00E9429
:10E2A000CBFE273031054105510551F489E197E056
:10E2B0000E94665A9C01812F63E271E24EE309C01D
:10E2C00089E197E00E94665A9C01812F63E271E226
:10E2D00040E26FDBFF2011F40C94237A6091050F6C
:10E2E0007091060F8091070F9091080F25E030E0A4
:10E2F00040E050E00E94CBFE27303105410551053A
:10E3000011F00C94237A0E941B608091C3039091BA
:10E31000C4039093100F80930F0F8091050F90917D
:10E32000060F9093120F8093110F82E08093C50324
:10E330008CE398E89093C4038093C3038CE191E24B
:10E340009093140F8093130F89E197E09093160F29
:10E350008093150F81E090E0A0E0B0E08093170F6C
:10E360009093180FA093190FB0931A0F87EE93E0B4
:10E37000A0E0B0E080931B0F90931C0FA0931D0FA3
:10E38000B0931E0F6091190770911A0780911B07B7
:10E3900090911C070C94187A083009F08CC0809179
:10E3A000C503882339F16091050F7091060F8091A4
:10E3B000070F9091080F25E030E040E050E00E9408
:10E3C000CBFE283031054105510551F48DE197E030
:10E3D0000E94665A9C01812F65E171E24EE309C0FB
:10E3E0008DE197E00E94665A9C01812F65E171E200
:10E3F00040E2DFDAFF2011F40C94237A6091050FDC
:10E400007091060F8091070F9091080F25E030E082
:10E4100040E050E00E94CBFE283031054105510517
:10E4200011F00C94237A0E941B608091C303909199
:10E43000C4039093100F80930F0F8091050F90915C
:10E44000060F9093120F8093110F82E08093C50303
:10E450008CE398E89093C4038093C3038EE091E229
:10E460009093140F8093130F8DE197E09093160F04
:10E470008093150F81E090E0A0E0B0E08093170F4B
:10E480009093180FA093190FB0931A0F87EE93E093
:10E49000A0E0B0E080931B0F90931C0FA0931D0F82
:10E4A000B0931E0F60911D0770911E0780911F078A
:10E4B00090912007BDC7093009F08AC08091C5033B
:10E4C000882339F16091050F7091060F8091070F35
:10E4D0009091080F25E030E040E050E00E94CBFE34
:10E4E000293031054105510551F481E297E00E9440
:10E4F000665A9C01812F67E071E24EE309C081E218
:10E5000097E00E94665A9C01812F67E071E240E229
:10E5100050DAFF2009F497C76091050F7091060F3C
:10E520008091070F9091080F25E030E040E050E027
:10E530000E94CBFE293031054105510509F083C702
:10E540000E941B608091C3039091C4039093100FAD
:10E5500080930F0F8091050F9091060F9093120FEB
:10E560008093110F82E08093C5038CE398E8909329
:10E57000C4038093C30380E091E29093140F8093CF
:10E58000130F81E297E09093160F8093150F81E0AF
:10E5900090E0A0E0B0E08093170F9093180FA09345
:10E5A000190FB0931A0F87EE93E0A0E0B0E08093CC
:10E5B0001B0F90931C0FA0931D0FB0931E0F609123
:10E5C000210770912207809123079091240730C77B
:10E5D0000A3009F086C08091C503882339F1609123
:10E5E000050F7091060F8091070F9091080F25E09D
:10E5F00030E040E050E00E94CBFE2A30310541057A
:10E60000510551F489E497E00E94665A9C01812FDC
:10E610006BEF70E24EE309C089E497E00E94665A0E
:10E620009C01812F6BEF70E240E2C3D9FF2009F417
:10E630000AC76091050F7091060F8091070F9091A6
:10E64000080F25E030E040E050E00E94CBFE2A3089
:10E6500031054105510509F0F6C60E941B60809105
:10E66000C3039091C4039093100F80930F0F809178
:10E67000050F9091060F9093120F8093110F82E077
:10E680008093C5038CE398E89093C4038093C303FD
:10E6900086EF90E29093140F8093130F89E497E034
:10E6A0009093160F8093150F1092170F1092180F5A
:10E6B0001092190F10921A0F87EE93E0A0E0B0E0CD
:10E6C00080931B0F90931C0FA0931D0FB0931E0FF0
:10E6D0006091490770914A0780914B0790914C07D0
:10E6E000A7C60B3009F086C08091C503882339F195
:10E6F0006091050F7091060F8091070F9091080FA0
:10E7000025E030E040E050E00E94CBFE2B303105A8
:10E710004105510551F481E697E00E94665A9C013B
:10E72000812F6CEE70E24EE309C081E697E00E9413
:10E73000665A9C01812F6CEE70E240E23AD9FF20CC
:10E7400009F481C66091050F7091060F8091070F43
:10E750009091080F25E030E040E050E00E94CBFEB1
:10E760002B3031054105510509F06DC60E941B6033
:10E770008091C3039091C4039093100F80930F0F67
:10E780008091050F9091060F9093120F8093110FB7
:10E7900082E08093C5038CE398E89093C403809350
:10E7A000C30382EE90E29093140F8093130F81E6DF
:10E7B00097E09093160F8093150F1092170F1092F9
:10E7C000180F1092190F10921A0F87EE93E0A0E025
:10E7D000B0E080931B0F90931C0FA0931D0FB0937C
:10E7E0001E0F60916107709162078091630790919D
:10E7F00064071EC60C3009F0A7C08091C5038823AA
:10E8000009F443C06091050F7091060F8091070FC6
:10E810009091080F25E030E040E050E00E94CBFEF0
:10E820002C30310541055105C1F4609139077091D3
:10E830003A0780913B0790913C070E9473FB6983E4
:10E840007A838B839C83CE0101960E947D5A9C0122
:10E85000812F6BED70E24EE317C060913907709124
:10E860003A0780913B0790913C070E9473FB6D83B0
:10E870007E838F839887CE0105960E947D5A9C01E6
:10E88000812F6BED70E240E294D8FF2009F4DBC5E4
:10E890006091050F7091060F8091070F9091080FFE
:10E8A00025E030E040E050E00E94CBFE2C30310506
:10E8B0004105510509F0C7C50E941B608091C30343
:10E8C0009091C4039093100F80930F0F8091050FC8
:10E8D0009091060F9093120F8093110F82E0809316
:10E8E000C5038EE594E89093C4038093C30384ED3D
:10E8F00090E29093140F8093130F89E397E0909325
:10E90000160F8093150F81E090E0A0E0B0E08093B7
:10E91000170F9093180FA093190FB0931A0F8EED45
:10E9200093E0A0E0B0E080931B0F90931C0FA093A6
:10E930001D0FB0931E0F6091390770913A078091B7
:10E940003B0790913C07FAC10D3009F0A6C08091B9
:10E95000C503882309F442C06091050F7091060F2A
:10E960008091070F9091080F25E030E040E050E0E3
:10E970000E94CBFE2D30310541055105B9F460915F
:10E980003D0770913E0780913F07909140070E949C
:10E9900073FB69877A878B879C87C1010E947D5AA8
:10E9A0009C01812F6DEC70E24EE316C060913D0733
:10E9B00070913E0780913F07909140070E9473FB42
:10E9C0006D877E878F87988BC2010E947D5A9C013C
:10E9D000812F6DEC70E240E20E94D96CFF2009F4B7
:10E9E00032C56091050F7091060F8091070F9091CD
:10E9F000080F25E030E040E050E00E94CBFE2D30D3
:10EA000031054105510509F01EC50E941B6080912A
:10EA1000C3039091C4039093100F80930F0F8091C4
:10EA2000050F9091060F9093120F8093110F82E0C3
:10EA30008093C5038EE594E89093C4038093C30349
:10EA400086EC90E29093140F8093130F8DE397E080
:10EA50009093160F8093150F81E090E0A0E0B0E056
:10EA60008093170F9093180FA093190FB0931A0F5C
:10EA70008EED93E0A0E0B0E080931B0F90931C0F0D
:10EA8000A0931D0FB0931E0F60913D0770913E073C
:10EA900080913F079091400751C10E3009F0A6C008
:10EAA0008091C503882309F442C06091050F7091DD
:10EAB000060F8091070F9091080F25E030E040E0AD
:10EAC00050E00E94CBFE2E30310541055105B9F4CE
:10EAD00060914107709142078091430790914407EC
:10EAE0000E9473FB698B7A8B8B8B9C8BC3010E947A
:10EAF0007D5A9C01812F6FEB70E24EE316C060914E
:10EB000041077091420780914307909144070E940A
:10EB100073FB6D8B7E8B8F8B988FC4010E947D5A07
:10EB20009C01812F6FEB70E240E20E94D96CFF20C4
:10EB300009F489C46091050F7091060F8091070F49
:10EB40009091080F25E030E040E050E00E94CBFEBD
:10EB50002E3031054105510509F075C40E941B6036
:10EB60008091C3039091C4039093100F80930F0F73
:10EB70008091050F9091060F9093120F8093110FC3
:10EB800082E08093C5038EE594E89093C40380935C
:10EB9000C30388EB90E29093140F8093130F81E4EA
:10EBA00097E09093160F8093150F81E090E0A0E01E
:10EBB000B0E08093170F9093180FA093190FB093A4
:10EBC0001A0F8EED93E0A0E0B0E080931B0F9093BE
:10EBD0001C0FA0931D0FB0931E0F60914107709101
:10EBE00042078091430790914407A8C00F3009F075
:10EBF000BEC08091C503882309F442C06091050F0F
:10EC00007091060F8091070F9091080F25E030E07A
:10EC100040E050E00E94CBFE2F3031054105510508
:10EC2000B9F460914507709146078091470790912C
:10EC300048070E9473FB698F7A8F8B8F9C8FC50169
:10EC40000E947D5A9C01812F61EB70E24EE316C059
:10EC5000609145077091460780914707909148075A
:10EC60000E9473FB6D8F7E8F8F8F98A3C6010E94C9
:10EC70007D5A9C01812F61EB70E240E20E94D96CC9
:10EC8000FF2009F4E0C36091050F7091060F809199
:10EC9000070F9091080F25E030E040E050E00E941F
:10ECA000CBFE2F3031054105510509F0CCC30E9440
:10ECB0001B608091C3039091C4039093100F8093C5
:10ECC0000F0F8091050F9091060F9093120F809374
:10ECD000110F82E08093C5038EE594E89093C403FE
:10ECE0008093C3038AEA90E29093140F8093130FEA
:10ECF00085E497E09093160F8093150F81E090E0E4
:10ED0000A0E0B0E08093170F9093180FA093190F15
:10ED1000B0931A0F8EED93E0A0E0B0E080931B0F4C
:10ED200090931C0FA0931D0FB0931E0F6091450789
:10ED30007091460780914707909148070E9473FBA6
:10ED40002AE037ED43E25CE30E94B3FD0E9447FBFB
:10ED50006093050F7093060F8093070F9093080F31
:10ED60008BEB99E39093200F80931F0FABC300317F
:10ED700009F08FC08091C503882341F16091050F90
:10ED80007091060F8091070F9091080F25E030E0F9
:10ED900040E050E00E94CBFE203131054105510595
:10EDA00051F481E597E00E947D5A9C01812F60EA31
:10EDB00070E24EE309C081E597E00E947D5A9C0114
:10EDC000812F60EA70E240E20E94D96CFF2009F4D2
:10EDD0003AC36091050F7091060F8091070F9091D3
:10EDE000080F25E030E040E050E00E94CBFE2031EB
:10EDF00031054105510509F026C30E941B60809131
:10EE0000C3039091C4039093100F80930F0F8091D0
:10EE1000050F9091060F9093120F8093110F82E0CF
:10EE20008093C50386EF96E89093C4038093C30351
:10EE300086E990E29093140F8093130F81E597E099
:10EE40009093160F8093150F81E090E0A0E0B0E062
:10EE50008093170F9093180FA093190FB0931A0F68
:10EE60008EED93E0A0E0B0E080931B0F90931C0F19
:10EE7000A0931D0FB0931E0F609151077091520720
:10EE800080915307909154072AE037ED43E25CE309
:10EE9000CDC2013109F08BC08091C503882341F1B7
:10EEA0006091050F7091060F8091070F9091080FE8
:10EEB00025E030E040E050E00E94CBFE21313105FA
:10EEC0004105510551F485E297E00E94AC5B9C013D
:10EED000812F6CE870E24EE309C085E297E00E9462
:10EEE000AC5B9C01812F6CE870E240E20E94D96C1F
:10EEF000FF2009F4A8C26091050F7091060F809160
:10EF0000070F9091080F25E030E040E050E00E94AC
:10EF1000CBFE213131054105510509F094C20E9413
:10EF20001B608091C3039091C4039093100F809352
:10EF30000F0F8091050F9091060F9093120F809301
:10EF4000110F82E08093C50380EB95E89093C40392
:10EF50008093C30382E890E29093140F8093130F81
:10EF600085E297E09093160F8093150F84EF91E060
:10EF7000A0E0B0E08093170F9093180FA093190FA3
:10EF8000B0931A0F8CED91E4AFE0B0E080931B0FCB
:10EF900090931C0FA0931D0FB0931E0F6091250737
:10EFA0007091260780912707909128078DC0023124
:10EFB00009F08FC08091C503882341F16091050F4E
:10EFC0007091060F8091070F9091080F25E030E0B7
:10EFD00040E050E00E94CBFE223131054105510551
:10EFE00051F489E297E00E94AC5B9C01812F68E7B5
:10EFF00070E24EE309C089E297E00E94AC5B9C019D
:10F00000812F68E770E240E20E94D96CFF2009F48A
:10F010001AC26091050F7091060F8091070F9091B1
:10F02000080F25E030E040E050E00E94CBFE2231A6
:10F0300031054105510509F006C20E941B6080910F
:10F04000C3039091C4039093100F80930F0F80918E
:10F05000050F9091060F9093120F8093110F82E08D
:10F060008093C50380EB95E89093C4038093C3031A
:10F070008EE690E29093140F8093130F89E297E04D
:10F080009093160F8093150F84EF91E0A0E0B0E00D
:10F090008093170F9093180FA093190FB0931A0F26
:10F0A0008CED91E4AFE0B0E080931B0F90931C0FC8
:10F0B000A0931D0FB0931E0F6091290770912A072E
:10F0C00080912B0790912C0720E030E048EC52E42F
:10F0D000ADC1033109F08BC08091C503882341F194
:10F0E0006091050F7091060F8091070F9091080FA6
:10F0F00025E030E040E050E00E94CBFE23313105B6
:10F100004105510551F48DE297E00E94255B9C0179
:10F11000812F64E670E24EE309C08DE297E00E9421
:10F12000255B9C01812F64E670E240E20E94D96C6D
:10F13000FF2009F488C16091050F7091060F80913E
:10F14000070F9091080F25E030E040E050E00E946A
:10F15000CBFE233131054105510509F074C10E94F0
:10F160001B608091C3039091C4039093100F809310
:10F170000F0F8091050F9091060F9093120F8093BF
:10F18000110F82E08093C50383E596E89093C40352
:10F190008093C3038AE590E29093140F8093130F3A
:10F1A0008DE297E09093160F8093150F82E390E025
:10F1B000A0E0B0E08093170F9093180FA093190F61
:10F1C000B0931A0F86E996E8A1E0B0E080931B0F98
:10F1D00090931C0FA0931D0FB0931E0F60912D07ED
:10F1E00070912E0780912F07909130071BC1043139
:10F1F00009F08BC08091C503882341F16091050F10
:10F200007091060F8091070F9091080F25E030E074
:10F2100040E050E00E94CBFE24313105410551050C
:10F2200051F481E397E00E94255B9C01812F60E50A
:10F2300070E24EE309C081E397E00E94255B9C01E8
:10F24000812F60E570E240E20E94D96CFF2009F452
:10F25000FAC06091050F7091060F8091070F909191
:10F26000080F25E030E040E050E00E94CBFE243162
:10F2700031054105510509F0E6C00E941B608091EF
:10F28000C3039091C4039093100F80930F0F80914C
:10F29000050F9091060F9093120F8093110F82E04B
:10F2A0008093C50383E596E89093C4038093C303DA
:10F2B00086E490E29093140F8093130F81E397E01C
:10F2C0009093160F8093150F82E390E0A0E0B0E0DA
:10F2D0008093170F9093180FA093190FB0931A0FE4
:10F2E00086E996E8A1E0B0E080931B0F90931C0F95
:10F2F000A0931D0FB0931E0F6091310770913207DC
:10F3000080913307909134078DC0053109F09BC07F
:10F310008091C503882341F16091050F7091060F1C
:10F320008091070F9091080F25E030E040E050E019
:10F330000E94CBFE253131054105510551F485E38D
:10F3400097E00E94255B9C01812F6CE370E24EE305
:10F3500009C085E397E00E94255B9C01812F6CE347
:10F3600070E240E20E94D96CFF2009F46CC0609109
:10F37000050F7091060F8091070F9091080F25E0FF
:10F3800030E040E050E00E94CBFE253131054105E0
:10F39000510509F058C00E941B608091C3039091F1
:10F3A000C4039093100F80930F0F8091050F9091DD
:10F3B000060F9093120F8093110F82E08093C50384
:10F3C00083E596E89093C4038093C30382E390E2BD
:10F3D0009093140F8093130F85E397E09093160F8B
:10F3E0008093150F82E390E0A0E0B0E08093170FC8
:10F3F0009093180FA093190FB0931A0F86E996E80F
:10F40000A1E0B0E080931B0F90931C0FA0931D0F01
:10F41000B0931E0F609135077091360780913707C2
:10F420009091380720E030E040E251E40E94B3FDC3
:10F430000E9447FB6093050F7093060F8093070FA0
:10F440009093080F3FC08091050F9091060FA091F7
:10F45000070FB091080F8E369105A105B10560F038
:10F460008DE690E0A0E0B0E08093050F9093060F4A
:10F47000A093070FB093080F6091050F7091060FCE
:10F480008091070F9091080F25E030E040E050E0B8
:10F490000E94CBFE422F8091FF0E90E0049630E058
:10F4A000821793074CF444504093FF0E81E0809301
:10F4B000C503042F01501FEF1F5F153018F40F5FB5
:10F4C0000C94996DA0960FB6F894DEBF0FBECDBF19
:10F4D000CF91DF911F910F91FF90EF90DF90CF9030
:10F4E000BF90AF909F908F907F906F905F904F9064
:10F4F0003F902F900895AF92BF92CF92DF92EF92FC
:10F50000FF920F931F938091050F9091060FA0918A
:10F51000070FB091080F81509048A040B04040F0D4
:10F520001092050F1092060F1092070F1092080FFD
:10F530006091050F7091060F8091070F9091080F51
:10F5400025E030E040E050E00E94CBFE79018A01E6
:10F550008091FF0E90E0A0E0B0E0E816F9060A07FF
:10F560001B0710F42093FF0E0091FF0E8091FE0EFA
:10F5700090E09695879596958795FF24F394F822C9
:10F5800010E038E1A32EB12CC12CD12CEE24E39451
:10F59000002309F03DC08091C5038823C1F080910C
:10F5A000050F9091060FA091070FB091080F0597D6
:10F5B000A105B10528F4812F60EA72E24BEF04C087
:10F5C000812F60EA72E240E22BEF0E94AA5CFF20EA
:10F5D00009F4FBC18091050F9091060FA091070FD0
:10F5E000B091080F0597A105B10508F0EEC10E9482
:10F5F0001B6083EA99E89093C4038093C30310923D
:10F60000050F1092060F1092070F1092080F15C2E7
:10F61000013009F083C08091C503882341F16091D6
:10F62000050F7091060F8091070F9091080F25E04C
:10F6300030E040E050E00E94CBFE21303105410532
:10F64000510551F48DEB9CE00E94315A9C01812FB1
:10F6500066E972E24EE309C08DEB9CE00E94315AEC
:10F660009C01812F66E972E240E20E94D96CFF2082
:10F6700009F4ABC16091050F7091060F8091070FDF
:10F680009091080F25E030E040E050E00E94CBFE72
:10F69000213031054105510509F097C10E941B60D9
:10F6A0008091C3039091C4039093100F80930F0F28
:10F6B0008091050F9091060F9093120F8093110F78
:10F6C00082E08093C50383ED98E89093C403809310
:10F6D000C3038CE892E29093140F8093130F8DEB89
:10F6E0009CE09093160F8093150F1092170F1092B5
:10F6F000180F1092190F10921A0F8FEF90E0A0E0E0
:10F70000B0E080931B0F90931C0FA0931D0FB0933C
:10F710001E0F8091BD0C9091BE0C0BC1023009F000
:10F7200083C08091C503882341F16091050F7091DA
:10F73000060F8091070F9091080F25E030E040E020
:10F7400050E00E94CBFE223031054105510551F4B5
:10F7500089EB9CE00E94315A9C01812F65E872E29E
:10F760004EE309C089EB9CE00E94315A9C01812F35
:10F7700065E872E240E20E94D96CFF2009F425C1DD
:10F780006091050F7091060F8091070F9091080FFF
:10F7900025E030E040E050E00E94CBFE2230310511
:10F7A0004105510509F011C10E941B608091C303FE
:10F7B0009091C4039093100F80930F0F8091050FC9
:10F7C0009091060F9093120F8093110F82E0809317
:10F7D000C50383ED98E89093C4038093C3038EE739
:10F7E00092E29093140F8093130F89EB9CE0909317
:10F7F000160F8093150F1092170F1092180F10927A
:10F80000190F10921A0F8BEE90E0A0E0B0E08093F9
:10F810001B0F90931C0FA0931D0FB0931E0F809190
:10F82000B90C9091BA0C85C0033009F08FC080915B
:10F83000C503882341F16091050F7091060F8091F7
:10F84000070F9091080F25E030E040E050E00E9463
:10F85000CBFE233031054105510551F48BEB9CE083
:10F860000E94315A9C01812F6AE772E24EE309C07F
:10F870008BEB9CE00E94315A9C01812F6AE772E277
:10F8800040E20E94D96CFF2009F49FC06091050FEF
:10F890007091060F8091070F9091080F25E030E0DE
:10F8A00040E050E00E94CBFE233031054105510578
:10F8B00009F08BC00E941B608091C3039091C40328
:10F8C0009093100F80930F0F8091050F9091060F6A
:10F8D0009093120F8093110F82E08093C50383ED04
:10F8E00098E89093C4038093C30386E792E29093D1
:10F8F000140F8093130F8BEB9CE09093160F809363
:10F90000150F1092170F1092180F1092190F1092D6
:10F910001A0F87E890E0A0E0B0E080931B0F90936F
:10F920001C0FA0931D0FB0931E0F8091BB0C9091E4
:10F93000BC0CAA2797FDA095BA2F8093050F909332
:10F94000060FA093070FB093080F77C00430E9F5B6
:10F950008091C5038823F9F06091050F7091060F1F
:10F960008091070F9091080F25E030E040E050E0D3
:10F970000E94CBFE243031054105510529F4812F29
:10F9800069E672E24EE304C0812F69E672E240E26A
:10F9900020E20E94AA5CFF20C1F06091050F7091E7
:10F9A000060F8091070F9091080F25E030E040E0AE
:10F9B00050E00E94CBFE243031054105510529F469
:10F9C0000E941B600E94F19C38C08091050F9091AD
:10F9D000060FA091070FB091080F4997A105B10537
:10F9E00040F0A092050FB092060FC092070FD09280
:10F9F000080F6091050F7091060F8091070F90918D
:10FA0000080F25E030E040E050E00E94CBFE422F9E
:10FA10008091FF0E90E0049630E08217930744F443
:10FA200044504093FF0EE092C503042F01501FEF96
:10FA30001F5F153010F40F5FABCD1F910F91FF903A
:10FA4000EF90DF90CF90BF90AF900895AF92BF92AC
:10FA5000CF92DF92EF92FF920F931F938091050F49
:10FA60009091060FA091070FB091080F8150904818
:10FA7000A040B04040F01092050F1092060F109277
:10FA8000070F1092080F6091050F7091060F80917B
:10FA9000070F9091080F25E030E040E050E00E9411
:10FAA000CBFE79018A018091FF0E90E0A0E0B0E0EA
:10FAB000E816F9060A071B0710F42093FF0E0091C1
:10FAC000FF0E8091FE0E90E096958795969587950E
:10FAD000FF24F394F82210E058E1A52EB12CC12C9C
:10FAE000D12CEE24E394002309F03DC08091C5039E
:10FAF0008823C1F08091050F9091060FA091070F08
:10FB0000B091080F0597A105B10528F4812F63EE88
:10FB100072E24BEF04C0812F63EE72E240E22BEF02
:10FB20000E94AA5CFF2009F4FBC18091050F90910F
:10FB3000060FA091070FB091080F0597A105B10519
:10FB400008F0EEC10E941B6083EA99E89093C40319
:10FB50008093C3031092050F1092060F1092070FA7
:10FB60001092080F15C2013009F083C08091C503BF
:10FB7000882341F16091050F7091060F8091070F66
:10FB80009091080F25E030E040E050E00E94CBFE6D
:10FB9000213031054105510551F487EB9CE00E946D
:10FBA000315A9C01812F69ED72E24EE309C087EB67
:10FBB0009CE00E94315A9C01812F69ED72E240E283
:10FBC0000E94D96CFF2009F4ABC16091050F7091C0
:10FBD000060F8091070F9091080F25E030E040E07C
:10FBE00050E00E94CBFE213031054105510509F05E
:10FBF00097C10E941B608091C3039091C4039093AE
:10FC0000100F80930F0F8091050F9091060F909326
:10FC1000120F8093110F82E08093C50383ED98E863
:10FC20009093C4038093C3038FEC92E29093140FDC
:10FC30008093130F87EB9CE09093160F8093150F22
:10FC40001092170F1092180F1092190F10921A0F8E
:10FC50008FEF90E0A0E0B0E080931B0F90931C0F1B
:10FC6000A0931D0FB0931E0F8091B70C9091B80C0C
:10FC70000BC1023009F083C08091C503882341F194
:10FC80006091050F7091060F8091070F9091080FFA
:10FC900025E030E040E050E00E94CBFE223031050C
:10FCA0004105510551F483EB9CE00E94315A9C01BF
:10FCB000812F68EC72E24EE309C083EB9CE00E9466
:10FCC000315A9C01812F68EC72E240E20E94D96CAB
:10FCD000FF2009F425C16091050F7091060F8091F6
:10FCE000070F9091080F25E030E040E050E00E94BF
:10FCF000CBFE223031054105510509F011C10E94AA
:10FD00001B608091C3039091C4039093100F809364
:10FD10000F0F8091050F9091060F9093120F809313
:10FD2000110F82E08093C50383ED98E89093C4039C
:10FD30008093C30381EC92E29093140F8093130F8E
:10FD400083EB9CE09093160F8093150F1092170F82
:10FD50001092180F1092190F10921A0F8BEE90E05C
:10FD6000A0E0B0E080931B0F90931C0FA0931D0F99
:10FD7000B0931E0F8091B30C9091B40C85C00330EA
:10FD800009F08FC08091C503882341F16091050F70
:10FD90007091060F8091070F9091080F25E030E0D9
:10FDA00040E050E00E94CBFE233031054105510573
:10FDB00051F485EB9CE00E94315A9C01812F6DEB40
:10FDC00072E24EE309C085EB9CE00E94315A9C012F
:10FDD000812F6DEB72E240E20E94D96CFF2009F4A2
:10FDE0009FC06091050F7091060F8091070F909151
:10FDF000080F25E030E040E050E00E94CBFE2330C9
:10FE000031054105510509F08BC00E941B608091AE
:10FE1000C3039091C4039093100F80930F0F8091B0
:10FE2000050F9091060F9093120F8093110F82E0AF
:10FE30008093C50383ED98E89093C4038093C30334
:10FE400089EB92E29093140F8093130F85EB9CE063
:10FE50009093160F8093150F1092170F1092180F92
:10FE60001092190F10921A0F87E890E0A0E0B0E00E
:10FE700080931B0F90931C0FA0931D0FB0931E0F28
:10FE80008091B50C9091B60CAA2797FDA095BA2F3A
:10FE90008093050F9093060FA093070FB093080F60
:10FEA00077C00430E9F58091C5038823F9F06091AB
:10FEB000050F7091060F8091070F9091080F25E0B4
:10FEC00030E040E050E00E94CBFE24303105410597
:10FED000510529F4812F6CEA72E24EE304C0812FB0
:10FEE0006CEA72E240E220E20E94AA5CFF20C1F0CC
:10FEF0006091050F7091060F8091070F9091080F88
:10FF000025E030E040E050E00E94CBFE2430310597
:10FF10004105510529F40E941B600E94F19C38C0E4
:10FF20008091050F9091060FA091070FB091080FD7
:10FF30004997A105B10540F0A092050FB092060FB8
:10FF4000C092070FD092080F6091050F7091060FB5
:10FF50008091070F9091080F25E030E040E050E0DD
:10FF60000E94CBFE422F8091FF0E90E0049630E07D
:10FF70008217930744F444504093FF0EE092C50368
:10FF8000042F01501FEF1F5F153010F40F5FABCD32
:10FF90001F910F91FF90EF90DF90CF90BF90AF90A7
:10FFA0000895AF92BF92CF92DF92EF92FF920F939C
:10FFB0001F938091050F9091060FA091070FB091AC
:10FFC000080F81509048A040B04040F01092050FBB
:10FFD0001092060F1092070F1092080F6091050FF4
:10FFE0007091060F8091070F9091080F25E030E087
:10FFF00040E050E00E94CBFE79018A018091FF0E23
:020000021000EC
:1000000090E0A0E0B0E0E816F9060A071B0710F43C
:100010002093FF0E0091FF0E8091FE0E90E09695CA
:10002000879596958795FF24F394F82210E077E260
:10003000A72EB12CC12CD12CEE24E394002309F07F
:100040003DC08091C5038823C1F08091050F909138
:10005000060FA091070FB091080F0597A105B105F4
:1000600028F4812F64E074E24BEF04C0812F64E038
:1000700074E240E22BEF0E94AA5CFF2009F498C3CF
:100080008091050F9091060FA091070FB091080F76
:100090000597A105B10508F08BC30E941B6081EE96
:1000A00097E69093C4038093C3031092050F1092B8
:1000B000060F1092070F1092080FB2C3013009F01B
:1000C00087C08091C503882341F16091050F70912D
:1000D000060F8091070F9091080F25E030E040E077
:1000E00050E00E94CBFE213031054105510551F40D
:1000F00086ED93E00E94315A9C01812F6EEF73E2EE
:100100004EE309C086ED93E00E94315A9C01812F95
:100110006EEF73E240E20E94D96CFF2009F448C3FD
:100120006091050F7091060F8091070F9091080F55
:1001300025E030E040E050E00E94CBFE2130310568
:100140004105510509F034C30E941B608091C3032F
:100150009091C4039093100F80930F0F8091050F1F
:100160009091060F9093120F8093110F82E080936D
:10017000C50383ED98E89093C4038093C30388EF8D
:1001800093E29093140F8093130F86ED93E0909376
:10019000160F8093150F8AE090E0A0E0B0E0809306
:1001A000170F9093180FA093190FB0931A0F87EEA3
:1001B00093E0A0E0B0E080931B0F90931C0FA093FE
:1001C0001D0FB0931E0F8091D6039091D703A1C24B
:1001D000023009F083C08091C503882341F160910A
:1001E000050F7091060F8091070F9091080F25E081
:1001F00030E040E050E00E94CBFE22303105410566
:10020000510551F485E694E10E94315A9C01812FF9
:1002100061EF73E24EE309C085E694E10E94315A32
:100220009C01812F61EF73E240E20E94D96CFF20B4
:1002300009F4BEC26091050F7091060F8091070FFF
:100240009091080F25E030E040E050E00E94CBFEA6
:10025000223031054105510509F0AAC20E941B60F8
:100260008091C3039091C4039093100F80930F0F5C
:100270008091050F9091060F9093120F8093110FAC
:1002800082E08093C50383ED98E89093C403809344
:10029000C3038AEE93E29093140F8093130F85E6C5
:1002A00094E19093160F8093150F1092170F1092F0
:1002B000180F1092190F10921A0F8BEE90E0A0E019
:1002C000B0E080931B0F90931C0FA0931D0FB09371
:1002D0001E0F80916514909166141BC2033009F0C3
:1002E00083C08091C503882341F16091050F70910F
:1002F000060F8091070F9091080F25E030E040E055
:1003000050E00E94CBFE233031054105510551F4E8
:1003100087E694E10E94315A9C01812F62EE73E2DC
:100320004EE309C087E694E10E94315A9C01812F77
:1003300062EE73E240E20E94D96CFF2009F438C2F9
:100340006091050F7091060F8091070F9091080F33
:1003500025E030E040E050E00E94CBFE2330310544
:100360004105510509F024C20E941B608091C3031E
:100370009091C4039093100F80930F0F8091050FFD
:100380009091060F9093120F8093110F82E080934B
:10039000C50383ED98E89093C4038093C3038AED6B
:1003A00093E29093140F8093130F87E694E1909358
:1003B000160F8093150F1092170F1092180F1092AE
:1003C000190F10921A0F8BEE90E0A0E0B0E080932E
:1003D0001B0F90931C0FA0931D0FB0931E0F8091C5
:1003E00067149091681495C1043009F083C080911E
:1003F000C503882341F16091050F7091060F80912C
:10040000070F9091080F25E030E040E050E00E9497
:10041000CBFE243031054105510551F487E694E1C6
:100420000E94315A9C01812F66ED73E24EE309C0B0
:1004300087E694E10E94315A9C01812F66ED73E2B8
:1004400040E20E94D96CFF2009F4B2C16091050F0F
:100450007091060F8091070F9091080F25E030E012
:1004600040E050E00E94CBFE2430310541055105AB
:1004700009F09EC10E941B608091C3039091C40348
:100480009093100F80930F0F8091050F9091060F9E
:100490009093120F8093110F82E08093C50383ED38
:1004A00098E89093C4038093C30382ED93E2909302
:1004B000140F8093130F87E694E19093160F8093A7
:1004C000150F1092170F1092180F1092190F10920B
:1004D0001A0F87E890E0A0E0B0E080931B0F9093A4
:1004E0001C0FA0931D0FB0931E0F80916714909165
:1004F00068140FC1053009F083C08091C5038823BB
:1005000041F16091050F7091060F8091070F909156
:10051000080F25E030E040E050E00E94CBFE25309F
:1005200031054105510551F484E892E10E94315AA8
:100530009C01812F68EC73E24EE309C084E892E1EC
:100540000E94315A9C01812F68EC73E240E20E94C4
:10055000D96CFF2009F42CC16091050F7091060F32
:100560008091070F9091080F25E030E040E050E0C7
:100570000E94CBFE253031054105510509F018C117
:100580000E941B608091C3039091C4039093100F4D
:1005900080930F0F8091050F9091060F9093120F8B
:1005A0008093110F82E08093C50383ED98E89093C8
:1005B000C4038093C3038EEB93E29093140F809354
:1005C000130F84E892E19093160F8093150F109209
:1005D000170F1092180F1092190F10921A0F8FEF19
:1005E00090E0A0E0B0E080931B0F90931C0FA093CD
:1005F0001D0FB0931E0F809184129091851289C0B7
:10060000063009F093C08091C503882341F16091C1
:10061000050F7091060F8091070F9091080F25E04C
:1006200030E040E050E00E94CBFE2630310541052D
:10063000510551F488ED93E00E94315A9C01812FBD
:1006400069EB73E24EE309C088ED93E00E94315AF2
:100650009C01812F69EB73E240E20E94D96CFF207C
:1006600009F4A6C06091050F7091060F8091070FE5
:100670009091080F25E030E040E050E00E94CBFE72
:10068000263031054105510509F092C00E941B60DA
:100690008091C3039091C4039093100F80930F0F28
:1006A0008091050F9091060F9093120F8093110F78
:1006B00082E08093C50383ED98E89093C403809310
:1006C000C30384EB93E29093140F8093130F88ED90
:1006D00093E09093160F8093150F8AE090E0A0E0CE
:1006E000B0E08093170F9093180FA093190FB09359
:1006F0001A0F87EE93E0A0E0B0E080931B0F909379
:100700001C0FA0931D0FB0931E0F8091D8039091E2
:10071000D903AA2797FDA095BA2F8093050F909330
:10072000060FA093070FB093080F7AC0073009F0A7
:100730003FC08091C5038823F9F06091050F709147
:10074000060F8091070F9091080F25E030E040E000
:1007500050E00E94CBFE273031054105510529F4B8
:10076000812F64EA73E24EE304C0812F64EA73E2EE
:1007700040E220E20E94AA5CFF20D1F06091050FC8
:100780007091060F8091070F9091080F25E030E0DF
:1007900040E050E00E94CBFE273031054105510575
:1007A00039F40E941B608FE993E20E94EECC38C0BE
:1007B0008091050F9091060FA091070FB091080F3F
:1007C0008897A105B10540F0A092050FB092060FE1
:1007D000C092070FD092080F6091050F7091060F1D
:1007E0008091070F9091080F25E030E040E050E045
:1007F0000E94CBFE422F8091FF0E90E0049630E0E5
:100800008217930744F444504093FF0EE092C503CF
:10081000042F01501FEF1F5F153010F40F5F0ECC37
:100820001F910F91FF90EF90DF90CF90BF90AF900E
:100830000895CF92DF92EF92FF920F931F937C0166
:10084000D62EC72E07EC1EE08091C70E8B5110925A
:10085000FB0E8093FC0EC80101976EEE72E10E94C0
:100860008BEFC7010E949A5C05501040C8016AE3F3
:100870000E942EF6ED2DFC2DDF010D900020E9F7F2
:100880002091C70E2B51EA1BFB0B7396CF01A3E0FF
:10089000880F991FAA95E1F78E1B9F0B8093FB0E83
:1008A0002093FC0EC8016D2D7C2D0E9452F61F91E5
:1008B0000F91FF90EF90DF90CF9008950F931F93CB
:1008C000DF93CF9300D00F92CDB7DEB72091170FF3
:1008D0003091180F4091190F50911A0F8091050F08
:1008E0009091060FA091070FB091080F8217930700
:1008F000A407B50744F42093050F3093060F4093E7
:10090000070F5093080F20911B0F30911C0F40913F
:100910001D0F50911E0F8091050F9091060FA09111
:10092000070FB091080F281739074A075B0744F4EF
:100930002093050F3093060F4093070F5093080F35
:100940008091C5038823F9F00091130F1091140FC3
:100950006091050F7091060F8091070F9091080F1D
:100960000E9473FB2AE037ED43E25CE30E94DAFA6F
:1009700069837A838B839C83CE0101960E947D5A82
:10098000BC01C80156DF8091FE0E82FF38C0009185
:10099000150F1091160F6091050F7091060F809141
:1009A000070F9091080F0E9473FB2AE037ED43E296
:1009B0005CE30E94DAFA0E9447FBF80160837183CE
:1009C000828393830E941B6080910F0F9091100F80
:1009D0009093C4038093C3038091110F9091120FE1
:1009E000A0E0B0E08093050F9093060FA093070F4F
:1009F000B093080FE0911F0FF091200F19950F9001
:100A00000F900F900F90CF91DF911F910F9108954C
:100A10000F931F93DF93CF9300D00F92CDB7DEB724
:100A20002091170F3091180F4091190F50911A0F04
:100A30008091050F9091060FA091070FB091080FBC
:100A400082179307A407B50744F42093050F30934A
:100A5000060F4093070F5093080F20911B0F309102
:100A60001C0F40911D0F50911E0F8091050F90910A
:100A7000060FA091070FB091080F281739074A07F2
:100A80005B0744F42093050F3093060F4093070F44
:100A90005093080F8091C5038823F9F00091130F3C
:100AA0001091140F6091050F7091060F8091070F40
:100AB0009091080F0E9473FB20E030E048EC52E474
:100AC0000E94DAFA69837A838B839C83CE01019634
:100AD0000E94AC5BBC01C801ACDE8091FE0E82FFBF
:100AE00036C00091150F1091160F6091050F70918F
:100AF000060F8091070F9091080F0E9473FB20E072
:100B000030E048EC52E40E94DAFAF8016083718325
:100B1000828393830E941B6080910F0F9091100F2E
:100B20009093C4038093C3038091110F9091120F8F
:100B3000A0E0B0E08093050F9093060FA093070FFD
:100B4000B093080FE0911F0FF091200F19950F90AF
:100B50000F900F900F90CF91DF911F910F910895FB
:100B60000F931F93DF93CF9300D00F92CDB7DEB7D3
:100B70002091170F3091180F4091190F50911A0FB3
:100B80008091050F9091060FA091070FB091080F6B
:100B900082179307A407B50744F42093050F3093F9
:100BA000060F4093070F5093080F20911B0F3091B1
:100BB0001C0F40911D0F50911E0F8091050F9091B9
:100BC000060FA091070FB091080F281739074A07A1
:100BD0005B0744F42093050F3093060F4093070FF3
:100BE0005093080F8091C5038823F9F00091130FEB
:100BF0001091140F6091050F7091060F8091070FEF
:100C00009091080F0E9473FB20E030E048EC52E422
:100C10000E94DAFA69837A838B839C83CE010196E2
:100C20000E94AC5BBC01C80104DE8091FE0E82FF15
:100C300031C00091150F1091160F6091050F709142
:100C4000060F8091070F9091080F0E9473FB20E020
:100C500030E048EC52E40E94DAFAF80160837183D4
:100C6000828393830E941B6080910F0F9091100FDD
:100C70009093C4038093C3038091110F9091120F3E
:100C8000A0E0B0E08093050F9093060FA093070FAC
:100C9000B093080F0F900F900F900F90CF91DF91AE
:100CA0001F910F9108950F931F93DF93CF9300D05F
:100CB0000F92CDB7DEB72091170F3091180F4091EA
:100CC000190F50911A0F8091050F9091060FA09166
:100CD000070FB091080F82179307A407B50744F4D4
:100CE0002093050F3093060F4093070F5093080F82
:100CF00020911B0F30911C0F40911D0F50911E0F22
:100D00008091050F9091060FA091070FB091080FE9
:100D1000281739074A075B0744F42093050F3093DF
:100D2000060F4093070F5093080F8091C503882347
:100D3000F9F00091130F1091140F6091050F70914D
:100D4000060F8091070F9091080F0E9473FB20E01F
:100D500030E040E251E40E94DAFA69837A838B83BF
:100D60009C83CE0101960E94255BBC01C80161DD18
:100D70008091FE0E82FF31C00091150F1091160F69
:100D80006091050F7091060F8091070F9091080FE9
:100D90000E9473FB20E030E040E251E40E94DAFA66
:100DA000F80160837183828393830E941B6080912A
:100DB0000F0F9091100F9093C4038093C303809101
:100DC000110F9091120FA0E0B0E08093050F909367
:100DD000060FA093070FB093080F0F900F900F907E
:100DE0000F90CF91DF911F910F9108950F931F9353
:100DF000DF93CF9300D00F92CDB7DEB72091170FBE
:100E00003091180F4091190F50911A0F8091050FD2
:100E10009091060FA091070FB091080F82179307CA
:100E2000A407B50744F42093050F3093060F4093B1
:100E3000070F5093080F20911B0F30911C0F40910A
:100E40001D0F50911E0F8091050F9091060FA091DC
:100E5000070FB091080F281739074A075B0744F4BA
:100E60002093050F3093060F4093070F5093080F00
:100E70008091C5038823F9F00091130F1091140F8E
:100E80006091050F7091060F8091070F9091080FE8
:100E90000E9473FB2AE037ED43E25CE30E94DAFA3A
:100EA00069837A838B839C83CE0101960E947D5A4D
:100EB000BC01C801BEDC8091FE0E82FF31C00091F2
:100EC000150F1091160F6091050F7091060F80910C
:100ED000070F9091080F0E9473FB2AE037ED43E261
:100EE0005CE30E94DAFAF801608371838283938362
:100EF0000E941B6080910F0F9091100F9093C4037C
:100F00008093C3038091110F9091120FA0E0B0E085
:100F10008093050F9093060FA093070FB093080FCF
:100F20000F900F900F900F90CF91DF911F910F9125
:100F300008950F931F93DF93CF9300D00F92CDB7F7
:100F4000DEB72091170F3091180F4091190F509173
:100F50001A0F8091050F9091060FA091070FB09185
:100F6000080F82179307A407B50744F42093050FD1
:100F70003093060F4093070F5093080F20911B0FDB
:100F800030911C0F40911D0F50911E0F8091050F45
:100F90009091060FA091070FB091080F28173907FD
:100FA0004A075B0744F42093050F3093060F4093E4
:100FB000070F5093080F8091C5038823F9F0009123
:100FC000130F1091140F6091050F7091060F80910F
:100FD000070F9091080F0E9473FB20E030E048EC6F
:100FE00052E40E94DAFA69837A838B839C83CE0170
:100FF00001960E94AD59BC01C8011BDC8091FE0E18
:1010000082FF31C00091150F1091160F6091050FEE
:101010007091060F8091070F9091080F0E9473FB4B
:1010200020E030E048EC52E40E94DAFAF8016083F4
:101030007183828393830E941B6080910F0F909134
:10104000100F9093C4038093C3038091110F90916C
:10105000120FA0E0B0E08093050F9093060FA093CD
:10106000070FB093080F0F900F900F900F90CF9134
:10107000DF911F910F9108950F931F93DF93CF93EB
:1010800000D00F92CDB7DEB72091170F3091180F17
:101090004091190F50911A0F8091050F9091060FF2
:1010A000A091070FB091080F82179307A407B50707
:1010B00044F42093050F3093060F4093070F50938D
:1010C000080F20911B0F30911C0F40911D0F509164
:1010D0001E0F8091050F9091060FA091070FB09100
:1010E000080F281739074A075B0744F42093050FB8
:1010F0003093060F4093070F5093080F8091C5035C
:101100008823C9F00091130F1091140F6091050FFF
:101110007091060F8091070F9091080F0E9473FB4A
:1011200069837A838B839C83CE0101960E94665AE1
:10113000BC01C8017EDB8091FE0E82FF2BC00091B6
:10114000150F1091160F6091050F7091060F809189
:10115000070F9091080F0E9473FBF8016083718361
:10116000828393830E941B6080910F0F9091100FD8
:101170009093C4038093C3038091110F9091120F39
:10118000A0E0B0E08093050F9093060FA093070FA7
:10119000B093080F0F900F900F900F90CF91DF91A9
:1011A0001F910F9108950F931F93DF93CF930F9289
:1011B0000F92CDB7DEB72091170F3091180F4091E5
:1011C000190F50911A0F8091050F9091060FA09161
:1011D000070FB091080F82179307A407B50744F4CF
:1011E0002093050F3093060F4093070F5093080F7D
:1011F00020911B0F30911C0F40911D0F50911E0F1D
:101200008091050F9091060FA091070FB091080FE4
:10121000281739074A075B0744F42093050F3093DA
:10122000060F4093070F5093080F8091C503882342
:1012300089F00091130F1091140F8091050F909178
:10124000060F9A838983CE0101960E94315ABC0110
:10125000C801EFDA8091FE0E82FF22C0E091150FE7
:10126000F091160F8091050F9091060F9183808366
:101270000E941B6080910F0F9091100F9093C403F8
:101280008093C3038091110F9091120FA0E0B0E002
:101290008093050F9093060FA093070FB093080F4C
:1012A0000F900F90CF91DF911F910F910895CF92E2
:1012B000DF92EF92FF920F931F93CF93DF93082F4C
:1012C000EB01F42E6901C9010E94DB2631E1E32E16
:1012D000E81A1092FB0E10E00F5F1F4FC801880F35
:1012E000991F800F911F880F991F880F991F809356
:1012F000FC0E82EC9EE06F2D0E942EF606C082EC62
:101300009EE00E942EF62196EA94FE0164916623E7
:10131000B1F782EC9EE06AE30E942EF606C082ECF2
:101320009EE060E20E942EF6EA94EE20C1F7C6012C
:101330000E949A5CDF91CF911F910F91FF90EF90E7
:10134000DF90CF900895EF92FF920F931F936091DB
:10135000F9037091FA038091FB039091FC030E94C2
:101360006ADC6093210F7093220F8093230F909378
:10137000240F6091FD037091FE038091FF03909113
:1013800000040E9476DC6093250F7093260F8093F3
:10139000270F9093280F8091050F9091060FA09131
:1013A000070FB091080F81509048A040B04040F026
:1013B0001092050F1092060F1092070F1092080F4F
:1013C0006091050F7091060F8091070F9091080FA3
:1013D00025E030E040E050E00E94CBFE79018A0138
:1013E0008091FF0E90E0A0E0B0E0E816F9060A0751
:1013F0001B0710F42093FF0E0091FF0E8091FE0E4C
:1014000090E09695879596958795FF24F394F8221A
:1014100010E0002389F58091C5038823C1F08091F5
:10142000050F9091060FA091070FB091080F059737
:10143000A105B10528F4812F61E672E24BEF04C0EB
:10144000812F61E672E240E22BEF0E94AA5CFF204E
:1014500009F426C78091050F9091060FA091070F00
:10146000B091080F0597A105B10508F019C70E94B2
:101470001B6085EC9AE607C7013009F083C08091B4
:10148000C503882341F16091050F7091060F80918B
:10149000070F9091080F25E030E040E050E00E94F7
:1014A000CBFE213031054105510551F485E694E12B
:1014B0000E94315A9C01812F6AE572E24EE309C015
:1014C00085E694E10E94315A9C01812F6AE572E21F
:1014D00040E20E94D96CFF2009F4E2C66091050F3A
:1014E0007091060F8091070F9091080F25E030E072
:1014F00040E050E00E94CBFE21303105410551050E
:1015000009F0CEC60E941B608091C3039091C40372
:101510009093100F80930F0F8091050F9091060FFD
:101520009093120F8093110F82E08093C50383ED97
:1015300098E89093C4038093C30383E592E2909369
:10154000140F8093130F85E694E19093160F809308
:10155000150F1092170F1092180F1092190F10926A
:101560001A0F8BEE90E0A0E0B0E080931B0F9093F9
:101570001C0FA0931D0FB0931E0F809165149091C6
:10158000661485C0023009F08FC08091C50388239E
:1015900041F16091050F7091060F8091070F9091B6
:1015A000080F25E030E040E050E00E94CBFE223002
:1015B00031054105510551F487E694E10E94315A05
:1015C0009C01812F6BE472E24EE309C087E694E14F
:1015D0000E94315A9C01812F6BE472E240E20E942A
:1015E000D96CFF2009F45CC66091050F7091060F5D
:1015F0008091070F9091080F25E030E040E050E027
:101600000E94CBFE223031054105510509F048C644
:101610000E941B608091C3039091C4039093100FAC
:1016200080930F0F8091050F9091060F9093120FEA
:101630008093110F82E08093C50383ED98E8909327
:10164000C4038093C30383E492E29093140F8093C6
:10165000130F87E694E19093160F8093150F109265
:10166000170F1092180F1092190F10921A0F8BEE7D
:1016700090E0A0E0B0E080931B0F90931C0FA0932C
:101680001D0FB0931E0F8091671490916814AA27C4
:1016900097FDA095BA2F8093050F9093060FA09306
:1016A000070FB093080F3AC6033009F083C080914A
:1016B000C503882341F16091050F7091060F809159
:1016C000070F9091080F25E030E040E050E00E94C5
:1016D000CBFE233031054105510551F487E694E1F5
:1016E0000E94315A9C01812F6FE372E24EE309C0E0
:1016F00087E694E10E94315A9C01812F6FE372E2E8
:1017000040E20E94D96CFF2009F4CAC56091050F20
:101710007091060F8091070F9091080F25E030E03F
:1017200040E050E00E94CBFE2330310541055105D9
:1017300009F0B6C50E941B608091C3039091C40359
:101740009093100F80930F0F8091050F9091060FCB
:101750009093120F8093110F82E08093C50383ED65
:1017600098E89093C4038093C3038BE392E2909331
:10177000140F8093130F87E694E19093160F8093D4
:10178000150F1092170F1092180F1092190F109238
:101790001A0F87E890E0A0E0B0E080931B0F9093D1
:1017A0001C0FA0931D0FB0931E0F80916714909192
:1017B00068146DCF043009F083C08091C50388237D
:1017C00041F16091050F7091060F8091070F909184
:1017D000080F25E030E040E050E00E94CBFE2430CE
:1017E00031054105510551F484E892E10E94315AD6
:1017F0009C01812F61E372E24EE309C084E892E12B
:101800000E94315A9C01812F61E372E240E20E9402
:10181000D96CFF2009F444C56091050F7091060F43
:101820008091070F9091080F25E030E040E050E0F4
:101830000E94CBFE243031054105510509F030C529
:101840000E941B608091C3039091C4039093100F7A
:1018500080930F0F8091050F9091060F9093120FB8
:101860008093110F82E08093C50383ED98E89093F5
:10187000C4038093C30387E292E29093140F809392
:10188000130F84E892E19093160F8093150F109236
:10189000170F1092180F1092190F10921A0F8FEF46
:1018A00090E0A0E0B0E080931B0F90931C0FA093FA
:1018B0001D0FB0931E0F8091841290918512E7CE78
:1018C000053009F051C08091C503882369F160910A
:1018D000050F7091060F8091070F9091080F25E07A
:1018E00030E040E050E00E94CBFE8091850725303B
:1018F00031054105510561F4882319F426E132E2EE
:1019000002C02AE132E2812F6EE172E24EE30BC0A7
:10191000882319F42EE032E202C022E132E2812F64
:101920006EE172E240E2C3DCFF2009F4B9C46091C9
:10193000050F7091060F8091070F9091080F25E019
:1019400030E040E050E00E94CBFE253031054105FB
:10195000510509F0A5C40E941B608091850791E0A4
:10196000892780938507DAC4063009F087C0809103
:10197000C503882341F16091050F7091060F809196
:10198000070F9091080F25E030E040E050E00E9402
:10199000CBFE263031054105510551F484E993E031
:1019A0000E94665A9C01812F67E072E24EE309C0F3
:1019B00084E993E00E94665A9C01812F67E072E2FD
:1019C00040E20E94D96CFF2009F46AC46091050FBF
:1019D0007091060F8091070F9091080F25E030E07D
:1019E00040E050E00E94CBFE263031054105510514
:1019F00009F056C40E941B608091C3039091C403F8
:101A00009093100F80930F0F8091050F9091060F08
:101A10009093120F8093110F82E08093C5038CE3A3
:101A200098E89093C4038093C30380E092E290937C
:101A3000140F8093130F84E993E09093160F809313
:101A4000150F1092170F1092180F1092190F109275
:101A50001A0F8BEE90E0A0E0B0E080931B0F909304
:101A60001C0FA0931D0FB0931E0F609194037091F3
:101A70009503809196039091970379C3073009F0FD
:101A800087C08091C503882341F16091050F709153
:101A9000060F8091070F9091080F25E030E040E09D
:101AA00050E00E94CBFE273031054105510551F42D
:101AB00080E993E00E94665A9C01812F69EF71E2F0
:101AC0004EE309C080E993E00E94665A9C01812F91
:101AD00069EF71E240E20E94D96CFF2009F4E0C393
:101AE0006091050F7091060F8091070F9091080F7C
:101AF00025E030E040E050E00E94CBFE2730310589
:101B00004105510509F0CCC30E941B608091C303BD
:101B10009091C4039093100F80930F0F8091050F45
:101B20009091060F9093120F8093110F82E0809393
:101B3000C5038CE398E89093C4038093C30382EFBA
:101B400091E29093140F8093130F80E993E09093A8
:101B5000160F8093150F1092170F1092180F1092F6
:101B6000190F10921A0F8BEE90E0A0E0B0E0809376
:101B70001B0F90931C0FA0931D0FB0931E0F60912D
:101B80009003709191038091920390919303EFC21F
:101B9000083009F087C08091C503882341F1609126
:101BA000050F7091060F8091070F9091080F25E0A7
:101BB00030E040E050E00E94CBFE28303105410586
:101BC000510551F488E993E00E94AD599C01812FA1
:101BD0006AEE71E24EE309C088E993E00E94AD59D4
:101BE0009C01812F6AEE71E240E20E94D96CFF20D5
:101BF00009F456C36091050F7091060F8091070F8D
:101C00009091080F25E030E040E050E00E94CBFECC
